Component: ARM Compiler 5.06 update 6 (build 750) Tool: armlink [4d35ed]

==============================================================================

Section Cross References

    main.o(i.libuarte1_rtc_handler) refers to nrfx_rtc.o(i.nrfx_rtc_cc_set) for nrfx_rtc_cc_set
    main.o(i.libuarte1_rtc_handler) refers to nrf_libuarte_async.o(i.nrf_libuarte_async_timeout_handler) for nrf_libuarte_async_timeout_handler
    main.o(i.libuarte1_rtc_handler) refers to main.o(.bss) for .bss
    main.o(i.libuarte1_rtc_handler) refers to main.o(.constdata) for .constdata
    main.o(i.libuarte_rtc_handler) refers to nrfx_rtc.o(i.nrfx_rtc_cc_set) for nrfx_rtc_cc_set
    main.o(i.libuarte_rtc_handler) refers to nrf_libuarte_async.o(i.nrf_libuarte_async_timeout_handler) for nrf_libuarte_async_timeout_handler
    main.o(i.libuarte_rtc_handler) refers to main.o(.bss) for .bss
    main.o(i.libuarte_rtc_handler) refers to main.o(.constdata) for .constdata
    main.o(i.main) refers to nrf_drv_clock.o(i.nrf_drv_clock_init) for nrf_drv_clock_init
    main.o(i.main) refers to app_error.o(i.app_error_handler_bare) for app_error_handler_bare
    main.o(i.main) refers to nrf_drv_clock.o(i.nrf_drv_clock_lfclk_request) for nrf_drv_clock_lfclk_request
    main.o(i.main) refers to nrf_log_frontend.o(i.nrf_log_init) for nrf_log_init
    main.o(i.main) refers to nrf_log_default_backends.o(i.nrf_log_default_backends_init) for nrf_log_default_backends_init
    main.o(i.main) refers to memcpya.o(.text) for __aeabi_memcpy4
    main.o(i.main) refers to nrf_libuarte_async.o(i.nrf_libuarte_async_init) for nrf_libuarte_async_init
    main.o(i.main) refers to nrf_libuarte_async.o(i.nrf_libuarte_async_enable) for nrf_libuarte_async_enable
    main.o(i.main) refers to nrf_libuarte_async.o(i.nrf_libuarte_async_tx) for nrf_libuarte_async_tx
    main.o(i.main) refers to nrf_log_frontend.o(i.nrf_log_frontend_dequeue) for nrf_log_frontend_dequeue
    main.o(i.main) refers to app_timer2.o(i.app_timer_cnt_get) for app_timer_cnt_get
    main.o(i.main) refers to main.o(.constdata) for .constdata
    main.o(i.main) refers to main.o(i.uart_event_handler) for uart_event_handler
    main.o(i.main) refers to main.o(.data) for .data
    main.o(i.uart_event_handler) refers to nrf_libuarte_async.o(i.nrf_libuarte_async_tx) for nrf_libuarte_async_tx
    main.o(i.uart_event_handler) refers to nrf_queue.o(i.nrf_queue_push) for nrf_queue_push
    main.o(i.uart_event_handler) refers to app_error.o(i.app_error_handler_bare) for app_error_handler_bare
    main.o(i.uart_event_handler) refers to boards.o(i.bsp_board_led_invert) for bsp_board_led_invert
    main.o(i.uart_event_handler) refers to nrf_libuarte_async.o(i.nrf_libuarte_async_rx_free) for nrf_libuarte_async_rx_free
    main.o(i.uart_event_handler) refers to nrf_queue.o(i.nrf_queue_is_empty) for nrf_queue_is_empty
    main.o(i.uart_event_handler) refers to nrf_queue.o(i.nrf_queue_generic_pop) for nrf_queue_generic_pop
    main.o(i.uart_event_handler) refers to main.o(.data) for .data
    main.o(i.uart_event_handler) refers to main.o(nrf_queue) for nrf_queue
    main.o(i.uart_event_handler1) refers to nrf_libuarte_async.o(i.nrf_libuarte_async_tx) for nrf_libuarte_async_tx
    main.o(i.uart_event_handler1) refers to nrf_queue.o(i.nrf_queue_push) for nrf_queue_push
    main.o(i.uart_event_handler1) refers to app_error.o(i.app_error_handler_bare) for app_error_handler_bare
    main.o(i.uart_event_handler1) refers to boards.o(i.bsp_board_led_invert) for bsp_board_led_invert
    main.o(i.uart_event_handler1) refers to nrf_libuarte_async.o(i.nrf_libuarte_async_rx_free) for nrf_libuarte_async_rx_free
    main.o(i.uart_event_handler1) refers to nrf_queue.o(i.nrf_queue_is_empty) for nrf_queue_is_empty
    main.o(i.uart_event_handler1) refers to nrf_queue.o(i.nrf_queue_generic_pop) for nrf_queue_generic_pop
    main.o(i.uart_event_handler1) refers to main.o(.data) for .data
    main.o(i.uart_event_handler1) refers to main.o(nrf_queue) for nrf_queue
    main.o(.constdata) refers to main.o(.bss) for libuarte_libuartectrl_blk
    main.o(.constdata) refers to main.o(nrf_balloc) for libuarte_rx_pool
    main.o(.constdata) refers to main.o(nrf_queue) for libuarte_rxdata_queue
    main.o(.constdata) refers to main.o(.constdata) for libuarte_libuarte
    main.o(.constdata) refers to main.o(.bss) for libuartectrl_blk
    main.o(.constdata) refers to main.o(i.libuarte_rtc_handler) for libuarte_rtc_handler
    main.o(.constdata) refers to main.o(.constdata) for libuarte1_libuarte
    main.o(.constdata) refers to main.o(i.libuarte1_rtc_handler) for libuarte1_rtc_handler
    main.o(.constdata) refers to main.o(.bss) for libuarte1_libuartectrl_blk
    main.o(nrf_balloc) refers to main.o(.data) for libuarte_rx_pool_nrf_balloc_cb
    main.o(nrf_balloc) refers to main.o(.data) for libuarte_rx_pool_nrf_balloc_pool_stack
    main.o(nrf_balloc) refers to main.o(.bss) for libuarte_rx_pool_nrf_balloc_pool_mem
    main.o(nrf_balloc) refers to main.o(.data) for libuarte1_rx_pool_nrf_balloc_cb
    main.o(nrf_balloc) refers to main.o(.data) for libuarte1_rx_pool_nrf_balloc_pool_stack
    main.o(nrf_balloc) refers to main.o(.bss) for libuarte1_rx_pool_nrf_balloc_pool_mem
    main.o(nrf_queue) refers to main.o(.bss) for libuarte_rxdata_queue_nrf_queue_cb
    main.o(nrf_queue) refers to main.o(.bss) for libuarte_rxdata_queue_nrf_queue_buffer
    main.o(nrf_queue) refers to main.o(.bss) for libuarte1_rxdata_queue_nrf_queue_cb
    main.o(nrf_queue) refers to main.o(.bss) for libuarte1_rxdata_queue_nrf_queue_buffer
    main.o(nrf_queue) refers to main.o(.bss) for m_buf_queue_nrf_queue_cb
    main.o(nrf_queue) refers to main.o(.bss) for m_buf_queue_nrf_queue_buffer
    boards.o(i.bsp_board_init) refers to boards.o(i.nrf_gpio_pin_port_decode) for nrf_gpio_pin_port_decode
    boards.o(i.bsp_board_init) refers to boards.o(i.bsp_board_leds_off) for bsp_board_leds_off
    boards.o(i.bsp_board_init) refers to boards.o(.constdata) for .constdata
    boards.o(i.bsp_board_led_idx_to_pin) refers to boards.o(.constdata) for .constdata
    boards.o(i.bsp_board_led_invert) refers to boards.o(i.nrf_gpio_pin_port_decode) for nrf_gpio_pin_port_decode
    boards.o(i.bsp_board_led_invert) refers to boards.o(.constdata) for .constdata
    boards.o(i.bsp_board_led_off) refers to boards.o(i.nrf_gpio_pin_write) for nrf_gpio_pin_write
    boards.o(i.bsp_board_led_off) refers to boards.o(.constdata) for .constdata
    boards.o(i.bsp_board_led_on) refers to boards.o(i.nrf_gpio_pin_write) for nrf_gpio_pin_write
    boards.o(i.bsp_board_led_on) refers to boards.o(.constdata) for .constdata
    boards.o(i.bsp_board_led_state_get) refers to boards.o(i.nrf_gpio_pin_port_decode) for nrf_gpio_pin_port_decode
    boards.o(i.bsp_board_led_state_get) refers to boards.o(.constdata) for .constdata
    boards.o(i.bsp_board_leds_off) refers to boards.o(i.bsp_board_led_off) for bsp_board_led_off
    boards.o(i.bsp_board_leds_on) refers to boards.o(i.bsp_board_led_on) for bsp_board_led_on
    boards.o(i.bsp_board_pin_to_led_idx) refers to boards.o(.constdata) for .constdata
    boards.o(i.nrf_gpio_pin_write) refers to boards.o(i.nrf_gpio_pin_port_decode) for nrf_gpio_pin_port_decode
    nrf_drv_clock.o(i.clock_clk_started_notify) refers to nrf_drv_clock.o(.bss) for .bss
    nrf_drv_clock.o(i.clock_irq_handler) refers to nrf_drv_clock.o(i.clock_clk_started_notify) for clock_clk_started_notify
    nrf_drv_clock.o(i.clock_irq_handler) refers to nrf_drv_clock.o(.bss) for .bss
    nrf_drv_clock.o(i.nrf_drv_clock_hfclk_release) refers to app_util_platform.o(i.app_util_critical_region_enter) for app_util_critical_region_enter
    nrf_drv_clock.o(i.nrf_drv_clock_hfclk_release) refers to nrfx_clock.o(i.nrfx_clock_hfclk_stop) for nrfx_clock_hfclk_stop
    nrf_drv_clock.o(i.nrf_drv_clock_hfclk_release) refers to app_util_platform.o(i.app_util_critical_region_exit) for app_util_critical_region_exit
    nrf_drv_clock.o(i.nrf_drv_clock_hfclk_release) refers to nrf_drv_clock.o(.bss) for .bss
    nrf_drv_clock.o(i.nrf_drv_clock_hfclk_request) refers to app_util_platform.o(i.app_util_critical_region_enter) for app_util_critical_region_enter
    nrf_drv_clock.o(i.nrf_drv_clock_hfclk_request) refers to nrf_drv_clock.o(i.item_enqueue) for item_enqueue
    nrf_drv_clock.o(i.nrf_drv_clock_hfclk_request) refers to nrfx_clock.o(i.nrfx_clock_hfclk_start) for nrfx_clock_hfclk_start
    nrf_drv_clock.o(i.nrf_drv_clock_hfclk_request) refers to app_util_platform.o(i.app_util_critical_region_exit) for app_util_critical_region_exit
    nrf_drv_clock.o(i.nrf_drv_clock_hfclk_request) refers to nrf_drv_clock.o(.bss) for .bss
    nrf_drv_clock.o(i.nrf_drv_clock_init) refers to nrfx_clock.o(i.nrfx_clock_init) for nrfx_clock_init
    nrf_drv_clock.o(i.nrf_drv_clock_init) refers to nrfx_clock.o(i.nrfx_clock_enable) for nrfx_clock_enable
    nrf_drv_clock.o(i.nrf_drv_clock_init) refers to nrf_drv_clock.o(i.nrf_wdt_started) for nrf_wdt_started
    nrf_drv_clock.o(i.nrf_drv_clock_init) refers to nrf_drv_clock.o(.bss) for .bss
    nrf_drv_clock.o(i.nrf_drv_clock_init) refers to nrf_drv_clock.o(i.clock_irq_handler) for clock_irq_handler
    nrf_drv_clock.o(i.nrf_drv_clock_init_check) refers to nrf_drv_clock.o(.bss) for .bss
    nrf_drv_clock.o(i.nrf_drv_clock_lfclk_release) refers to app_util_platform.o(i.app_util_critical_region_enter) for app_util_critical_region_enter
    nrf_drv_clock.o(i.nrf_drv_clock_lfclk_release) refers to nrf_drv_clock.o(i.nrf_wdt_started) for nrf_wdt_started
    nrf_drv_clock.o(i.nrf_drv_clock_lfclk_release) refers to nrfx_clock.o(i.nrfx_clock_lfclk_stop) for nrfx_clock_lfclk_stop
    nrf_drv_clock.o(i.nrf_drv_clock_lfclk_release) refers to app_util_platform.o(i.app_util_critical_region_exit) for app_util_critical_region_exit
    nrf_drv_clock.o(i.nrf_drv_clock_lfclk_release) refers to nrf_drv_clock.o(.bss) for .bss
    nrf_drv_clock.o(i.nrf_drv_clock_lfclk_request) refers to app_util_platform.o(i.app_util_critical_region_enter) for app_util_critical_region_enter
    nrf_drv_clock.o(i.nrf_drv_clock_lfclk_request) refers to nrf_drv_clock.o(i.item_enqueue) for item_enqueue
    nrf_drv_clock.o(i.nrf_drv_clock_lfclk_request) refers to nrfx_clock.o(i.nrfx_clock_lfclk_start) for nrfx_clock_lfclk_start
    nrf_drv_clock.o(i.nrf_drv_clock_lfclk_request) refers to app_util_platform.o(i.app_util_critical_region_exit) for app_util_critical_region_exit
    nrf_drv_clock.o(i.nrf_drv_clock_lfclk_request) refers to nrf_drv_clock.o(.bss) for .bss
    nrf_drv_clock.o(i.nrf_drv_clock_uninit) refers to nrfx_clock.o(i.nrfx_clock_disable) for nrfx_clock_disable
    nrf_drv_clock.o(i.nrf_drv_clock_uninit) refers to nrfx_clock.o(i.nrfx_clock_uninit) for nrfx_clock_uninit
    nrf_drv_clock.o(i.nrf_drv_clock_uninit) refers to nrf_drv_clock.o(.bss) for .bss
    nrf_drv_clock.o(log_const_data) refers to nrf_drv_clock.o(.conststrlit) for .conststrlit
    nrf_nvic.o(i.sd_nvic_critical_region_enter) refers to nrf_nvic.o(.data) for .data
    nrf_nvic.o(i.sd_nvic_critical_region_exit) refers to nrf_nvic.o(.data) for .data
    nrfx_atomic.o(i.nrfx_atomic_flag_clear) refers to nrfx_atomic.o(i.nrfx_atomic_u32_and) for nrfx_atomic_u32_and
    nrfx_atomic.o(i.nrfx_atomic_flag_clear_fetch) refers to nrfx_atomic.o(i.nrfx_atomic_u32_fetch_and) for nrfx_atomic_u32_fetch_and
    nrfx_atomic.o(i.nrfx_atomic_flag_set) refers to nrfx_atomic.o(i.nrfx_atomic_u32_or) for nrfx_atomic_u32_or
    nrfx_atomic.o(i.nrfx_atomic_flag_set_fetch) refers to nrfx_atomic.o(i.nrfx_atomic_u32_fetch_or) for nrfx_atomic_u32_fetch_or
    nrfx_atomic.o(i.nrfx_atomic_u32_add) refers to nrfx_atomic.o(.emb_text) for __asm___13_nrfx_atomic_c_3bd32246__nrfx_atomic_internal_add
    nrfx_atomic.o(i.nrfx_atomic_u32_and) refers to nrfx_atomic.o(.emb_text) for __asm___13_nrfx_atomic_c_3bd32246__nrfx_atomic_internal_and
    nrfx_atomic.o(i.nrfx_atomic_u32_cmp_exch) refers to nrfx_atomic.o(.emb_text) for __asm___13_nrfx_atomic_c_3bd32246__nrfx_atomic_internal_cmp_exch
    nrfx_atomic.o(i.nrfx_atomic_u32_fetch_add) refers to nrfx_atomic.o(.emb_text) for __asm___13_nrfx_atomic_c_3bd32246__nrfx_atomic_internal_add
    nrfx_atomic.o(i.nrfx_atomic_u32_fetch_and) refers to nrfx_atomic.o(.emb_text) for __asm___13_nrfx_atomic_c_3bd32246__nrfx_atomic_internal_and
    nrfx_atomic.o(i.nrfx_atomic_u32_fetch_or) refers to nrfx_atomic.o(.emb_text) for __asm___13_nrfx_atomic_c_3bd32246__nrfx_atomic_internal_orr
    nrfx_atomic.o(i.nrfx_atomic_u32_fetch_store) refers to nrfx_atomic.o(.emb_text) for __asm___13_nrfx_atomic_c_3bd32246__nrfx_atomic_internal_mov
    nrfx_atomic.o(i.nrfx_atomic_u32_fetch_sub) refers to nrfx_atomic.o(.emb_text) for __asm___13_nrfx_atomic_c_3bd32246__nrfx_atomic_internal_sub
    nrfx_atomic.o(i.nrfx_atomic_u32_fetch_sub_hs) refers to nrfx_atomic.o(.emb_text) for __asm___13_nrfx_atomic_c_3bd32246__nrfx_atomic_internal_sub_hs
    nrfx_atomic.o(i.nrfx_atomic_u32_fetch_xor) refers to nrfx_atomic.o(.emb_text) for __asm___13_nrfx_atomic_c_3bd32246__nrfx_atomic_internal_eor
    nrfx_atomic.o(i.nrfx_atomic_u32_or) refers to nrfx_atomic.o(.emb_text) for __asm___13_nrfx_atomic_c_3bd32246__nrfx_atomic_internal_orr
    nrfx_atomic.o(i.nrfx_atomic_u32_store) refers to nrfx_atomic.o(.emb_text) for __asm___13_nrfx_atomic_c_3bd32246__nrfx_atomic_internal_mov
    nrfx_atomic.o(i.nrfx_atomic_u32_sub) refers to nrfx_atomic.o(.emb_text) for __asm___13_nrfx_atomic_c_3bd32246__nrfx_atomic_internal_sub
    nrfx_atomic.o(i.nrfx_atomic_u32_sub_hs) refers to nrfx_atomic.o(.emb_text) for __asm___13_nrfx_atomic_c_3bd32246__nrfx_atomic_internal_sub_hs
    nrfx_atomic.o(i.nrfx_atomic_u32_xor) refers to nrfx_atomic.o(.emb_text) for __asm___13_nrfx_atomic_c_3bd32246__nrfx_atomic_internal_eor
    nrfx_clock.o(i.POWER_CLOCK_IRQHandler) refers to nrfx_clock.o(i.nrf_clock_event_check) for nrf_clock_event_check
    nrfx_clock.o(i.POWER_CLOCK_IRQHandler) refers to nrfx_clock.o(i.nrf_clock_event_clear) for nrf_clock_event_clear
    nrfx_clock.o(i.POWER_CLOCK_IRQHandler) refers to nrfx_clock.o(.data) for .data
    nrfx_clock.o(i.nrfx_clock_hfclk_start) refers to nrfx_clock.o(i.nrf_clock_event_clear) for nrf_clock_event_clear
    nrfx_clock.o(i.nrfx_clock_hfclk_stop) refers to nrfx_clock.o(i.nrf_clock_event_clear) for nrf_clock_event_clear
    nrfx_clock.o(i.nrfx_clock_hfclk_stop) refers to nrfx_clock.o(.data) for .data
    nrfx_clock.o(i.nrfx_clock_init) refers to nrfx_clock.o(.data) for .data
    nrfx_clock.o(i.nrfx_clock_lfclk_start) refers to nrfx_clock.o(i.nrf_clock_event_clear) for nrf_clock_event_clear
    nrfx_clock.o(i.nrfx_clock_lfclk_stop) refers to nrfx_clock.o(i.nrf_clock_event_clear) for nrf_clock_event_clear
    nrfx_clock.o(i.nrfx_clock_uninit) refers to nrfx_clock.o(i.nrfx_clock_lfclk_stop) for nrfx_clock_lfclk_stop
    nrfx_clock.o(i.nrfx_clock_uninit) refers to nrfx_clock.o(i.nrfx_clock_hfclk_stop) for nrfx_clock_hfclk_stop
    nrfx_clock.o(i.nrfx_clock_uninit) refers to nrfx_clock.o(.data) for .data
    nrfx_clock.o(log_const_data) refers to nrfx_clock.o(.conststrlit) for .conststrlit
    nrfx_ppi.o(i.is_allocated_channel) refers to nrfx_ppi.o(.data) for .data
    nrfx_ppi.o(i.is_allocated_group) refers to nrfx_ppi.o(.data) for .data
    nrfx_ppi.o(i.nrfx_ppi_channel_alloc) refers to app_util_platform.o(i.app_util_critical_region_enter) for app_util_critical_region_enter
    nrfx_ppi.o(i.nrfx_ppi_channel_alloc) refers to nrfx_ppi.o(i.is_allocated_channel) for is_allocated_channel
    nrfx_ppi.o(i.nrfx_ppi_channel_alloc) refers to app_util_platform.o(i.app_util_critical_region_exit) for app_util_critical_region_exit
    nrfx_ppi.o(i.nrfx_ppi_channel_alloc) refers to nrf_strerror.o(i.nrf_strerror_get) for nrf_strerror_get
    nrfx_ppi.o(i.nrfx_ppi_channel_alloc) refers to nrf_log_frontend.o(i.nrf_log_frontend_std_2) for nrf_log_frontend_std_2
    nrfx_ppi.o(i.nrfx_ppi_channel_alloc) refers to nrf_log_frontend.o(i.nrf_log_frontend_std_1) for nrf_log_frontend_std_1
    nrfx_ppi.o(i.nrfx_ppi_channel_alloc) refers to nrfx_ppi.o(log_const_data) for log_const_data
    nrfx_ppi.o(i.nrfx_ppi_channel_alloc) refers to nrfx_ppi.o(.constdata) for .constdata
    nrfx_ppi.o(i.nrfx_ppi_channel_alloc) refers to nrfx_ppi.o(.data) for .data
    nrfx_ppi.o(i.nrfx_ppi_channel_assign) refers to nrfx_ppi.o(i.is_programmable_app_channel) for is_programmable_app_channel
    nrfx_ppi.o(i.nrfx_ppi_channel_assign) refers to nrfx_ppi.o(i.is_allocated_channel) for is_allocated_channel
    nrfx_ppi.o(i.nrfx_ppi_channel_assign) refers to nrf_log_frontend.o(i.nrf_log_frontend_std_3) for nrf_log_frontend_std_3
    nrfx_ppi.o(i.nrfx_ppi_channel_assign) refers to nrf_strerror.o(i.nrf_strerror_get) for nrf_strerror_get
    nrfx_ppi.o(i.nrfx_ppi_channel_assign) refers to nrf_log_frontend.o(i.nrf_log_frontend_std_2) for nrf_log_frontend_std_2
    nrfx_ppi.o(i.nrfx_ppi_channel_assign) refers to nrfx_ppi.o(log_const_data) for log_const_data
    nrfx_ppi.o(i.nrfx_ppi_channel_assign) refers to nrfx_ppi.o(.constdata) for .constdata
    nrfx_ppi.o(i.nrfx_ppi_channel_disable) refers to nrfx_ppi.o(i.is_programmable_app_channel) for is_programmable_app_channel
    nrfx_ppi.o(i.nrfx_ppi_channel_disable) refers to nrfx_ppi.o(i.is_allocated_channel) for is_allocated_channel
    nrfx_ppi.o(i.nrfx_ppi_channel_disable) refers to nrf_strerror.o(i.nrf_strerror_get) for nrf_strerror_get
    nrfx_ppi.o(i.nrfx_ppi_channel_disable) refers to nrf_log_frontend.o(i.nrf_log_frontend_std_2) for nrf_log_frontend_std_2
    nrfx_ppi.o(i.nrfx_ppi_channel_disable) refers to nrfx_ppi.o(log_const_data) for log_const_data
    nrfx_ppi.o(i.nrfx_ppi_channel_disable) refers to nrfx_ppi.o(.constdata) for .constdata
    nrfx_ppi.o(i.nrfx_ppi_channel_enable) refers to nrfx_ppi.o(i.is_programmable_app_channel) for is_programmable_app_channel
    nrfx_ppi.o(i.nrfx_ppi_channel_enable) refers to nrfx_ppi.o(i.is_allocated_channel) for is_allocated_channel
    nrfx_ppi.o(i.nrfx_ppi_channel_enable) refers to nrf_strerror.o(i.nrf_strerror_get) for nrf_strerror_get
    nrfx_ppi.o(i.nrfx_ppi_channel_enable) refers to nrf_log_frontend.o(i.nrf_log_frontend_std_2) for nrf_log_frontend_std_2
    nrfx_ppi.o(i.nrfx_ppi_channel_enable) refers to nrfx_ppi.o(log_const_data) for log_const_data
    nrfx_ppi.o(i.nrfx_ppi_channel_enable) refers to nrfx_ppi.o(.constdata) for .constdata
    nrfx_ppi.o(i.nrfx_ppi_channel_fork_assign) refers to nrfx_ppi.o(i.is_allocated_channel) for is_allocated_channel
    nrfx_ppi.o(i.nrfx_ppi_channel_fork_assign) refers to nrf_log_frontend.o(i.nrf_log_frontend_std_2) for nrf_log_frontend_std_2
    nrfx_ppi.o(i.nrfx_ppi_channel_fork_assign) refers to nrf_strerror.o(i.nrf_strerror_get) for nrf_strerror_get
    nrfx_ppi.o(i.nrfx_ppi_channel_fork_assign) refers to nrfx_ppi.o(log_const_data) for log_const_data
    nrfx_ppi.o(i.nrfx_ppi_channel_fork_assign) refers to nrfx_ppi.o(.constdata) for .constdata
    nrfx_ppi.o(i.nrfx_ppi_channel_free) refers to nrfx_ppi.o(i.is_programmable_app_channel) for is_programmable_app_channel
    nrfx_ppi.o(i.nrfx_ppi_channel_free) refers to app_util_platform.o(i.app_util_critical_region_enter) for app_util_critical_region_enter
    nrfx_ppi.o(i.nrfx_ppi_channel_free) refers to app_util_platform.o(i.app_util_critical_region_exit) for app_util_critical_region_exit
    nrfx_ppi.o(i.nrfx_ppi_channel_free) refers to nrf_strerror.o(i.nrf_strerror_get) for nrf_strerror_get
    nrfx_ppi.o(i.nrfx_ppi_channel_free) refers to nrf_log_frontend.o(i.nrf_log_frontend_std_2) for nrf_log_frontend_std_2
    nrfx_ppi.o(i.nrfx_ppi_channel_free) refers to nrfx_ppi.o(.data) for .data
    nrfx_ppi.o(i.nrfx_ppi_channel_free) refers to nrfx_ppi.o(log_const_data) for log_const_data
    nrfx_ppi.o(i.nrfx_ppi_channel_free) refers to nrfx_ppi.o(.constdata) for .constdata
    nrfx_ppi.o(i.nrfx_ppi_channels_include_in_group) refers to nrfx_ppi.o(i.is_app_group) for is_app_group
    nrfx_ppi.o(i.nrfx_ppi_channels_include_in_group) refers to nrfx_ppi.o(i.is_allocated_group) for is_allocated_group
    nrfx_ppi.o(i.nrfx_ppi_channels_include_in_group) refers to app_util_platform.o(i.app_util_critical_region_enter) for app_util_critical_region_enter
    nrfx_ppi.o(i.nrfx_ppi_channels_include_in_group) refers to app_util_platform.o(i.app_util_critical_region_exit) for app_util_critical_region_exit
    nrfx_ppi.o(i.nrfx_ppi_channels_include_in_group) refers to nrf_strerror.o(i.nrf_strerror_get) for nrf_strerror_get
    nrfx_ppi.o(i.nrfx_ppi_channels_include_in_group) refers to nrf_log_frontend.o(i.nrf_log_frontend_std_2) for nrf_log_frontend_std_2
    nrfx_ppi.o(i.nrfx_ppi_channels_include_in_group) refers to nrfx_ppi.o(log_const_data) for log_const_data
    nrfx_ppi.o(i.nrfx_ppi_channels_include_in_group) refers to nrfx_ppi.o(.constdata) for .constdata
    nrfx_ppi.o(i.nrfx_ppi_channels_remove_from_group) refers to nrfx_ppi.o(i.is_app_group) for is_app_group
    nrfx_ppi.o(i.nrfx_ppi_channels_remove_from_group) refers to nrfx_ppi.o(i.is_allocated_group) for is_allocated_group
    nrfx_ppi.o(i.nrfx_ppi_channels_remove_from_group) refers to app_util_platform.o(i.app_util_critical_region_enter) for app_util_critical_region_enter
    nrfx_ppi.o(i.nrfx_ppi_channels_remove_from_group) refers to app_util_platform.o(i.app_util_critical_region_exit) for app_util_critical_region_exit
    nrfx_ppi.o(i.nrfx_ppi_channels_remove_from_group) refers to nrf_strerror.o(i.nrf_strerror_get) for nrf_strerror_get
    nrfx_ppi.o(i.nrfx_ppi_channels_remove_from_group) refers to nrf_log_frontend.o(i.nrf_log_frontend_std_2) for nrf_log_frontend_std_2
    nrfx_ppi.o(i.nrfx_ppi_channels_remove_from_group) refers to nrfx_ppi.o(log_const_data) for log_const_data
    nrfx_ppi.o(i.nrfx_ppi_channels_remove_from_group) refers to nrfx_ppi.o(.constdata) for .constdata
    nrfx_ppi.o(i.nrfx_ppi_free_all) refers to nrfx_ppi.o(.data) for .data
    nrfx_ppi.o(i.nrfx_ppi_group_alloc) refers to app_util_platform.o(i.app_util_critical_region_enter) for app_util_critical_region_enter
    nrfx_ppi.o(i.nrfx_ppi_group_alloc) refers to nrfx_ppi.o(i.is_allocated_group) for is_allocated_group
    nrfx_ppi.o(i.nrfx_ppi_group_alloc) refers to app_util_platform.o(i.app_util_critical_region_exit) for app_util_critical_region_exit
    nrfx_ppi.o(i.nrfx_ppi_group_alloc) refers to nrf_strerror.o(i.nrf_strerror_get) for nrf_strerror_get
    nrfx_ppi.o(i.nrfx_ppi_group_alloc) refers to nrf_log_frontend.o(i.nrf_log_frontend_std_2) for nrf_log_frontend_std_2
    nrfx_ppi.o(i.nrfx_ppi_group_alloc) refers to nrf_log_frontend.o(i.nrf_log_frontend_std_1) for nrf_log_frontend_std_1
    nrfx_ppi.o(i.nrfx_ppi_group_alloc) refers to nrfx_ppi.o(log_const_data) for log_const_data
    nrfx_ppi.o(i.nrfx_ppi_group_alloc) refers to nrfx_ppi.o(.constdata) for .constdata
    nrfx_ppi.o(i.nrfx_ppi_group_alloc) refers to nrfx_ppi.o(.data) for .data
    nrfx_ppi.o(i.nrfx_ppi_group_disable) refers to nrfx_ppi.o(i.is_app_group) for is_app_group
    nrfx_ppi.o(i.nrfx_ppi_group_disable) refers to nrf_strerror.o(i.nrf_strerror_get) for nrf_strerror_get
    nrfx_ppi.o(i.nrfx_ppi_group_disable) refers to nrf_log_frontend.o(i.nrf_log_frontend_std_2) for nrf_log_frontend_std_2
    nrfx_ppi.o(i.nrfx_ppi_group_disable) refers to nrfx_ppi.o(log_const_data) for log_const_data
    nrfx_ppi.o(i.nrfx_ppi_group_disable) refers to nrfx_ppi.o(.constdata) for .constdata
    nrfx_ppi.o(i.nrfx_ppi_group_enable) refers to nrfx_ppi.o(i.is_app_group) for is_app_group
    nrfx_ppi.o(i.nrfx_ppi_group_enable) refers to nrfx_ppi.o(i.is_allocated_group) for is_allocated_group
    nrfx_ppi.o(i.nrfx_ppi_group_enable) refers to nrf_strerror.o(i.nrf_strerror_get) for nrf_strerror_get
    nrfx_ppi.o(i.nrfx_ppi_group_enable) refers to nrf_log_frontend.o(i.nrf_log_frontend_std_2) for nrf_log_frontend_std_2
    nrfx_ppi.o(i.nrfx_ppi_group_enable) refers to nrfx_ppi.o(log_const_data) for log_const_data
    nrfx_ppi.o(i.nrfx_ppi_group_enable) refers to nrfx_ppi.o(.constdata) for .constdata
    nrfx_ppi.o(i.nrfx_ppi_group_free) refers to nrfx_ppi.o(i.is_app_group) for is_app_group
    nrfx_ppi.o(i.nrfx_ppi_group_free) refers to nrfx_ppi.o(i.is_allocated_group) for is_allocated_group
    nrfx_ppi.o(i.nrfx_ppi_group_free) refers to app_util_platform.o(i.app_util_critical_region_enter) for app_util_critical_region_enter
    nrfx_ppi.o(i.nrfx_ppi_group_free) refers to app_util_platform.o(i.app_util_critical_region_exit) for app_util_critical_region_exit
    nrfx_ppi.o(i.nrfx_ppi_group_free) refers to nrf_strerror.o(i.nrf_strerror_get) for nrf_strerror_get
    nrfx_ppi.o(i.nrfx_ppi_group_free) refers to nrf_log_frontend.o(i.nrf_log_frontend_std_2) for nrf_log_frontend_std_2
    nrfx_ppi.o(i.nrfx_ppi_group_free) refers to nrfx_ppi.o(.data) for .data
    nrfx_ppi.o(i.nrfx_ppi_group_free) refers to nrfx_ppi.o(log_const_data) for log_const_data
    nrfx_ppi.o(i.nrfx_ppi_group_free) refers to nrfx_ppi.o(.constdata) for .constdata
    nrfx_ppi.o(log_const_data) refers to nrfx_ppi.o(.conststrlit) for .conststrlit
    nrfx_rtc.o(i.RTC0_IRQHandler) refers to nrfx_rtc.o(i.irq_handler) for irq_handler
    nrfx_rtc.o(i.RTC2_IRQHandler) refers to nrfx_rtc.o(i.irq_handler) for irq_handler
    nrfx_rtc.o(i.irq_handler) refers to nrfx_rtc.o(i.nrf_rtc_event_clear) for nrf_rtc_event_clear
    nrfx_rtc.o(i.irq_handler) refers to nrfx_rtc.o(.data) for .data
    nrfx_rtc.o(i.nrfx_rtc_cc_disable) refers to nrfx_rtc.o(i.nrf_rtc_event_clear) for nrf_rtc_event_clear
    nrfx_rtc.o(i.nrfx_rtc_cc_set) refers to nrfx_rtc.o(i.nrf_rtc_event_clear) for nrf_rtc_event_clear
    nrfx_rtc.o(i.nrfx_rtc_cc_set) refers to nrfx_rtc.o(.data) for .data
    nrfx_rtc.o(i.nrfx_rtc_disable) refers to nrfx_rtc.o(.data) for .data
    nrfx_rtc.o(i.nrfx_rtc_enable) refers to nrfx_rtc.o(.data) for .data
    nrfx_rtc.o(i.nrfx_rtc_init) refers to nrfx_rtc.o(.data) for .data
    nrfx_rtc.o(i.nrfx_rtc_max_ticks_get) refers to nrfx_rtc.o(.data) for .data
    nrfx_rtc.o(i.nrfx_rtc_overflow_enable) refers to nrfx_rtc.o(i.nrf_rtc_event_clear) for nrf_rtc_event_clear
    nrfx_rtc.o(i.nrfx_rtc_tick_enable) refers to nrfx_rtc.o(i.nrf_rtc_event_clear) for nrf_rtc_event_clear
    nrfx_rtc.o(i.nrfx_rtc_uninit) refers to nrfx_rtc.o(.data) for .data
    nrfx_rtc.o(log_const_data) refers to nrfx_rtc.o(.conststrlit) for .conststrlit
    nrfx_timer.o(i.TIMER0_IRQHandler) refers to nrfx_timer.o(i.irq_handler) for irq_handler
    nrfx_timer.o(i.TIMER0_IRQHandler) refers to nrfx_timer.o(.bss) for .bss
    nrfx_timer.o(i.TIMER1_IRQHandler) refers to nrfx_timer.o(i.irq_handler) for irq_handler
    nrfx_timer.o(i.TIMER1_IRQHandler) refers to nrfx_timer.o(.bss) for .bss
    nrfx_timer.o(i.irq_handler) refers to nrfx_timer.o(i.nrf_timer_event_clear) for nrf_timer_event_clear
    nrfx_timer.o(i.nrfx_timer_compare) refers to nrfx_timer.o(i.nrf_timer_event_clear) for nrf_timer_event_clear
    nrfx_timer.o(i.nrfx_timer_compare_int_enable) refers to nrfx_timer.o(i.nrf_timer_event_clear) for nrf_timer_event_clear
    nrfx_timer.o(i.nrfx_timer_disable) refers to nrfx_timer.o(.bss) for .bss
    nrfx_timer.o(i.nrfx_timer_enable) refers to nrfx_timer.o(.bss) for .bss
    nrfx_timer.o(i.nrfx_timer_extended_compare) refers to nrfx_timer.o(i.nrfx_timer_compare) for nrfx_timer_compare
    nrfx_timer.o(i.nrfx_timer_init) refers to nrfx_timer.o(i.nrf_timer_event_clear) for nrf_timer_event_clear
    nrfx_timer.o(i.nrfx_timer_init) refers to nrfx_timer.o(.bss) for .bss
    nrfx_timer.o(i.nrfx_timer_is_enabled) refers to nrfx_timer.o(.bss) for .bss
    nrfx_timer.o(i.nrfx_timer_uninit) refers to nrfx_timer.o(i.nrfx_timer_disable) for nrfx_timer_disable
    nrfx_timer.o(i.nrfx_timer_uninit) refers to nrfx_timer.o(.bss) for .bss
    nrfx_timer.o(log_const_data) refers to nrfx_timer.o(.conststrlit) for .conststrlit
    app_error.o(i.app_error_handler_bare) refers to app_error_weak.o(i.app_error_fault_handler) for app_error_fault_handler
    app_error.o(i.app_error_save_and_stop) refers to app_error.o(.bss) for .bss
    app_error_handler_keil.o(.emb_text) refers to app_error_weak.o(i.app_error_fault_handler) for app_error_fault_handler
    app_error_weak.o(i.app_error_fault_handler) refers to nrf_log_frontend.o(i.nrf_log_panic) for nrf_log_panic
    app_error_weak.o(i.app_error_fault_handler) refers to nrf_log_frontend.o(i.nrf_log_frontend_dequeue) for nrf_log_frontend_dequeue
    app_error_weak.o(i.app_error_fault_handler) refers to nrf_log_frontend.o(i.nrf_log_frontend_std_0) for nrf_log_frontend_std_0
    app_error_weak.o(i.app_error_fault_handler) refers to nrf_log_frontend.o(log_const_data) for m_nrf_log_app_logs_data_const
    app_scheduler.o(i.app_sched_event_put) refers to app_util_platform.o(i.app_util_critical_region_enter) for app_util_critical_region_enter
    app_scheduler.o(i.app_sched_event_put) refers to app_util_platform.o(i.app_util_critical_region_exit) for app_util_critical_region_exit
    app_scheduler.o(i.app_sched_event_put) refers to memcpya.o(.text) for __aeabi_memcpy
    app_scheduler.o(i.app_sched_event_put) refers to app_scheduler.o(.data) for .data
    app_scheduler.o(i.app_sched_execute) refers to app_scheduler.o(.data) for .data
    app_scheduler.o(i.app_sched_init) refers to app_scheduler.o(.data) for .data
    app_scheduler.o(i.app_sched_queue_space_get) refers to app_scheduler.o(.data) for .data
    app_timer2.o(i.app_timer_cnt_get) refers to drv_rtc.o(i.drv_rtc_counter_get) for drv_rtc_counter_get
    app_timer2.o(i.app_timer_cnt_get) refers to app_timer2.o(.data) for .data
    app_timer2.o(i.app_timer_init) refers to nrf_atfifo.o(i.nrf_atfifo_init) for nrf_atfifo_init
    app_timer2.o(i.app_timer_init) refers to drv_rtc.o(i.drv_rtc_init) for drv_rtc_init
    app_timer2.o(i.app_timer_init) refers to drv_rtc.o(i.drv_rtc_overflow_enable) for drv_rtc_overflow_enable
    app_timer2.o(i.app_timer_init) refers to drv_rtc.o(i.drv_rtc_compare_set) for drv_rtc_compare_set
    app_timer2.o(i.app_timer_init) refers to app_timer2.o(.constdata) for .constdata
    app_timer2.o(i.app_timer_init) refers to app_timer2.o(.bss) for .bss
    app_timer2.o(i.app_timer_init) refers to app_timer2.o(i.rtc_irq) for rtc_irq
    app_timer2.o(i.app_timer_init) refers to app_timer2.o(.data) for .data
    app_timer2.o(i.app_timer_pause) refers to drv_rtc.o(i.drv_rtc_stop) for drv_rtc_stop
    app_timer2.o(i.app_timer_pause) refers to app_timer2.o(.data) for .data
    app_timer2.o(i.app_timer_resume) refers to drv_rtc.o(i.drv_rtc_start) for drv_rtc_start
    app_timer2.o(i.app_timer_resume) refers to app_timer2.o(.data) for .data
    app_timer2.o(i.app_timer_start) refers to app_util_platform.o(i.app_util_critical_region_enter) for app_util_critical_region_enter
    app_timer2.o(i.app_timer_start) refers to app_util_platform.o(i.app_util_critical_region_exit) for app_util_critical_region_exit
    app_timer2.o(i.app_timer_start) refers to app_timer2.o(i.get_now) for get_now
    app_timer2.o(i.app_timer_start) refers to app_timer2.o(i.timer_req_schedule) for timer_req_schedule
    app_timer2.o(i.app_timer_stop) refers to app_util_platform.o(i.app_util_critical_region_enter) for app_util_critical_region_enter
    app_timer2.o(i.app_timer_stop) refers to app_util_platform.o(i.app_util_critical_region_exit) for app_util_critical_region_exit
    app_timer2.o(i.app_timer_stop) refers to app_timer2.o(i.timer_req_schedule) for timer_req_schedule
    app_timer2.o(i.app_timer_stop_all) refers to app_timer2.o(i.timer_req_schedule) for timer_req_schedule
    app_timer2.o(i.app_timer_stop_all) refers to app_timer2.o(.data) for .data
    app_timer2.o(i.get_now) refers to drv_rtc.o(i.drv_rtc_counter_get) for drv_rtc_counter_get
    app_timer2.o(i.get_now) refers to app_timer2.o(.data) for .data
    app_timer2.o(i.rtc_irq) refers to drv_rtc.o(i.drv_rtc_overflow_pending) for drv_rtc_overflow_pending
    app_timer2.o(i.rtc_irq) refers to drv_rtc.o(i.drv_rtc_compare_pending) for drv_rtc_compare_pending
    app_timer2.o(i.rtc_irq) refers to app_timer2.o(i.timer_expire) for timer_expire
    app_timer2.o(i.rtc_irq) refers to app_timer2.o(i.get_now) for get_now
    app_timer2.o(i.rtc_irq) refers to app_timer2.o(i.timer_req_process) for timer_req_process
    app_timer2.o(i.rtc_irq) refers to app_timer2.o(i.rtc_update) for rtc_update
    app_timer2.o(i.rtc_irq) refers to app_timer2.o(.data) for .data
    app_timer2.o(i.rtc_schedule) refers to app_timer2.o(i.get_now) for get_now
    app_timer2.o(i.rtc_schedule) refers to app_timer2.o(i.app_timer_cnt_get) for app_timer_cnt_get
    app_timer2.o(i.rtc_schedule) refers to drv_rtc.o(i.drv_rtc_windowed_compare_set) for drv_rtc_windowed_compare_set
    app_timer2.o(i.rtc_schedule) refers to drv_rtc.o(i.drv_rtc_compare_disable) for drv_rtc_compare_disable
    app_timer2.o(i.rtc_schedule) refers to app_timer2.o(i.timer_expire) for timer_expire
    app_timer2.o(i.rtc_schedule) refers to app_timer2.o(.data) for .data
    app_timer2.o(i.rtc_update) refers to nrf_sortlist.o(i.nrf_sortlist_peek) for nrf_sortlist_peek
    app_timer2.o(i.rtc_update) refers to nrf_sortlist.o(i.nrf_sortlist_add) for nrf_sortlist_add
    app_timer2.o(i.rtc_update) refers to app_timer2.o(i.sortlist_pop) for sortlist_pop
    app_timer2.o(i.rtc_update) refers to app_timer2.o(i.rtc_schedule) for rtc_schedule
    app_timer2.o(i.rtc_update) refers to drv_rtc.o(i.drv_rtc_stop) for drv_rtc_stop
    app_timer2.o(i.rtc_update) refers to drv_rtc.o(i.drv_rtc_start) for drv_rtc_start
    app_timer2.o(i.rtc_update) refers to app_timer2.o(.data) for .data
    app_timer2.o(i.rtc_update) refers to app_timer2.o(.constdata) for .constdata
    app_timer2.o(i.sortlist_pop) refers to nrf_sortlist.o(i.nrf_sortlist_pop) for nrf_sortlist_pop
    app_timer2.o(i.sortlist_pop) refers to app_timer2.o(.constdata) for .constdata
    app_timer2.o(i.timer_expire) refers to app_timer2.o(i.get_now) for get_now
    app_timer2.o(i.timer_expire) refers to app_util_platform.o(i.app_util_critical_region_enter) for app_util_critical_region_enter
    app_timer2.o(i.timer_expire) refers to app_util_platform.o(i.app_util_critical_region_exit) for app_util_critical_region_exit
    app_timer2.o(i.timer_expire) refers to nrf_sortlist.o(i.nrf_sortlist_add) for nrf_sortlist_add
    app_timer2.o(i.timer_expire) refers to app_timer2.o(.data) for .data
    app_timer2.o(i.timer_expire) refers to app_timer2.o(.constdata) for .constdata
    app_timer2.o(i.timer_req_process) refers to nrf_atfifo.o(i.nrf_atfifo_item_get) for nrf_atfifo_item_get
    app_timer2.o(i.timer_req_process) refers to nrf_sortlist.o(i.nrf_sortlist_add) for nrf_sortlist_add
    app_timer2.o(i.timer_req_process) refers to nrf_sortlist.o(i.nrf_sortlist_remove) for nrf_sortlist_remove
    app_timer2.o(i.timer_req_process) refers to app_timer2.o(i.sortlist_pop) for sortlist_pop
    app_timer2.o(i.timer_req_process) refers to nrf_atfifo.o(i.nrf_atfifo_item_free) for nrf_atfifo_item_free
    app_timer2.o(i.timer_req_process) refers to app_timer2.o(.constdata) for .constdata
    app_timer2.o(i.timer_req_process) refers to app_timer2.o(.data) for .data
    app_timer2.o(i.timer_req_schedule) refers to nrf_atfifo.o(i.nrf_atfifo_item_alloc) for nrf_atfifo_item_alloc
    app_timer2.o(i.timer_req_schedule) refers to nrf_atfifo.o(i.nrf_atfifo_item_put) for nrf_atfifo_item_put
    app_timer2.o(i.timer_req_schedule) refers to drv_rtc.o(i.drv_rtc_irq_trigger) for drv_rtc_irq_trigger
    app_timer2.o(i.timer_req_schedule) refers to app_timer2.o(.constdata) for .constdata
    app_timer2.o(i.timer_req_schedule) refers to app_timer2.o(.data) for .data
    app_timer2.o(.constdata) refers to app_timer2.o(.bss) for m_req_fifo_inst
    app_timer2.o(.constdata) refers to app_timer2.o(.data) for m_app_timer_sortlist_sortlist_cb
    app_timer2.o(.constdata) refers to app_timer2.o(i.compare_func) for compare_func
    app_timer2.o(log_const_data) refers to app_timer2.o(.conststrlit) for .conststrlit
    app_util_platform.o(i.app_util_critical_region_enter) refers to app_util_platform.o(i.app_util_disable_irq) for app_util_disable_irq
    app_util_platform.o(i.app_util_critical_region_exit) refers to app_util_platform.o(i.app_util_enable_irq) for app_util_enable_irq
    app_util_platform.o(i.app_util_disable_irq) refers to app_util_platform.o(.data) for .data
    app_util_platform.o(i.app_util_enable_irq) refers to app_util_platform.o(.data) for .data
    drv_rtc.o(i.RTC1_IRQHandler) refers to drv_rtc.o(.data) for .data
    drv_rtc.o(i.drv_rtc_compare_enable) refers to drv_rtc.o(i.evt_enable) for evt_enable
    drv_rtc.o(i.drv_rtc_compare_pending) refers to drv_rtc.o(i.evt_pending) for evt_pending
    drv_rtc.o(i.drv_rtc_compare_set) refers to drv_rtc.o(i.nrf_rtc_event_clear) for nrf_rtc_event_clear
    drv_rtc.o(i.drv_rtc_init) refers to nrf_log_frontend.o(i.nrf_log_frontend_std_0) for nrf_log_frontend_std_0
    drv_rtc.o(i.drv_rtc_init) refers to drv_rtc.o(.data) for .data
    drv_rtc.o(i.drv_rtc_init) refers to app_timer2.o(log_const_data) for m_nrf_log_app_timer_logs_data_const
    drv_rtc.o(i.drv_rtc_overflow_enable) refers to drv_rtc.o(i.evt_enable) for evt_enable
    drv_rtc.o(i.drv_rtc_overflow_pending) refers to drv_rtc.o(i.evt_pending) for evt_pending
    drv_rtc.o(i.drv_rtc_tick_enable) refers to drv_rtc.o(i.evt_enable) for evt_enable
    drv_rtc.o(i.drv_rtc_tick_pending) refers to drv_rtc.o(i.evt_pending) for evt_pending
    drv_rtc.o(i.drv_rtc_uninit) refers to nrf_log_frontend.o(i.nrf_log_frontend_std_0) for nrf_log_frontend_std_0
    drv_rtc.o(i.drv_rtc_uninit) refers to drv_rtc.o(.data) for .data
    drv_rtc.o(i.drv_rtc_uninit) refers to app_timer2.o(log_const_data) for m_nrf_log_app_timer_logs_data_const
    drv_rtc.o(i.drv_rtc_windowed_compare_set) refers to drv_rtc.o(i.nrf_rtc_event_clear) for nrf_rtc_event_clear
    drv_rtc.o(i.drv_rtc_windowed_compare_set) refers to drv_rtc.o(i.nrfx_coredep_delay_us) for nrfx_coredep_delay_us
    drv_rtc.o(i.drv_rtc_windowed_compare_set) refers to drv_rtc.o(i.evt_enable) for evt_enable
    drv_rtc.o(i.evt_pending) refers to drv_rtc.o(i.nrf_rtc_event_clear) for nrf_rtc_event_clear
    drv_rtc.o(i.nrfx_coredep_delay_us) refers to drv_rtc.o(.constdata) for .constdata
    nrf_assert.o(i.assert_nrf_callback) refers to app_error_weak.o(i.app_error_fault_handler) for app_error_fault_handler
    nrf_atfifo.o(i.nrf_atfifo_alloc_put) refers to nrf_atfifo.o(i.nrf_atfifo_item_alloc) for nrf_atfifo_item_alloc
    nrf_atfifo.o(i.nrf_atfifo_alloc_put) refers to memcpya.o(.text) for __aeabi_memcpy
    nrf_atfifo.o(i.nrf_atfifo_alloc_put) refers to nrf_atfifo.o(i.nrf_atfifo_item_put) for nrf_atfifo_item_put
    nrf_atfifo.o(i.nrf_atfifo_clear) refers to nrf_atfifo.o(.emb_text) for __asm___12_nrf_atfifo_c_51f461e1__nrf_atfifo_space_clear
    nrf_atfifo.o(i.nrf_atfifo_get_free) refers to nrf_atfifo.o(i.nrf_atfifo_item_get) for nrf_atfifo_item_get
    nrf_atfifo.o(i.nrf_atfifo_get_free) refers to memcpya.o(.text) for __aeabi_memcpy
    nrf_atfifo.o(i.nrf_atfifo_get_free) refers to nrf_atfifo.o(i.nrf_atfifo_item_free) for nrf_atfifo_item_free
    nrf_atfifo.o(i.nrf_atfifo_item_alloc) refers to nrf_atfifo.o(.emb_text) for __asm___12_nrf_atfifo_c_51f461e1__nrf_atfifo_wspace_req
    nrf_atfifo.o(i.nrf_atfifo_item_free) refers to nrf_atfifo.o(.emb_text) for __asm___12_nrf_atfifo_c_51f461e1__nrf_atfifo_rspace_close
    nrf_atfifo.o(i.nrf_atfifo_item_get) refers to nrf_atfifo.o(.emb_text) for __asm___12_nrf_atfifo_c_51f461e1__nrf_atfifo_rspace_req
    nrf_atfifo.o(i.nrf_atfifo_item_put) refers to nrf_atfifo.o(.emb_text) for __asm___12_nrf_atfifo_c_51f461e1__nrf_atfifo_wspace_close
    nrf_atomic.o(i.nrf_atomic_flag_clear) refers to nrf_atomic.o(i.nrf_atomic_u32_and) for nrf_atomic_u32_and
    nrf_atomic.o(i.nrf_atomic_flag_clear_fetch) refers to nrf_atomic.o(i.nrf_atomic_u32_fetch_and) for nrf_atomic_u32_fetch_and
    nrf_atomic.o(i.nrf_atomic_flag_set) refers to nrf_atomic.o(i.nrf_atomic_u32_or) for nrf_atomic_u32_or
    nrf_atomic.o(i.nrf_atomic_flag_set_fetch) refers to nrf_atomic.o(i.nrf_atomic_u32_fetch_or) for nrf_atomic_u32_fetch_or
    nrf_atomic.o(i.nrf_atomic_u32_add) refers to nrf_atomic.o(.emb_text) for __asm___12_nrf_atomic_c_85ca2469__nrf_atomic_internal_add
    nrf_atomic.o(i.nrf_atomic_u32_and) refers to nrf_atomic.o(.emb_text) for __asm___12_nrf_atomic_c_85ca2469__nrf_atomic_internal_and
    nrf_atomic.o(i.nrf_atomic_u32_cmp_exch) refers to nrf_atomic.o(.emb_text) for __asm___12_nrf_atomic_c_85ca2469__nrf_atomic_internal_cmp_exch
    nrf_atomic.o(i.nrf_atomic_u32_fetch_add) refers to nrf_atomic.o(.emb_text) for __asm___12_nrf_atomic_c_85ca2469__nrf_atomic_internal_add
    nrf_atomic.o(i.nrf_atomic_u32_fetch_and) refers to nrf_atomic.o(.emb_text) for __asm___12_nrf_atomic_c_85ca2469__nrf_atomic_internal_and
    nrf_atomic.o(i.nrf_atomic_u32_fetch_or) refers to nrf_atomic.o(.emb_text) for __asm___12_nrf_atomic_c_85ca2469__nrf_atomic_internal_orr
    nrf_atomic.o(i.nrf_atomic_u32_fetch_store) refers to nrf_atomic.o(.emb_text) for __asm___12_nrf_atomic_c_85ca2469__nrf_atomic_internal_mov
    nrf_atomic.o(i.nrf_atomic_u32_fetch_sub) refers to nrf_atomic.o(.emb_text) for __asm___12_nrf_atomic_c_85ca2469__nrf_atomic_internal_sub
    nrf_atomic.o(i.nrf_atomic_u32_fetch_sub_hs) refers to nrf_atomic.o(.emb_text) for __asm___12_nrf_atomic_c_85ca2469__nrf_atomic_internal_sub_hs
    nrf_atomic.o(i.nrf_atomic_u32_fetch_xor) refers to nrf_atomic.o(.emb_text) for __asm___12_nrf_atomic_c_85ca2469__nrf_atomic_internal_eor
    nrf_atomic.o(i.nrf_atomic_u32_or) refers to nrf_atomic.o(.emb_text) for __asm___12_nrf_atomic_c_85ca2469__nrf_atomic_internal_orr
    nrf_atomic.o(i.nrf_atomic_u32_store) refers to nrf_atomic.o(.emb_text) for __asm___12_nrf_atomic_c_85ca2469__nrf_atomic_internal_mov
    nrf_atomic.o(i.nrf_atomic_u32_sub) refers to nrf_atomic.o(.emb_text) for __asm___12_nrf_atomic_c_85ca2469__nrf_atomic_internal_sub
    nrf_atomic.o(i.nrf_atomic_u32_sub_hs) refers to nrf_atomic.o(.emb_text) for __asm___12_nrf_atomic_c_85ca2469__nrf_atomic_internal_sub_hs
    nrf_atomic.o(i.nrf_atomic_u32_xor) refers to nrf_atomic.o(.emb_text) for __asm___12_nrf_atomic_c_85ca2469__nrf_atomic_internal_eor
    nrf_balloc.o(i.nrf_balloc_alloc) refers to app_util_platform.o(i.app_util_critical_region_enter) for app_util_critical_region_enter
    nrf_balloc.o(i.nrf_balloc_alloc) refers to app_util_platform.o(i.app_util_critical_region_exit) for app_util_critical_region_exit
    nrf_balloc.o(i.nrf_balloc_free) refers to app_util_platform.o(i.app_util_critical_region_enter) for app_util_critical_region_enter
    nrf_balloc.o(i.nrf_balloc_free) refers to app_util_platform.o(i.app_util_critical_region_exit) for app_util_critical_region_exit
    nrf_fprintf.o(i.nrf_fprintf) refers to nrf_fprintf_format.o(i.nrf_fprintf_fmt) for nrf_fprintf_fmt
    nrf_fprintf_format.o(i.buffer_add) refers to nrf_fprintf.o(i.nrf_fprintf_buffer_flush) for nrf_fprintf_buffer_flush
    nrf_fprintf_format.o(i.int_print) refers to nrf_fprintf_format.o(i.buffer_add) for buffer_add
    nrf_fprintf_format.o(i.int_print) refers to nrf_fprintf_format.o(i.unsigned_print) for unsigned_print
    nrf_fprintf_format.o(i.nrf_fprintf_fmt) refers to nrf_fprintf_format.o(i.buffer_add) for buffer_add
    nrf_fprintf_format.o(i.nrf_fprintf_fmt) refers to nrf_fprintf.o(i.nrf_fprintf_buffer_flush) for nrf_fprintf_buffer_flush
    nrf_fprintf_format.o(i.nrf_fprintf_fmt) refers to nrf_fprintf_format.o(i.int_print) for int_print
    nrf_fprintf_format.o(i.nrf_fprintf_fmt) refers to nrf_fprintf_format.o(i.unsigned_print) for unsigned_print
    nrf_fprintf_format.o(i.nrf_fprintf_fmt) refers to strlen.o(.text) for strlen
    nrf_fprintf_format.o(i.unsigned_print) refers to nrf_fprintf_format.o(i.buffer_add) for buffer_add
    nrf_fprintf_format.o(i.unsigned_print) refers to nrf_fprintf_format.o(.constdata) for .constdata
    nrf_libuarte_async.o(i.app_timer_handler) refers to app_timer2.o(i.app_timer_cnt_get) for app_timer_cnt_get
    nrf_libuarte_async.o(i.app_timer_handler) refers to uldiv.o(.text) for __aeabi_uldivmod
    nrf_libuarte_async.o(i.app_timer_handler) refers to app_timer2.o(i.app_timer_start) for app_timer_start
    nrf_libuarte_async.o(i.app_timer_handler) refers to app_timer2.o(i.app_timer_cnt_diff_compute) for app_timer_cnt_diff_compute
    nrf_libuarte_async.o(i.app_timer_handler) refers to nrf_libuarte_async.o(i.nrf_libuarte_async_timeout_handler) for nrf_libuarte_async_timeout_handler
    nrf_libuarte_async.o(i.nrf_libuarte_async_enable) refers to nrf_balloc.o(i.nrf_balloc_alloc) for nrf_balloc_alloc
    nrf_libuarte_async.o(i.nrf_libuarte_async_enable) refers to app_error.o(i.app_error_handler_bare) for app_error_handler_bare
    nrf_libuarte_async.o(i.nrf_libuarte_async_enable) refers to nrfx_timer.o(i.nrfx_timer_clear) for nrfx_timer_clear
    nrf_libuarte_async.o(i.nrf_libuarte_async_enable) refers to nrfx_ppi.o(i.nrfx_ppi_channel_enable) for nrfx_ppi_channel_enable
    nrf_libuarte_async.o(i.nrf_libuarte_async_enable) refers to nrf_libuarte_drv.o(i.nrf_libuarte_drv_rx_start) for nrf_libuarte_drv_rx_start
    nrf_libuarte_async.o(i.nrf_libuarte_async_enable) refers to uldiv.o(.text) for __aeabi_uldivmod
    nrf_libuarte_async.o(i.nrf_libuarte_async_enable) refers to app_timer2.o(i.app_timer_start) for app_timer_start
    nrf_libuarte_async.o(i.nrf_libuarte_async_init) refers to nrfx_rtc.o(i.nrfx_rtc_init) for nrfx_rtc_init
    nrf_libuarte_async.o(i.nrf_libuarte_async_init) refers to nrfx_rtc.o(i.nrfx_rtc_cc_set) for nrfx_rtc_cc_set
    nrf_libuarte_async.o(i.nrf_libuarte_async_init) refers to nrfx_timer.o(i.nrfx_timer_init) for nrfx_timer_init
    nrf_libuarte_async.o(i.nrf_libuarte_async_init) refers to nrfx_timer.o(i.nrfx_timer_compare) for nrfx_timer_compare
    nrf_libuarte_async.o(i.nrf_libuarte_async_init) refers to app_timer2.o(i.app_timer_create) for app_timer_create
    nrf_libuarte_async.o(i.nrf_libuarte_async_init) refers to app_error.o(i.app_error_handler_bare) for app_error_handler_bare
    nrf_libuarte_async.o(i.nrf_libuarte_async_init) refers to nrfx_ppi.o(i.nrfx_ppi_channel_alloc) for nrfx_ppi_channel_alloc
    nrf_libuarte_async.o(i.nrf_libuarte_async_init) refers to nrfx_ppi.o(i.nrfx_ppi_channel_assign) for nrfx_ppi_channel_assign
    nrf_libuarte_async.o(i.nrf_libuarte_async_init) refers to nrfx_ppi.o(i.nrfx_ppi_channel_fork_assign) for nrfx_ppi_channel_fork_assign
    nrf_libuarte_async.o(i.nrf_libuarte_async_init) refers to memseta.o(.text) for __aeabi_memclr4
    nrf_libuarte_async.o(i.nrf_libuarte_async_init) refers to nrf_libuarte_drv.o(i.nrf_libuarte_drv_init) for nrf_libuarte_drv_init
    nrf_libuarte_async.o(i.nrf_libuarte_async_init) refers to nrf_balloc.o(i.nrf_balloc_init) for nrf_balloc_init
    nrf_libuarte_async.o(i.nrf_libuarte_async_init) refers to nrf_queue.o(i.nrf_queue_reset) for nrf_queue_reset
    nrf_libuarte_async.o(i.nrf_libuarte_async_init) refers to nrf_libuarte_async.o(.constdata) for .constdata
    nrf_libuarte_async.o(i.nrf_libuarte_async_init) refers to nrf_libuarte_async.o(i.tmr_evt_handler) for tmr_evt_handler
    nrf_libuarte_async.o(i.nrf_libuarte_async_init) refers to nrf_libuarte_async.o(i.app_timer_handler) for app_timer_handler
    nrf_libuarte_async.o(i.nrf_libuarte_async_init) refers to nrf_libuarte_async.o(i.uart_evt_handler) for uart_evt_handler
    nrf_libuarte_async.o(i.nrf_libuarte_async_rts_clear) refers to nrf_libuarte_drv.o(i.nrf_libuarte_drv_rts_clear) for nrf_libuarte_drv_rts_clear
    nrf_libuarte_async.o(i.nrf_libuarte_async_rts_set) refers to nrf_libuarte_drv.o(i.nrf_libuarte_drv_rts_set) for nrf_libuarte_drv_rts_set
    nrf_libuarte_async.o(i.nrf_libuarte_async_rx_free) refers to nrf_balloc.o(i.nrf_balloc_free) for nrf_balloc_free
    nrf_libuarte_async.o(i.nrf_libuarte_async_rx_free) refers to app_error.o(i.app_error_handler_bare) for app_error_handler_bare
    nrf_libuarte_async.o(i.nrf_libuarte_async_rx_free) refers to nrf_libuarte_async.o(i.rx_buffer_schedule) for rx_buffer_schedule
    nrf_libuarte_async.o(i.nrf_libuarte_async_tx) refers to nrf_libuarte_drv.o(i.nrf_libuarte_drv_tx) for nrf_libuarte_drv_tx
    nrf_libuarte_async.o(i.nrf_libuarte_async_uninit) refers to nrfx_ppi.o(i.nrfx_ppi_channel_disable) for nrfx_ppi_channel_disable
    nrf_libuarte_async.o(i.nrf_libuarte_async_uninit) refers to nrfx_ppi.o(i.nrfx_ppi_channel_free) for nrfx_ppi_channel_free
    nrf_libuarte_async.o(i.nrf_libuarte_async_uninit) refers to nrfx_rtc.o(i.nrfx_rtc_disable) for nrfx_rtc_disable
    nrf_libuarte_async.o(i.nrf_libuarte_async_uninit) refers to nrfx_rtc.o(i.nrfx_rtc_uninit) for nrfx_rtc_uninit
    nrf_libuarte_async.o(i.nrf_libuarte_async_uninit) refers to nrfx_timer.o(i.nrfx_timer_disable) for nrfx_timer_disable
    nrf_libuarte_async.o(i.nrf_libuarte_async_uninit) refers to nrfx_timer.o(i.nrfx_timer_uninit) for nrfx_timer_uninit
    nrf_libuarte_async.o(i.nrf_libuarte_async_uninit) refers to app_timer2.o(i.app_timer_stop) for app_timer_stop
    nrf_libuarte_async.o(i.nrf_libuarte_async_uninit) refers to nrf_libuarte_drv.o(i.nrf_libuarte_drv_uninit) for nrf_libuarte_drv_uninit
    nrf_libuarte_async.o(i.rx_buffer_schedule) refers to nrf_balloc.o(i.nrf_balloc_alloc) for nrf_balloc_alloc
    nrf_libuarte_async.o(i.rx_buffer_schedule) refers to nrf_queue.o(i.nrf_queue_push) for nrf_queue_push
    nrf_libuarte_async.o(i.rx_buffer_schedule) refers to nrf_libuarte_drv.o(i.nrf_libuarte_drv_rx_buf_rsp) for nrf_libuarte_drv_rx_buf_rsp
    nrf_libuarte_async.o(i.tmr_evt_handler) refers to nrf_libuarte_async.o(i.nrf_libuarte_async_timeout_handler) for nrf_libuarte_async_timeout_handler
    nrf_libuarte_async.o(i.uart_evt_handler) refers to nrf_libuarte_async.o(i.rx_buffer_schedule) for rx_buffer_schedule
    nrf_libuarte_async.o(i.uart_evt_handler) refers to nrf_queue.o(i.nrf_queue_generic_pop) for nrf_queue_generic_pop
    nrf_libuarte_async.o(i.uart_evt_handler) refers to app_error.o(i.app_error_handler_bare) for app_error_handler_bare
    nrf_libuarte_async.o(i.uart_evt_handler) refers to nrf_libuarte_async.o(.constdata) for .constdata
    nrf_libuarte_async.o(log_const_data) refers to nrf_libuarte_async.o(.conststrlit) for .conststrlit
    nrf_libuarte_drv.o(i.UARTE0_UART0_IRQHandler) refers to nrf_libuarte_drv.o(i.irq_handler) for irq_handler
    nrf_libuarte_drv.o(i.UARTE0_UART0_IRQHandler) refers to nrf_libuarte_drv.o(.data) for .data
    nrf_libuarte_drv.o(i.UARTE1_IRQHandler) refers to nrf_libuarte_drv.o(i.irq_handler) for irq_handler
    nrf_libuarte_drv.o(i.UARTE1_IRQHandler) refers to nrf_libuarte_drv.o(.data) for .data
    nrf_libuarte_drv.o(i.irq_handler) refers to nrf_libuarte_drv.o(i.nrf_uarte_event_check) for nrf_uarte_event_check
    nrf_libuarte_drv.o(i.irq_handler) refers to nrf_libuarte_drv.o(i.nrf_uarte_event_clear) for nrf_uarte_event_clear
    nrf_libuarte_drv.o(i.irq_handler) refers to nrf_libuarte_drv.o(i.tx_ppi_disable) for tx_ppi_disable
    nrf_libuarte_drv.o(i.irq_handler) refers to nrf_libuarte_drv.o(.constdata) for .constdata
    nrf_libuarte_drv.o(i.nrf_gpio_cfg) refers to nrf_libuarte_drv.o(i.nrf_gpio_pin_port_decode) for nrf_gpio_pin_port_decode
    nrf_libuarte_drv.o(i.nrf_gpio_cfg_output) refers to nrf_libuarte_drv.o(i.nrf_gpio_cfg) for nrf_gpio_cfg
    nrf_libuarte_drv.o(i.nrf_libuarte_drv_init) refers to nrf_libuarte_drv.o(i.nrf_gpio_pin_port_decode) for nrf_gpio_pin_port_decode
    nrf_libuarte_drv.o(i.nrf_libuarte_drv_init) refers to nrf_libuarte_drv.o(i.nrf_gpio_cfg_output) for nrf_gpio_cfg_output
    nrf_libuarte_drv.o(i.nrf_libuarte_drv_init) refers to nrf_libuarte_drv.o(i.nrf_gpio_cfg) for nrf_gpio_cfg
    nrf_libuarte_drv.o(i.nrf_libuarte_drv_init) refers to nrfx_timer.o(i.nrfx_timer_init) for nrfx_timer_init
    nrf_libuarte_drv.o(i.nrf_libuarte_drv_init) refers to nrf_libuarte_drv.o(i.ppi_configure) for ppi_configure
    nrf_libuarte_drv.o(i.nrf_libuarte_drv_init) refers to nrf_libuarte_drv.o(.data) for .data
    nrf_libuarte_drv.o(i.nrf_libuarte_drv_init) refers to nrf_libuarte_drv.o(.constdata) for .constdata
    nrf_libuarte_drv.o(i.nrf_libuarte_drv_init) refers to nrf_libuarte_drv.o(i.tmr_evt_handler) for tmr_evt_handler
    nrf_libuarte_drv.o(i.nrf_libuarte_drv_rx_start) refers to nrfx_timer.o(i.nrfx_timer_enable) for nrfx_timer_enable
    nrf_libuarte_drv.o(i.nrf_libuarte_drv_rx_start) refers to nrfx_timer.o(i.nrfx_timer_clear) for nrfx_timer_clear
    nrf_libuarte_drv.o(i.nrf_libuarte_drv_rx_start) refers to nrf_libuarte_drv.o(i.nrf_uarte_event_clear) for nrf_uarte_event_clear
    nrf_libuarte_drv.o(i.nrf_libuarte_drv_rx_start) refers to nrf_libuarte_drv.o(i.ppi_ch_enable) for ppi_ch_enable
    nrf_libuarte_drv.o(i.nrf_libuarte_drv_rx_stop) refers to nrf_libuarte_drv.o(i.rx_ppi_disable) for rx_ppi_disable
    nrf_libuarte_drv.o(i.nrf_libuarte_drv_tx) refers to nrf_libuarte_drv.o(i.nrf_uarte_event_clear) for nrf_uarte_event_clear
    nrf_libuarte_drv.o(i.nrf_libuarte_drv_tx) refers to nrf_libuarte_drv.o(i.nrf_uarte_event_check) for nrf_uarte_event_check
    nrf_libuarte_drv.o(i.nrf_libuarte_drv_tx) refers to nrf_libuarte_drv.o(i.ppi_ch_enable) for ppi_ch_enable
    nrf_libuarte_drv.o(i.nrf_libuarte_drv_uninit) refers to nrf_libuarte_drv.o(i.rx_ppi_disable) for rx_ppi_disable
    nrf_libuarte_drv.o(i.nrf_libuarte_drv_uninit) refers to nrf_libuarte_drv.o(i.tx_ppi_disable) for tx_ppi_disable
    nrf_libuarte_drv.o(i.nrf_libuarte_drv_uninit) refers to nrf_libuarte_drv.o(i.nrf_uarte_event_clear) for nrf_uarte_event_clear
    nrf_libuarte_drv.o(i.nrf_libuarte_drv_uninit) refers to nrf_libuarte_drv.o(i.nrf_uarte_event_check) for nrf_uarte_event_check
    nrf_libuarte_drv.o(i.nrf_libuarte_drv_uninit) refers to nrfx_timer.o(i.nrfx_timer_disable) for nrfx_timer_disable
    nrf_libuarte_drv.o(i.nrf_libuarte_drv_uninit) refers to nrfx_timer.o(i.nrfx_timer_uninit) for nrfx_timer_uninit
    nrf_libuarte_drv.o(i.nrf_libuarte_drv_uninit) refers to nrf_libuarte_drv.o(i.ppi_free) for ppi_free
    nrf_libuarte_drv.o(i.ppi_ch_disable) refers to nrfx_ppi.o(i.nrfx_ppi_channel_disable) for nrfx_ppi_channel_disable
    nrf_libuarte_drv.o(i.ppi_ch_enable) refers to nrfx_ppi.o(i.nrfx_ppi_channel_enable) for nrfx_ppi_channel_enable
    nrf_libuarte_drv.o(i.ppi_channel_configure) refers to nrfx_ppi.o(i.nrfx_ppi_channel_alloc) for nrfx_ppi_channel_alloc
    nrf_libuarte_drv.o(i.ppi_channel_configure) refers to nrfx_ppi.o(i.nrfx_ppi_channel_assign) for nrfx_ppi_channel_assign
    nrf_libuarte_drv.o(i.ppi_channel_configure) refers to nrfx_ppi.o(i.nrfx_ppi_channel_fork_assign) for nrfx_ppi_channel_fork_assign
    nrf_libuarte_drv.o(i.ppi_configure) refers to nrf_libuarte_drv.o(i.ppi_channel_configure) for ppi_channel_configure
    nrf_libuarte_drv.o(i.ppi_configure) refers to nrf_libuarte_drv.o(i.ppi_group_configure) for ppi_group_configure
    nrf_libuarte_drv.o(i.ppi_configure) refers to nrf_libuarte_drv.o(i.ppi_free) for ppi_free
    nrf_libuarte_drv.o(i.ppi_free) refers to nrfx_ppi.o(i.nrfx_ppi_channel_disable) for nrfx_ppi_channel_disable
    nrf_libuarte_drv.o(i.ppi_free) refers to nrfx_ppi.o(i.nrfx_ppi_channel_free) for nrfx_ppi_channel_free
    nrf_libuarte_drv.o(i.ppi_free) refers to nrfx_ppi.o(i.nrfx_ppi_group_free) for nrfx_ppi_group_free
    nrf_libuarte_drv.o(i.ppi_group_configure) refers to nrfx_ppi.o(i.nrfx_ppi_group_alloc) for nrfx_ppi_group_alloc
    nrf_libuarte_drv.o(i.ppi_group_configure) refers to nrfx_ppi.o(i.nrfx_ppi_channels_include_in_group) for nrfx_ppi_channels_include_in_group
    nrf_libuarte_drv.o(i.ppi_group_configure) refers to nrfx_ppi.o(i.nrfx_ppi_group_enable) for nrfx_ppi_group_enable
    nrf_libuarte_drv.o(i.rx_ppi_disable) refers to nrf_libuarte_drv.o(i.ppi_ch_disable) for ppi_ch_disable
    nrf_libuarte_drv.o(i.tx_ppi_disable) refers to nrf_libuarte_drv.o(i.ppi_ch_disable) for ppi_ch_disable
    nrf_libuarte_drv.o(log_const_data) refers to nrf_libuarte_drv.o(.conststrlit) for .conststrlit
    nrf_memobj.o(i.memobj_op) refers to memcpya.o(.text) for __aeabi_memcpy
    nrf_memobj.o(i.nrf_memobj_alloc) refers to nrf_balloc.o(i.nrf_balloc_alloc) for nrf_balloc_alloc
    nrf_memobj.o(i.nrf_memobj_alloc) refers to nrf_memobj.o(i.nrf_memobj_free) for nrf_memobj_free
    nrf_memobj.o(i.nrf_memobj_free) refers to nrf_balloc.o(i.nrf_balloc_free) for nrf_balloc_free
    nrf_memobj.o(i.nrf_memobj_get) refers to nrf_atomic.o(i.nrf_atomic_u32_add) for nrf_atomic_u32_add
    nrf_memobj.o(i.nrf_memobj_pool_init) refers to nrf_balloc.o(i.nrf_balloc_init) for nrf_balloc_init
    nrf_memobj.o(i.nrf_memobj_put) refers to nrf_atomic.o(i.nrf_atomic_u32_sub) for nrf_atomic_u32_sub
    nrf_memobj.o(i.nrf_memobj_put) refers to nrf_memobj.o(i.nrf_memobj_free) for nrf_memobj_free
    nrf_memobj.o(i.nrf_memobj_read) refers to nrf_memobj.o(i.memobj_op) for memobj_op
    nrf_memobj.o(i.nrf_memobj_write) refers to nrf_memobj.o(i.memobj_op) for memobj_op
    nrf_queue.o(i.nrf_queue_available_get) refers to nrf_queue.o(i.nrf_queue_utilization_get) for nrf_queue_utilization_get
    nrf_queue.o(i.nrf_queue_generic_pop) refers to app_util_platform.o(i.app_util_critical_region_enter) for app_util_critical_region_enter
    nrf_queue.o(i.nrf_queue_generic_pop) refers to nrf_queue.o(i.nrf_queue_is_empty) for nrf_queue_is_empty
    nrf_queue.o(i.nrf_queue_generic_pop) refers to app_util_platform.o(i.app_util_critical_region_exit) for app_util_critical_region_exit
    nrf_queue.o(i.nrf_queue_generic_pop) refers to nrf_queue.o(i.nrf_queue_next_idx) for nrf_queue_next_idx
    nrf_queue.o(i.nrf_queue_generic_pop) refers to memcpya.o(.text) for __aeabi_memcpy
    nrf_queue.o(i.nrf_queue_in) refers to app_util_platform.o(i.app_util_critical_region_enter) for app_util_critical_region_enter
    nrf_queue.o(i.nrf_queue_in) refers to nrf_queue.o(i.nrf_queue_available_get) for nrf_queue_available_get
    nrf_queue.o(i.nrf_queue_in) refers to nrf_queue.o(i.queue_write) for queue_write
    nrf_queue.o(i.nrf_queue_in) refers to app_util_platform.o(i.app_util_critical_region_exit) for app_util_critical_region_exit
    nrf_queue.o(i.nrf_queue_out) refers to app_util_platform.o(i.app_util_critical_region_enter) for app_util_critical_region_enter
    nrf_queue.o(i.nrf_queue_out) refers to nrf_queue.o(i.queue_utilization_get) for queue_utilization_get
    nrf_queue.o(i.nrf_queue_out) refers to nrf_queue.o(i.queue_read) for queue_read
    nrf_queue.o(i.nrf_queue_out) refers to app_util_platform.o(i.app_util_critical_region_exit) for app_util_critical_region_exit
    nrf_queue.o(i.nrf_queue_push) refers to app_util_platform.o(i.app_util_critical_region_enter) for app_util_critical_region_enter
    nrf_queue.o(i.nrf_queue_push) refers to nrf_queue.o(i.nrf_queue_is_full) for nrf_queue_is_full
    nrf_queue.o(i.nrf_queue_push) refers to app_util_platform.o(i.app_util_critical_region_exit) for app_util_critical_region_exit
    nrf_queue.o(i.nrf_queue_push) refers to nrf_queue.o(i.nrf_queue_next_idx) for nrf_queue_next_idx
    nrf_queue.o(i.nrf_queue_push) refers to memcpya.o(.text) for __aeabi_memcpy
    nrf_queue.o(i.nrf_queue_push) refers to nrf_queue.o(i.queue_utilization_get) for queue_utilization_get
    nrf_queue.o(i.nrf_queue_read) refers to app_util_platform.o(i.app_util_critical_region_enter) for app_util_critical_region_enter
    nrf_queue.o(i.nrf_queue_read) refers to nrf_queue.o(i.queue_utilization_get) for queue_utilization_get
    nrf_queue.o(i.nrf_queue_read) refers to nrf_queue.o(i.queue_read) for queue_read
    nrf_queue.o(i.nrf_queue_read) refers to app_util_platform.o(i.app_util_critical_region_exit) for app_util_critical_region_exit
    nrf_queue.o(i.nrf_queue_reset) refers to app_util_platform.o(i.app_util_critical_region_enter) for app_util_critical_region_enter
    nrf_queue.o(i.nrf_queue_reset) refers to app_util_platform.o(i.app_util_critical_region_exit) for app_util_critical_region_exit
    nrf_queue.o(i.nrf_queue_utilization_get) refers to app_util_platform.o(i.app_util_critical_region_enter) for app_util_critical_region_enter
    nrf_queue.o(i.nrf_queue_utilization_get) refers to nrf_queue.o(i.queue_utilization_get) for queue_utilization_get
    nrf_queue.o(i.nrf_queue_utilization_get) refers to app_util_platform.o(i.app_util_critical_region_exit) for app_util_critical_region_exit
    nrf_queue.o(i.nrf_queue_write) refers to app_util_platform.o(i.app_util_critical_region_enter) for app_util_critical_region_enter
    nrf_queue.o(i.nrf_queue_write) refers to nrf_queue.o(i.nrf_queue_available_get) for nrf_queue_available_get
    nrf_queue.o(i.nrf_queue_write) refers to app_util_platform.o(i.app_util_critical_region_exit) for app_util_critical_region_exit
    nrf_queue.o(i.nrf_queue_write) refers to nrf_queue.o(i.queue_write) for queue_write
    nrf_queue.o(i.queue_read) refers to nrf_queue.o(i.continous_items_get) for continous_items_get
    nrf_queue.o(i.queue_read) refers to memcpya.o(.text) for __aeabi_memcpy
    nrf_queue.o(i.queue_write) refers to nrf_queue.o(i.nrf_queue_available_get) for nrf_queue_available_get
    nrf_queue.o(i.queue_write) refers to nrf_queue.o(i.continous_items_get) for continous_items_get
    nrf_queue.o(i.queue_write) refers to memcpya.o(.text) for __aeabi_memcpy
    nrf_queue.o(i.queue_write) refers to nrf_queue.o(i.nrf_queue_next_idx) for nrf_queue_next_idx
    nrf_queue.o(i.queue_write) refers to nrf_queue.o(i.queue_utilization_get) for queue_utilization_get
    nrf_ringbuf.o(i.nrf_ringbuf_alloc) refers to nrf_atomic.o(i.nrf_atomic_flag_set_fetch) for nrf_atomic_flag_set_fetch
    nrf_ringbuf.o(i.nrf_ringbuf_alloc) refers to nrf_atomic.o(i.nrf_atomic_flag_clear) for nrf_atomic_flag_clear
    nrf_ringbuf.o(i.nrf_ringbuf_cpy_get) refers to nrf_atomic.o(i.nrf_atomic_flag_set_fetch) for nrf_atomic_flag_set_fetch
    nrf_ringbuf.o(i.nrf_ringbuf_cpy_get) refers to memcpya.o(.text) for __aeabi_memcpy
    nrf_ringbuf.o(i.nrf_ringbuf_cpy_get) refers to nrf_atomic.o(i.nrf_atomic_flag_clear) for nrf_atomic_flag_clear
    nrf_ringbuf.o(i.nrf_ringbuf_cpy_put) refers to nrf_atomic.o(i.nrf_atomic_flag_set_fetch) for nrf_atomic_flag_set_fetch
    nrf_ringbuf.o(i.nrf_ringbuf_cpy_put) refers to memcpya.o(.text) for __aeabi_memcpy
    nrf_ringbuf.o(i.nrf_ringbuf_cpy_put) refers to nrf_atomic.o(i.nrf_atomic_flag_clear) for nrf_atomic_flag_clear
    nrf_ringbuf.o(i.nrf_ringbuf_free) refers to nrf_atomic.o(i.nrf_atomic_flag_clear) for nrf_atomic_flag_clear
    nrf_ringbuf.o(i.nrf_ringbuf_get) refers to nrf_atomic.o(i.nrf_atomic_flag_set_fetch) for nrf_atomic_flag_set_fetch
    nrf_ringbuf.o(i.nrf_ringbuf_get) refers to nrf_atomic.o(i.nrf_atomic_flag_clear) for nrf_atomic_flag_clear
    nrf_ringbuf.o(i.nrf_ringbuf_put) refers to nrf_atomic.o(i.nrf_atomic_flag_clear_fetch) for nrf_atomic_flag_clear_fetch
    nrf_sortlist.o(log_const_data) refers to nrf_sortlist.o(.conststrlit) for .conststrlit
    nrf_strerror.o(i.nrf_strerror_find) refers to nrf_strerror.o(.constdata) for .constdata
    nrf_strerror.o(i.nrf_strerror_get) refers to nrf_strerror.o(i.nrf_strerror_find) for nrf_strerror_find
    nrf_strerror.o(i.nrf_strerror_get) refers to nrf_strerror.o(.constdata) for .constdata
    nrf_strerror.o(.constdata) refers to nrf_strerror.o(.conststring) for .conststring
    nrf_log_backend_rtt.o(i.nrf_log_backend_rtt_init) refers to segger_rtt.o(i.SEGGER_RTT_Init) for SEGGER_RTT_Init
    nrf_log_backend_rtt.o(i.nrf_log_backend_rtt_put) refers to nrf_log_backend_serial.o(i.nrf_log_backend_serial_put) for nrf_log_backend_serial_put
    nrf_log_backend_rtt.o(i.nrf_log_backend_rtt_put) refers to nrf_log_backend_rtt.o(i.serial_tx) for serial_tx
    nrf_log_backend_rtt.o(i.nrf_log_backend_rtt_put) refers to nrf_log_backend_rtt.o(.bss) for .bss
    nrf_log_backend_rtt.o(i.serial_tx) refers to segger_rtt.o(i.SEGGER_RTT_WriteNoLock) for SEGGER_RTT_WriteNoLock
    nrf_log_backend_rtt.o(i.serial_tx) refers to nrf_log_backend_rtt.o(.data) for .data
    nrf_log_backend_rtt.o(i.serial_tx) refers to nrf_log_backend_rtt.o(.constdata) for .constdata
    nrf_log_backend_rtt.o(.constdata) refers to nrf_log_backend_rtt.o(i.nrf_log_backend_rtt_put) for nrf_log_backend_rtt_put
    nrf_log_backend_rtt.o(.constdata) refers to nrf_log_backend_rtt.o(i.nrf_log_backend_rtt_panic_set) for nrf_log_backend_rtt_panic_set
    nrf_log_backend_rtt.o(.constdata) refers to nrf_log_backend_rtt.o(i.nrf_log_backend_rtt_flush) for nrf_log_backend_rtt_flush
    nrf_log_backend_serial.o(i.nrf_log_backend_serial_put) refers to nrf_memobj.o(i.nrf_memobj_get) for nrf_memobj_get
    nrf_log_backend_serial.o(i.nrf_log_backend_serial_put) refers to memseta.o(.text) for __aeabi_memclr4
    nrf_log_backend_serial.o(i.nrf_log_backend_serial_put) refers to nrf_memobj.o(i.nrf_memobj_read) for nrf_memobj_read
    nrf_log_backend_serial.o(i.nrf_log_backend_serial_put) refers to nrf_log_str_formatter.o(i.nrf_log_std_entry_process) for nrf_log_std_entry_process
    nrf_log_backend_serial.o(i.nrf_log_backend_serial_put) refers to nrf_log_str_formatter.o(i.nrf_log_hexdump_entry_process) for nrf_log_hexdump_entry_process
    nrf_log_backend_serial.o(i.nrf_log_backend_serial_put) refers to nrf_memobj.o(i.nrf_memobj_put) for nrf_memobj_put
    nrf_log_default_backends.o(i.nrf_log_default_backends_init) refers to nrf_log_backend_rtt.o(i.nrf_log_backend_rtt_init) for nrf_log_backend_rtt_init
    nrf_log_default_backends.o(i.nrf_log_default_backends_init) refers to nrf_log_frontend.o(i.nrf_log_backend_add) for nrf_log_backend_add
    nrf_log_default_backends.o(i.nrf_log_default_backends_init) refers to nrf_log_default_backends.o(log_backends) for log_backends
    nrf_log_default_backends.o(log_backends) refers to nrf_log_backend_rtt.o(.constdata) for nrf_log_backend_rtt_api
    nrf_log_default_backends.o(log_backends) refers to nrf_log_default_backends.o(.conststrlit) for .conststrlit
    nrf_log_default_backends.o(log_backends) refers to nrf_log_default_backends.o(.data) for log_backend_cb_rtt_log_backend
    nrf_log_frontend.o(i.buf_prealloc) refers to app_util_platform.o(i.app_util_critical_region_enter) for app_util_critical_region_enter
    nrf_log_frontend.o(i.buf_prealloc) refers to nrf_atomic.o(i.nrf_atomic_u32_add) for nrf_atomic_u32_add
    nrf_log_frontend.o(i.buf_prealloc) refers to nrf_log_frontend.o(i.log_skip) for log_skip
    nrf_log_frontend.o(i.buf_prealloc) refers to app_util_platform.o(i.app_util_critical_region_exit) for app_util_critical_region_exit
    nrf_log_frontend.o(i.buf_prealloc) refers to nrf_log_frontend.o(.bss) for .bss
    nrf_log_frontend.o(i.buf_prealloc) refers to nrf_log_frontend.o(.data) for .data
    nrf_log_frontend.o(i.buffer_is_empty) refers to nrf_log_frontend.o(.bss) for .bss
    nrf_log_frontend.o(i.dropped_sat16_get) refers to nrf_atomic.o(i.nrf_atomic_u32_fetch_store) for nrf_atomic_u32_fetch_store
    nrf_log_frontend.o(i.dropped_sat16_get) refers to nrf_log_frontend.o(.bss) for .bss
    nrf_log_frontend.o(i.log_skip) refers to nrf_atomic.o(i.nrf_atomic_flag_set) for nrf_atomic_flag_set
    nrf_log_frontend.o(i.log_skip) refers to nrf_log_frontend.o(i.invalid_packets_omit) for invalid_packets_omit
    nrf_log_frontend.o(i.log_skip) refers to nrf_atomic.o(i.nrf_atomic_flag_clear_fetch) for nrf_atomic_flag_clear_fetch
    nrf_log_frontend.o(i.log_skip) refers to nrf_log_frontend.o(.bss) for .bss
    nrf_log_frontend.o(i.log_skip) refers to nrf_log_frontend.o(.data) for .data
    nrf_log_frontend.o(i.module_idx_get) refers to nrf_log_frontend.o(i.nrf_log_module_cnt_get) for nrf_log_module_cnt_get
    nrf_log_frontend.o(i.nrf_log_backend_add) refers to nrf_log_frontend.o(.bss) for .bss
    nrf_log_frontend.o(i.nrf_log_backend_remove) refers to nrf_log_frontend.o(.bss) for .bss
    nrf_log_frontend.o(i.nrf_log_frontend_dequeue) refers to nrf_log_frontend.o(i.buffer_is_empty) for buffer_is_empty
    nrf_log_frontend.o(i.nrf_log_frontend_dequeue) refers to nrf_log_frontend.o(i.invalid_packets_omit) for invalid_packets_omit
    nrf_log_frontend.o(i.nrf_log_frontend_dequeue) refers to nrf_memobj.o(i.nrf_memobj_alloc) for nrf_memobj_alloc
    nrf_log_frontend.o(i.nrf_log_frontend_dequeue) refers to nrf_memobj.o(i.nrf_memobj_get) for nrf_memobj_get
    nrf_log_frontend.o(i.nrf_log_frontend_dequeue) refers to nrf_memobj.o(i.nrf_memobj_write) for nrf_memobj_write
    nrf_log_frontend.o(i.nrf_log_frontend_dequeue) refers to nrf_memobj.o(i.nrf_memobj_put) for nrf_memobj_put
    nrf_log_frontend.o(i.nrf_log_frontend_dequeue) refers to app_util_platform.o(i.app_util_critical_region_enter) for app_util_critical_region_enter
    nrf_log_frontend.o(i.nrf_log_frontend_dequeue) refers to app_util_platform.o(i.app_util_critical_region_exit) for app_util_critical_region_exit
    nrf_log_frontend.o(i.nrf_log_frontend_dequeue) refers to nrf_log_frontend.o(i.nrf_log_frontend_std_0) for nrf_log_frontend_std_0
    nrf_log_frontend.o(i.nrf_log_frontend_dequeue) refers to nrf_log_frontend.o(.bss) for .bss
    nrf_log_frontend.o(i.nrf_log_frontend_dequeue) refers to nrf_log_frontend.o(.data) for .data
    nrf_log_frontend.o(i.nrf_log_frontend_dequeue) refers to nrf_log_frontend.o(nrf_balloc) for nrf_balloc
    nrf_log_frontend.o(i.nrf_log_frontend_dequeue) refers to nrf_log_frontend.o(log_const_data) for log_const_data
    nrf_log_frontend.o(i.nrf_log_frontend_hexdump) refers to nrf_log_frontend.o(i.buf_prealloc) for buf_prealloc
    nrf_log_frontend.o(i.nrf_log_frontend_hexdump) refers to memcpya.o(.text) for __aeabi_memcpy
    nrf_log_frontend.o(i.nrf_log_frontend_hexdump) refers to nrf_log_frontend.o(i.dropped_sat16_get) for dropped_sat16_get
    nrf_log_frontend.o(i.nrf_log_frontend_hexdump) refers to nrf_log_frontend.o(i.nrf_log_frontend_dequeue) for nrf_log_frontend_dequeue
    nrf_log_frontend.o(i.nrf_log_frontend_hexdump) refers to nrf_log_frontend.o(i.log_pending_hook) for log_pending_hook
    nrf_log_frontend.o(i.nrf_log_frontend_hexdump) refers to nrf_log_frontend.o(.data) for .data
    nrf_log_frontend.o(i.nrf_log_frontend_hexdump) refers to nrf_log_frontend.o(.bss) for .bss
    nrf_log_frontend.o(i.nrf_log_frontend_std_0) refers to nrf_log_frontend.o(i.std_n) for std_n
    nrf_log_frontend.o(i.nrf_log_frontend_std_1) refers to nrf_log_frontend.o(i.std_n) for std_n
    nrf_log_frontend.o(i.nrf_log_frontend_std_2) refers to nrf_log_frontend.o(i.std_n) for std_n
    nrf_log_frontend.o(i.nrf_log_frontend_std_3) refers to nrf_log_frontend.o(i.std_n) for std_n
    nrf_log_frontend.o(i.nrf_log_frontend_std_4) refers to nrf_log_frontend.o(i.std_n) for std_n
    nrf_log_frontend.o(i.nrf_log_frontend_std_5) refers to nrf_log_frontend.o(i.std_n) for std_n
    nrf_log_frontend.o(i.nrf_log_frontend_std_6) refers to nrf_log_frontend.o(i.std_n) for std_n
    nrf_log_frontend.o(i.nrf_log_init) refers to nrf_memobj.o(i.nrf_memobj_pool_init) for nrf_memobj_pool_init
    nrf_log_frontend.o(i.nrf_log_init) refers to nrf_ringbuf.o(i.nrf_ringbuf_init) for nrf_ringbuf_init
    nrf_log_frontend.o(i.nrf_log_init) refers to nrf_log_frontend.o(.bss) for .bss
    nrf_log_frontend.o(i.nrf_log_init) refers to nrf_log_frontend.o(nrf_balloc) for nrf_balloc
    nrf_log_frontend.o(i.nrf_log_init) refers to nrf_log_frontend.o(.constdata) for .constdata
    nrf_log_frontend.o(i.nrf_log_module_filter_get) refers to nrf_log_frontend.o(i.module_idx_get) for module_idx_get
    nrf_log_frontend.o(i.nrf_log_module_name_get) refers to nrf_log_frontend.o(i.module_idx_get) for module_idx_get
    nrf_log_frontend.o(i.nrf_log_panic) refers to nrf_log_frontend.o(.bss) for .bss
    nrf_log_frontend.o(i.nrf_log_push) refers to strlen.o(.text) for strlen
    nrf_log_frontend.o(i.nrf_log_push) refers to nrf_ringbuf.o(i.nrf_ringbuf_alloc) for nrf_ringbuf_alloc
    nrf_log_frontend.o(i.nrf_log_push) refers to memcpya.o(.text) for __aeabi_memcpy
    nrf_log_frontend.o(i.nrf_log_push) refers to nrf_ringbuf.o(i.nrf_ringbuf_put) for nrf_ringbuf_put
    nrf_log_frontend.o(i.nrf_log_push) refers to nrf_ringbuf.o(i.nrf_ringbuf_free) for nrf_ringbuf_free
    nrf_log_frontend.o(i.nrf_log_push) refers to nrf_log_frontend.o(.bss) for .bss
    nrf_log_frontend.o(i.nrf_log_push) refers to nrf_log_frontend.o(.constdata) for .constdata
    nrf_log_frontend.o(i.std_n) refers to nrf_log_frontend.o(i.buf_prealloc) for buf_prealloc
    nrf_log_frontend.o(i.std_n) refers to nrf_log_frontend.o(i.dropped_sat16_get) for dropped_sat16_get
    nrf_log_frontend.o(i.std_n) refers to nrf_log_frontend.o(i.nrf_log_frontend_dequeue) for nrf_log_frontend_dequeue
    nrf_log_frontend.o(i.std_n) refers to nrf_log_frontend.o(i.log_pending_hook) for log_pending_hook
    nrf_log_frontend.o(i.std_n) refers to nrf_log_frontend.o(.data) for .data
    nrf_log_frontend.o(i.std_n) refers to nrf_log_frontend.o(.bss) for .bss
    nrf_log_frontend.o(.constdata) refers to nrf_log_frontend.o(.bss) for m_log_push_ringbuf_buf
    nrf_log_frontend.o(.constdata) refers to nrf_log_frontend.o(.bss) for m_log_push_ringbuf_cb
    nrf_log_frontend.o(log_const_data) refers to nrf_log_frontend.o(.conststrlit) for .conststrlit
    nrf_log_frontend.o(nrf_balloc) refers to nrf_log_frontend.o(.data) for log_mempool_nrf_balloc_cb
    nrf_log_frontend.o(nrf_balloc) refers to nrf_log_frontend.o(.data) for log_mempool_nrf_balloc_pool_stack
    nrf_log_frontend.o(nrf_balloc) refers to nrf_log_frontend.o(.bss) for log_mempool_nrf_balloc_pool_mem
    nrf_log_str_formatter.o(i.nrf_log_hexdump_entry_process) refers to nrf_log_str_formatter.o(i.prefix_process) for prefix_process
    nrf_log_str_formatter.o(i.nrf_log_hexdump_entry_process) refers to nrf_fprintf.o(i.nrf_fprintf) for nrf_fprintf
    nrf_log_str_formatter.o(i.nrf_log_hexdump_entry_process) refers to ctype_o.o(.text) for __rt_ctype_table
    nrf_log_str_formatter.o(i.nrf_log_hexdump_entry_process) refers to nrf_log_str_formatter.o(i.postfix_process) for postfix_process
    nrf_log_str_formatter.o(i.nrf_log_std_entry_process) refers to nrf_log_str_formatter.o(i.prefix_process) for prefix_process
    nrf_log_str_formatter.o(i.nrf_log_std_entry_process) refers to nrf_fprintf.o(i.nrf_fprintf) for nrf_fprintf
    nrf_log_str_formatter.o(i.nrf_log_std_entry_process) refers to nrf_log_str_formatter.o(i.postfix_process) for postfix_process
    nrf_log_str_formatter.o(i.nrf_log_str_formatter_timestamp_freq_set) refers to nrf_log_str_formatter.o(.data) for .data
    nrf_log_str_formatter.o(i.postfix_process) refers to nrf_fprintf.o(i.nrf_fprintf) for nrf_fprintf
    nrf_log_str_formatter.o(i.postfix_process) refers to nrf_fprintf.o(i.nrf_fprintf_buffer_flush) for nrf_fprintf_buffer_flush
    nrf_log_str_formatter.o(i.postfix_process) refers to nrf_log_str_formatter.o(.data) for .data
    nrf_log_str_formatter.o(i.prefix_process) refers to nrf_fprintf.o(i.nrf_fprintf) for nrf_fprintf
    nrf_log_str_formatter.o(i.prefix_process) refers to nrf_log_frontend.o(i.nrf_log_color_id_get) for nrf_log_color_id_get
    nrf_log_str_formatter.o(i.prefix_process) refers to nrf_log_frontend.o(i.nrf_log_module_name_get) for nrf_log_module_name_get
    nrf_log_str_formatter.o(i.prefix_process) refers to nrf_log_str_formatter.o(.data) for .data
    nrf_log_str_formatter.o(.data) refers to nrf_log_str_formatter.o(.conststring) for .conststring
    segger_rtt.o(i.SEGGER_RTT_AllocDownBuffer) refers to segger_rtt.o(i._DoInit) for _DoInit
    segger_rtt.o(i.SEGGER_RTT_AllocDownBuffer) refers to app_util_platform.o(i.app_util_critical_region_enter) for app_util_critical_region_enter
    segger_rtt.o(i.SEGGER_RTT_AllocDownBuffer) refers to app_util_platform.o(i.app_util_critical_region_exit) for app_util_critical_region_exit
    segger_rtt.o(i.SEGGER_RTT_AllocDownBuffer) refers to segger_rtt.o(.bss) for .bss
    segger_rtt.o(i.SEGGER_RTT_AllocUpBuffer) refers to segger_rtt.o(i._DoInit) for _DoInit
    segger_rtt.o(i.SEGGER_RTT_AllocUpBuffer) refers to app_util_platform.o(i.app_util_critical_region_enter) for app_util_critical_region_enter
    segger_rtt.o(i.SEGGER_RTT_AllocUpBuffer) refers to app_util_platform.o(i.app_util_critical_region_exit) for app_util_critical_region_exit
    segger_rtt.o(i.SEGGER_RTT_AllocUpBuffer) refers to segger_rtt.o(.bss) for .bss
    segger_rtt.o(i.SEGGER_RTT_ConfigDownBuffer) refers to segger_rtt.o(i._DoInit) for _DoInit
    segger_rtt.o(i.SEGGER_RTT_ConfigDownBuffer) refers to app_util_platform.o(i.app_util_critical_region_enter) for app_util_critical_region_enter
    segger_rtt.o(i.SEGGER_RTT_ConfigDownBuffer) refers to app_util_platform.o(i.app_util_critical_region_exit) for app_util_critical_region_exit
    segger_rtt.o(i.SEGGER_RTT_ConfigDownBuffer) refers to segger_rtt.o(.bss) for .bss
    segger_rtt.o(i.SEGGER_RTT_ConfigUpBuffer) refers to segger_rtt.o(i._DoInit) for _DoInit
    segger_rtt.o(i.SEGGER_RTT_ConfigUpBuffer) refers to app_util_platform.o(i.app_util_critical_region_enter) for app_util_critical_region_enter
    segger_rtt.o(i.SEGGER_RTT_ConfigUpBuffer) refers to app_util_platform.o(i.app_util_critical_region_exit) for app_util_critical_region_exit
    segger_rtt.o(i.SEGGER_RTT_ConfigUpBuffer) refers to segger_rtt.o(.bss) for .bss
    segger_rtt.o(i.SEGGER_RTT_GetKey) refers to segger_rtt.o(i.SEGGER_RTT_Read) for SEGGER_RTT_Read
    segger_rtt.o(i.SEGGER_RTT_HasData) refers to segger_rtt.o(.bss) for .bss
    segger_rtt.o(i.SEGGER_RTT_HasKey) refers to segger_rtt.o(i._DoInit) for _DoInit
    segger_rtt.o(i.SEGGER_RTT_HasKey) refers to segger_rtt.o(.bss) for .bss
    segger_rtt.o(i.SEGGER_RTT_Init) refers to segger_rtt.o(i._DoInit) for _DoInit
    segger_rtt.o(i.SEGGER_RTT_PutChar) refers to segger_rtt.o(i._DoInit) for _DoInit
    segger_rtt.o(i.SEGGER_RTT_PutChar) refers to app_util_platform.o(i.app_util_critical_region_enter) for app_util_critical_region_enter
    segger_rtt.o(i.SEGGER_RTT_PutChar) refers to app_util_platform.o(i.app_util_critical_region_exit) for app_util_critical_region_exit
    segger_rtt.o(i.SEGGER_RTT_PutChar) refers to segger_rtt.o(.bss) for .bss
    segger_rtt.o(i.SEGGER_RTT_PutCharSkip) refers to segger_rtt.o(i._DoInit) for _DoInit
    segger_rtt.o(i.SEGGER_RTT_PutCharSkip) refers to app_util_platform.o(i.app_util_critical_region_enter) for app_util_critical_region_enter
    segger_rtt.o(i.SEGGER_RTT_PutCharSkip) refers to app_util_platform.o(i.app_util_critical_region_exit) for app_util_critical_region_exit
    segger_rtt.o(i.SEGGER_RTT_PutCharSkip) refers to segger_rtt.o(.bss) for .bss
    segger_rtt.o(i.SEGGER_RTT_PutCharSkipNoLock) refers to segger_rtt.o(.bss) for .bss
    segger_rtt.o(i.SEGGER_RTT_Read) refers to app_util_platform.o(i.app_util_critical_region_enter) for app_util_critical_region_enter
    segger_rtt.o(i.SEGGER_RTT_Read) refers to segger_rtt.o(i.SEGGER_RTT_ReadNoLock) for SEGGER_RTT_ReadNoLock
    segger_rtt.o(i.SEGGER_RTT_Read) refers to app_util_platform.o(i.app_util_critical_region_exit) for app_util_critical_region_exit
    segger_rtt.o(i.SEGGER_RTT_ReadNoLock) refers to segger_rtt.o(i._DoInit) for _DoInit
    segger_rtt.o(i.SEGGER_RTT_ReadNoLock) refers to memcpya.o(.text) for __aeabi_memcpy
    segger_rtt.o(i.SEGGER_RTT_ReadNoLock) refers to segger_rtt.o(.bss) for .bss
    segger_rtt.o(i.SEGGER_RTT_SetFlagsDownBuffer) refers to segger_rtt.o(i._DoInit) for _DoInit
    segger_rtt.o(i.SEGGER_RTT_SetFlagsDownBuffer) refers to app_util_platform.o(i.app_util_critical_region_enter) for app_util_critical_region_enter
    segger_rtt.o(i.SEGGER_RTT_SetFlagsDownBuffer) refers to app_util_platform.o(i.app_util_critical_region_exit) for app_util_critical_region_exit
    segger_rtt.o(i.SEGGER_RTT_SetFlagsDownBuffer) refers to segger_rtt.o(.bss) for .bss
    segger_rtt.o(i.SEGGER_RTT_SetFlagsUpBuffer) refers to segger_rtt.o(i._DoInit) for _DoInit
    segger_rtt.o(i.SEGGER_RTT_SetFlagsUpBuffer) refers to app_util_platform.o(i.app_util_critical_region_enter) for app_util_critical_region_enter
    segger_rtt.o(i.SEGGER_RTT_SetFlagsUpBuffer) refers to app_util_platform.o(i.app_util_critical_region_exit) for app_util_critical_region_exit
    segger_rtt.o(i.SEGGER_RTT_SetFlagsUpBuffer) refers to segger_rtt.o(.bss) for .bss
    segger_rtt.o(i.SEGGER_RTT_SetNameDownBuffer) refers to segger_rtt.o(i._DoInit) for _DoInit
    segger_rtt.o(i.SEGGER_RTT_SetNameDownBuffer) refers to app_util_platform.o(i.app_util_critical_region_enter) for app_util_critical_region_enter
    segger_rtt.o(i.SEGGER_RTT_SetNameDownBuffer) refers to app_util_platform.o(i.app_util_critical_region_exit) for app_util_critical_region_exit
    segger_rtt.o(i.SEGGER_RTT_SetNameDownBuffer) refers to segger_rtt.o(.bss) for .bss
    segger_rtt.o(i.SEGGER_RTT_SetNameUpBuffer) refers to segger_rtt.o(i._DoInit) for _DoInit
    segger_rtt.o(i.SEGGER_RTT_SetNameUpBuffer) refers to app_util_platform.o(i.app_util_critical_region_enter) for app_util_critical_region_enter
    segger_rtt.o(i.SEGGER_RTT_SetNameUpBuffer) refers to app_util_platform.o(i.app_util_critical_region_exit) for app_util_critical_region_exit
    segger_rtt.o(i.SEGGER_RTT_SetNameUpBuffer) refers to segger_rtt.o(.bss) for .bss
    segger_rtt.o(i.SEGGER_RTT_SetTerminal) refers to segger_rtt.o(i._DoInit) for _DoInit
    segger_rtt.o(i.SEGGER_RTT_SetTerminal) refers to app_util_platform.o(i.app_util_critical_region_enter) for app_util_critical_region_enter
    segger_rtt.o(i.SEGGER_RTT_SetTerminal) refers to segger_rtt.o(i._GetAvailWriteSpace) for _GetAvailWriteSpace
    segger_rtt.o(i.SEGGER_RTT_SetTerminal) refers to segger_rtt.o(i._WriteNoCheck) for _WriteNoCheck
    segger_rtt.o(i.SEGGER_RTT_SetTerminal) refers to segger_rtt.o(i._WriteBlocking) for _WriteBlocking
    segger_rtt.o(i.SEGGER_RTT_SetTerminal) refers to app_util_platform.o(i.app_util_critical_region_exit) for app_util_critical_region_exit
    segger_rtt.o(i.SEGGER_RTT_SetTerminal) refers to segger_rtt.o(.bss) for .bss
    segger_rtt.o(i.SEGGER_RTT_SetTerminal) refers to segger_rtt.o(.data) for .data
    segger_rtt.o(i.SEGGER_RTT_TerminalOut) refers to segger_rtt.o(i._DoInit) for _DoInit
    segger_rtt.o(i.SEGGER_RTT_TerminalOut) refers to strlen.o(.text) for strlen
    segger_rtt.o(i.SEGGER_RTT_TerminalOut) refers to app_util_platform.o(i.app_util_critical_region_enter) for app_util_critical_region_enter
    segger_rtt.o(i.SEGGER_RTT_TerminalOut) refers to segger_rtt.o(i._GetAvailWriteSpace) for _GetAvailWriteSpace
    segger_rtt.o(i.SEGGER_RTT_TerminalOut) refers to segger_rtt.o(i._PostTerminalSwitch) for _PostTerminalSwitch
    segger_rtt.o(i.SEGGER_RTT_TerminalOut) refers to segger_rtt.o(i._WriteBlocking) for _WriteBlocking
    segger_rtt.o(i.SEGGER_RTT_TerminalOut) refers to app_util_platform.o(i.app_util_critical_region_exit) for app_util_critical_region_exit
    segger_rtt.o(i.SEGGER_RTT_TerminalOut) refers to segger_rtt.o(.bss) for .bss
    segger_rtt.o(i.SEGGER_RTT_TerminalOut) refers to segger_rtt.o(.data) for .data
    segger_rtt.o(i.SEGGER_RTT_WaitKey) refers to segger_rtt.o(i.SEGGER_RTT_GetKey) for SEGGER_RTT_GetKey
    segger_rtt.o(i.SEGGER_RTT_Write) refers to segger_rtt.o(i._DoInit) for _DoInit
    segger_rtt.o(i.SEGGER_RTT_Write) refers to app_util_platform.o(i.app_util_critical_region_enter) for app_util_critical_region_enter
    segger_rtt.o(i.SEGGER_RTT_Write) refers to segger_rtt.o(i.SEGGER_RTT_WriteNoLock) for SEGGER_RTT_WriteNoLock
    segger_rtt.o(i.SEGGER_RTT_Write) refers to app_util_platform.o(i.app_util_critical_region_exit) for app_util_critical_region_exit
    segger_rtt.o(i.SEGGER_RTT_Write) refers to segger_rtt.o(.bss) for .bss
    segger_rtt.o(i.SEGGER_RTT_WriteNoLock) refers to segger_rtt.o(i._GetAvailWriteSpace) for _GetAvailWriteSpace
    segger_rtt.o(i.SEGGER_RTT_WriteNoLock) refers to segger_rtt.o(i._WriteNoCheck) for _WriteNoCheck
    segger_rtt.o(i.SEGGER_RTT_WriteNoLock) refers to segger_rtt.o(i._WriteBlocking) for _WriteBlocking
    segger_rtt.o(i.SEGGER_RTT_WriteNoLock) refers to segger_rtt.o(.bss) for .bss
    segger_rtt.o(i.SEGGER_RTT_WriteSkipNoLock) refers to memcpya.o(.text) for __aeabi_memcpy
    segger_rtt.o(i.SEGGER_RTT_WriteSkipNoLock) refers to segger_rtt.o(.bss) for .bss
    segger_rtt.o(i.SEGGER_RTT_WriteString) refers to strlen.o(.text) for strlen
    segger_rtt.o(i.SEGGER_RTT_WriteString) refers to segger_rtt.o(i.SEGGER_RTT_Write) for SEGGER_RTT_Write
    segger_rtt.o(i.SEGGER_RTT_WriteWithOverwriteNoLock) refers to memcpya.o(.text) for __aeabi_memcpy
    segger_rtt.o(i.SEGGER_RTT_WriteWithOverwriteNoLock) refers to segger_rtt.o(.bss) for .bss
    segger_rtt.o(i._DoInit) refers to strcpy.o(.text) for strcpy
    segger_rtt.o(i._DoInit) refers to segger_rtt.o(.bss) for .bss
    segger_rtt.o(i._PostTerminalSwitch) refers to segger_rtt.o(i._WriteBlocking) for _WriteBlocking
    segger_rtt.o(i._PostTerminalSwitch) refers to segger_rtt.o(.data) for .data
    segger_rtt.o(i._WriteBlocking) refers to memcpya.o(.text) for __aeabi_memcpy
    segger_rtt.o(i._WriteNoCheck) refers to memcpya.o(.text) for __aeabi_memcpy
    segger_rtt_syscalls_keil.o(i._sys_open) refers to strcmp.o(.text) for strcmp
    segger_rtt_syscalls_keil.o(i._sys_open) refers to segger_rtt_syscalls_keil.o(.constdata) for .constdata
    segger_rtt_syscalls_keil.o(i._sys_write) refers to segger_rtt.o(i.SEGGER_RTT_Write) for SEGGER_RTT_Write
    segger_rtt_syscalls_keil.o(i._ttywrch) refers to fputc.o(i.fputc) for fputc
    segger_rtt_syscalls_keil.o(i._ttywrch) refers to fflush.o(.text) for fflush
    segger_rtt_syscalls_keil.o(i._ttywrch) refers to stdout.o(.data) for __stdout
    segger_rtt_printf.o(i.SEGGER_RTT_printf) refers to segger_rtt_printf.o(i.SEGGER_RTT_vprintf) for SEGGER_RTT_vprintf
    segger_rtt_printf.o(i.SEGGER_RTT_vprintf) refers to segger_rtt_printf.o(i._StoreChar) for _StoreChar
    segger_rtt_printf.o(i.SEGGER_RTT_vprintf) refers to segger_rtt_printf.o(i._PrintInt) for _PrintInt
    segger_rtt_printf.o(i.SEGGER_RTT_vprintf) refers to segger_rtt_printf.o(i._PrintUnsigned) for _PrintUnsigned
    segger_rtt_printf.o(i.SEGGER_RTT_vprintf) refers to segger_rtt.o(i.SEGGER_RTT_Write) for SEGGER_RTT_Write
    segger_rtt_printf.o(i._PrintInt) refers to segger_rtt_printf.o(i._StoreChar) for _StoreChar
    segger_rtt_printf.o(i._PrintInt) refers to segger_rtt_printf.o(i._PrintUnsigned) for _PrintUnsigned
    segger_rtt_printf.o(i._PrintUnsigned) refers to segger_rtt_printf.o(i._StoreChar) for _StoreChar
    segger_rtt_printf.o(i._PrintUnsigned) refers to segger_rtt_printf.o(.constdata) for .constdata
    segger_rtt_printf.o(i._StoreChar) refers to segger_rtt.o(i.SEGGER_RTT_Write) for SEGGER_RTT_Write
    arm_startup_nrf52840.o(RESET) refers to arm_startup_nrf52840.o(STACK) for __initial_sp
    arm_startup_nrf52840.o(RESET) refers to arm_startup_nrf52840.o(.text) for Reset_Handler
    arm_startup_nrf52840.o(RESET) refers to nrfx_clock.o(i.POWER_CLOCK_IRQHandler) for POWER_CLOCK_IRQHandler
    arm_startup_nrf52840.o(RESET) refers to nrf_libuarte_drv.o(i.UARTE0_UART0_IRQHandler) for UARTE0_UART0_IRQHandler
    arm_startup_nrf52840.o(RESET) refers to nrfx_timer.o(i.TIMER0_IRQHandler) for TIMER0_IRQHandler
    arm_startup_nrf52840.o(RESET) refers to nrfx_timer.o(i.TIMER1_IRQHandler) for TIMER1_IRQHandler
    arm_startup_nrf52840.o(RESET) refers to nrfx_rtc.o(i.RTC0_IRQHandler) for RTC0_IRQHandler
    arm_startup_nrf52840.o(RESET) refers to drv_rtc.o(i.RTC1_IRQHandler) for RTC1_IRQHandler
    arm_startup_nrf52840.o(RESET) refers to nrfx_rtc.o(i.RTC2_IRQHandler) for RTC2_IRQHandler
    arm_startup_nrf52840.o(RESET) refers to nrf_libuarte_drv.o(i.UARTE1_IRQHandler) for UARTE1_IRQHandler
    arm_startup_nrf52840.o(.text) refers to system_nrf52.o(i.SystemInit) for SystemInit
    arm_startup_nrf52840.o(.text) refers to entry.o(.ARM.Collect$$$$00000000) for __main
    system_nrf52.o(i.SystemCoreClockUpdate) refers to system_nrf52.o(.data) for .data
    system_nrf52.o(i.SystemInit) refers to system_nrf52.o(i.nvmc_config) for nvmc_config
    system_nrf52.o(i.SystemInit) refers to system_nrf52.o(.data) for .data
    entry.o(.ARM.Collect$$$$00000000) refers (Special) to entry10a.o(.ARM.Collect$$$$0000000D) for __rt_final_cpp
    entry.o(.ARM.Collect$$$$00000000) refers (Special) to entry11a.o(.ARM.Collect$$$$0000000F) for __rt_final_exit
    entry.o(.ARM.Collect$$$$00000000) refers (Special) to entry7b.o(.ARM.Collect$$$$00000008) for _main_clock
    entry.o(.ARM.Collect$$$$00000000) refers (Special) to entry8b.o(.ARM.Collect$$$$0000000A) for _main_cpp_init
    entry.o(.ARM.Collect$$$$00000000) refers (Special) to entry9a.o(.ARM.Collect$$$$0000000B) for _main_init
    entry.o(.ARM.Collect$$$$00000000) refers (Special) to entry5.o(.ARM.Collect$$$$00000004) for _main_scatterload
    entry.o(.ARM.Collect$$$$00000000) refers (Special) to entry2.o(.ARM.Collect$$$$00000001) for _main_stk
    fputc.o(i.fputc) refers (Special) to iusesemip.o(.text) for __I$use$semihosting$fputc
    fputc.o(i.fputc) refers (Special) to semi.o(.text) for __semihosting_library_function
    uldiv.o(.text) refers to llushr.o(.text) for __aeabi_llsr
    uldiv.o(.text) refers to llshl.o(.text) for __aeabi_llsl
    ctype_o.o(.text) refers to ctype_o.o(.constdata) for .constdata
    ctype_o.o(.constdata) refers to ctype_o.o(.constdata) for __ctype_table
    isalnum_o.o(.text) refers to ctype_o.o(.text) for __rt_ctype_table
    isalpha_o.o(.text) refers to ctype_o.o(.text) for __rt_ctype_table
    isblank_o.o(.text) refers to ctype_o.o(.constdata) for __ctype_table
    iscntrl_o.o(.text) refers to ctype_o.o(.text) for __rt_ctype_table
    isdigit_o.o(.text) refers to ctype_o.o(.text) for __rt_ctype_table
    isgraph_o.o(.text) refers to ctype_o.o(.text) for __rt_ctype_table
    islower_o.o(.text) refers to ctype_o.o(.text) for __rt_ctype_table
    isprint_o.o(.text) refers to ctype_o.o(.text) for __rt_ctype_table
    ispunct_o.o(.text) refers to ctype_o.o(.text) for __rt_ctype_table
    isspace_o.o(.text) refers to ctype_o.o(.text) for __rt_ctype_table
    isupper_o.o(.text) refers to ctype_o.o(.text) for __rt_ctype_table
    isxdigit_o.o(.text) refers to ctype_o.o(.text) for __rt_ctype_table
    entry2.o(.ARM.Collect$$$$00000001) refers to entry2.o(.ARM.Collect$$$$00002712) for __lit__00000000
    entry2.o(.ARM.Collect$$$$00002712) refers to arm_startup_nrf52840.o(STACK) for __initial_sp
    entry2.o(__vectab_stack_and_reset_area) refers to arm_startup_nrf52840.o(STACK) for __initial_sp
    entry2.o(__vectab_stack_and_reset_area) refers to entry.o(.ARM.Collect$$$$00000000) for __main
    entry5.o(.ARM.Collect$$$$00000004) refers to init.o(.text) for __scatterload
    entry9a.o(.ARM.Collect$$$$0000000B) refers to main.o(i.main) for main
    entry9b.o(.ARM.Collect$$$$0000000C) refers to main.o(i.main) for main
    init.o(.text) refers to entry5.o(.ARM.Collect$$$$00000004) for __main_after_scatterload


==============================================================================

Removing Unused input sections from the image.

    Removing main.o(.rev16_text), (4 bytes).
    Removing main.o(.revsh_text), (4 bytes).
    Removing main.o(.rrx_text), (6 bytes).
    Removing main.o(i.uart_event_handler1), (140 bytes).
    Removing boards.o(.rev16_text), (4 bytes).
    Removing boards.o(.revsh_text), (4 bytes).
    Removing boards.o(.rrx_text), (6 bytes).
    Removing boards.o(i.bsp_board_init), (52 bytes).
    Removing boards.o(i.bsp_board_led_idx_to_pin), (12 bytes).
    Removing boards.o(i.bsp_board_led_off), (16 bytes).
    Removing boards.o(i.bsp_board_led_on), (16 bytes).
    Removing boards.o(i.bsp_board_led_state_get), (40 bytes).
    Removing boards.o(i.bsp_board_leds_off), (18 bytes).
    Removing boards.o(i.bsp_board_leds_on), (18 bytes).
    Removing boards.o(i.bsp_board_pin_to_led_idx), (36 bytes).
    Removing boards.o(i.nrf_gpio_pin_write), (38 bytes).
    Removing nrf_drv_clock.o(.rev16_text), (4 bytes).
    Removing nrf_drv_clock.o(.revsh_text), (4 bytes).
    Removing nrf_drv_clock.o(.rrx_text), (6 bytes).
    Removing nrf_drv_clock.o(i.nrf_drv_clock_calibration_abort), (4 bytes).
    Removing nrf_drv_clock.o(i.nrf_drv_clock_calibration_start), (4 bytes).
    Removing nrf_drv_clock.o(i.nrf_drv_clock_hfclk_is_running), (28 bytes).
    Removing nrf_drv_clock.o(i.nrf_drv_clock_hfclk_release), (44 bytes).
    Removing nrf_drv_clock.o(i.nrf_drv_clock_hfclk_request), (72 bytes).
    Removing nrf_drv_clock.o(i.nrf_drv_clock_init_check), (12 bytes).
    Removing nrf_drv_clock.o(i.nrf_drv_clock_is_calibrating), (4 bytes).
    Removing nrf_drv_clock.o(i.nrf_drv_clock_lfclk_is_running), (16 bytes).
    Removing nrf_drv_clock.o(i.nrf_drv_clock_lfclk_release), (48 bytes).
    Removing nrf_drv_clock.o(i.nrf_drv_clock_uninit), (24 bytes).
    Removing nrf_drv_clock.o(.constdata), (19 bytes).
    Removing nrf_drv_clock.o(.constdata), (32 bytes).
    Removing nrf_drv_clock.o(.constdata), (32 bytes).
    Removing nrf_drv_clock.o(.constdata), (29 bytes).
    Removing nrf_nvic.o(.rev16_text), (4 bytes).
    Removing nrf_nvic.o(.revsh_text), (4 bytes).
    Removing nrf_nvic.o(.rrx_text), (6 bytes).
    Removing nrf_nvic.o(i.sd_nvic_ClearPendingIRQ), (28 bytes).
    Removing nrf_nvic.o(i.sd_nvic_DisableIRQ), (36 bytes).
    Removing nrf_nvic.o(i.sd_nvic_EnableIRQ), (28 bytes).
    Removing nrf_nvic.o(i.sd_nvic_GetPendingIRQ), (46 bytes).
    Removing nrf_nvic.o(i.sd_nvic_GetPriority), (40 bytes).
    Removing nrf_nvic.o(i.sd_nvic_SetPendingIRQ), (28 bytes).
    Removing nrf_nvic.o(i.sd_nvic_SetPriority), (34 bytes).
    Removing nrf_nvic.o(i.sd_nvic_SystemReset), (36 bytes).
    Removing nrf_nvic.o(i.sd_nvic_critical_region_enter), (28 bytes).
    Removing nrf_nvic.o(i.sd_nvic_critical_region_exit), (24 bytes).
    Removing nrf_nvic.o(.data), (1 bytes).
    Removing nrf_soc.o(.rev16_text), (4 bytes).
    Removing nrf_soc.o(.revsh_text), (4 bytes).
    Removing nrf_soc.o(.rrx_text), (6 bytes).
    Removing nrf_soc.o(i.sd_app_evt_wait), (6 bytes).
    Removing nrfx_atomic.o(.rev16_text), (4 bytes).
    Removing nrfx_atomic.o(.revsh_text), (4 bytes).
    Removing nrfx_atomic.o(.rrx_text), (6 bytes).
    Removing nrfx_atomic.o(.emb_text), (226 bytes).
    Removing nrfx_atomic.o(i.nrfx_atomic_flag_clear), (6 bytes).
    Removing nrfx_atomic.o(i.nrfx_atomic_flag_clear_fetch), (6 bytes).
    Removing nrfx_atomic.o(i.nrfx_atomic_flag_set), (6 bytes).
    Removing nrfx_atomic.o(i.nrfx_atomic_flag_set_fetch), (6 bytes).
    Removing nrfx_atomic.o(i.nrfx_atomic_u32_add), (12 bytes).
    Removing nrfx_atomic.o(i.nrfx_atomic_u32_and), (12 bytes).
    Removing nrfx_atomic.o(i.nrfx_atomic_u32_cmp_exch), (4 bytes).
    Removing nrfx_atomic.o(i.nrfx_atomic_u32_fetch_add), (10 bytes).
    Removing nrfx_atomic.o(i.nrfx_atomic_u32_fetch_and), (10 bytes).
    Removing nrfx_atomic.o(i.nrfx_atomic_u32_fetch_or), (10 bytes).
    Removing nrfx_atomic.o(i.nrfx_atomic_u32_fetch_store), (10 bytes).
    Removing nrfx_atomic.o(i.nrfx_atomic_u32_fetch_sub), (10 bytes).
    Removing nrfx_atomic.o(i.nrfx_atomic_u32_fetch_sub_hs), (10 bytes).
    Removing nrfx_atomic.o(i.nrfx_atomic_u32_fetch_xor), (10 bytes).
    Removing nrfx_atomic.o(i.nrfx_atomic_u32_or), (12 bytes).
    Removing nrfx_atomic.o(i.nrfx_atomic_u32_store), (12 bytes).
    Removing nrfx_atomic.o(i.nrfx_atomic_u32_sub), (12 bytes).
    Removing nrfx_atomic.o(i.nrfx_atomic_u32_sub_hs), (12 bytes).
    Removing nrfx_atomic.o(i.nrfx_atomic_u32_xor), (12 bytes).
    Removing nrfx_clock.o(.rev16_text), (4 bytes).
    Removing nrfx_clock.o(.revsh_text), (4 bytes).
    Removing nrfx_clock.o(.rrx_text), (6 bytes).
    Removing nrfx_clock.o(i.nrfx_clock_calibration_start), (4 bytes).
    Removing nrfx_clock.o(i.nrfx_clock_calibration_timer_start), (2 bytes).
    Removing nrfx_clock.o(i.nrfx_clock_calibration_timer_stop), (2 bytes).
    Removing nrfx_clock.o(i.nrfx_clock_disable), (30 bytes).
    Removing nrfx_clock.o(i.nrfx_clock_hfclk_start), (22 bytes).
    Removing nrfx_clock.o(i.nrfx_clock_hfclk_stop), (60 bytes).
    Removing nrfx_clock.o(i.nrfx_clock_is_calibrating), (4 bytes).
    Removing nrfx_clock.o(i.nrfx_clock_lfclk_stop), (48 bytes).
    Removing nrfx_clock.o(i.nrfx_clock_uninit), (24 bytes).
    Removing nrfx_clock.o(.constdata), (16 bytes).
    Removing nrfx_clock.o(.constdata), (29 bytes).
    Removing nrfx_ppi.o(.rev16_text), (4 bytes).
    Removing nrfx_ppi.o(.revsh_text), (4 bytes).
    Removing nrfx_ppi.o(.rrx_text), (6 bytes).
    Removing nrfx_ppi.o(i.nrfx_ppi_channels_remove_from_group), (144 bytes).
    Removing nrfx_ppi.o(i.nrfx_ppi_free_all), (72 bytes).
    Removing nrfx_ppi.o(i.nrfx_ppi_group_disable), (108 bytes).
    Removing nrfx_rtc.o(.rev16_text), (4 bytes).
    Removing nrfx_rtc.o(.revsh_text), (4 bytes).
    Removing nrfx_rtc.o(.rrx_text), (6 bytes).
    Removing nrfx_rtc.o(i.nrfx_rtc_cc_disable), (56 bytes).
    Removing nrfx_rtc.o(i.nrfx_rtc_disable), (24 bytes).
    Removing nrfx_rtc.o(i.nrfx_rtc_enable), (24 bytes).
    Removing nrfx_rtc.o(i.nrfx_rtc_max_ticks_get), (32 bytes).
    Removing nrfx_rtc.o(i.nrfx_rtc_overflow_disable), (16 bytes).
    Removing nrfx_rtc.o(i.nrfx_rtc_overflow_enable), (36 bytes).
    Removing nrfx_rtc.o(i.nrfx_rtc_tick_disable), (16 bytes).
    Removing nrfx_rtc.o(i.nrfx_rtc_tick_enable), (36 bytes).
    Removing nrfx_rtc.o(i.nrfx_rtc_uninit), (80 bytes).
    Removing nrfx_rtc.o(.constdata), (14 bytes).
    Removing nrfx_rtc.o(.constdata), (20 bytes).
    Removing nrfx_rtc.o(.constdata), (16 bytes).
    Removing nrfx_timer.o(.rev16_text), (4 bytes).
    Removing nrfx_timer.o(.revsh_text), (4 bytes).
    Removing nrfx_timer.o(.rrx_text), (6 bytes).
    Removing nrfx_timer.o(i.nrfx_timer_capture), (30 bytes).
    Removing nrfx_timer.o(i.nrfx_timer_compare_int_disable), (14 bytes).
    Removing nrfx_timer.o(i.nrfx_timer_compare_int_enable), (36 bytes).
    Removing nrfx_timer.o(i.nrfx_timer_disable), (28 bytes).
    Removing nrfx_timer.o(i.nrfx_timer_extended_compare), (42 bytes).
    Removing nrfx_timer.o(i.nrfx_timer_increment), (8 bytes).
    Removing nrfx_timer.o(i.nrfx_timer_is_enabled), (32 bytes).
    Removing nrfx_timer.o(i.nrfx_timer_pause), (8 bytes).
    Removing nrfx_timer.o(i.nrfx_timer_resume), (8 bytes).
    Removing nrfx_timer.o(i.nrfx_timer_uninit), (92 bytes).
    Removing nrfx_timer.o(.constdata), (16 bytes).
    Removing app_error.o(.rev16_text), (4 bytes).
    Removing app_error.o(.revsh_text), (4 bytes).
    Removing app_error.o(.rrx_text), (6 bytes).
    Removing app_error.o(i.app_error_save_and_stop), (100 bytes).
    Removing app_error.o(.bss), (32 bytes).
    Removing app_error_handler_keil.o(.rev16_text), (4 bytes).
    Removing app_error_handler_keil.o(.revsh_text), (4 bytes).
    Removing app_error_handler_keil.o(.rrx_text), (6 bytes).
    Removing app_error_handler_keil.o(.emb_text), (26 bytes).
    Removing app_error_weak.o(.rev16_text), (4 bytes).
    Removing app_error_weak.o(.revsh_text), (4 bytes).
    Removing app_error_weak.o(.rrx_text), (6 bytes).
    Removing app_scheduler.o(.rev16_text), (4 bytes).
    Removing app_scheduler.o(.revsh_text), (4 bytes).
    Removing app_scheduler.o(.rrx_text), (6 bytes).
    Removing app_scheduler.o(i.app_sched_event_put), (156 bytes).
    Removing app_scheduler.o(i.app_sched_execute), (64 bytes).
    Removing app_scheduler.o(i.app_sched_init), (44 bytes).
    Removing app_scheduler.o(i.app_sched_queue_space_get), (36 bytes).
    Removing app_scheduler.o(.data), (16 bytes).
    Removing app_timer2.o(.rev16_text), (4 bytes).
    Removing app_timer2.o(.revsh_text), (4 bytes).
    Removing app_timer2.o(.rrx_text), (6 bytes).
    Removing app_timer2.o(i.app_timer_init), (92 bytes).
    Removing app_timer2.o(i.app_timer_pause), (12 bytes).
    Removing app_timer2.o(i.app_timer_resume), (12 bytes).
    Removing app_timer2.o(i.app_timer_stop), (58 bytes).
    Removing app_timer2.o(i.app_timer_stop_all), (20 bytes).
    Removing app_timer2.o(i.rtc_irq), (92 bytes).
    Removing app_timer2.o(i.rtc_schedule), (108 bytes).
    Removing app_timer2.o(i.rtc_update), (140 bytes).
    Removing app_timer2.o(i.sortlist_pop), (12 bytes).
    Removing app_timer2.o(i.timer_expire), (136 bytes).
    Removing app_timer2.o(i.timer_req_process), (128 bytes).
    Removing app_timer2.o(.bss), (88 bytes).
    Removing app_util_platform.o(.rev16_text), (4 bytes).
    Removing app_util_platform.o(.revsh_text), (4 bytes).
    Removing app_util_platform.o(.rrx_text), (6 bytes).
    Removing app_util_platform.o(i.current_int_priority_get), (48 bytes).
    Removing app_util_platform.o(i.privilege_level_get), (26 bytes).
    Removing drv_rtc.o(.rev16_text), (4 bytes).
    Removing drv_rtc.o(.revsh_text), (4 bytes).
    Removing drv_rtc.o(.rrx_text), (6 bytes).
    Removing drv_rtc.o(i.drv_rtc_compare_disable), (20 bytes).
    Removing drv_rtc.o(i.drv_rtc_compare_enable), (12 bytes).
    Removing drv_rtc.o(i.drv_rtc_compare_get), (14 bytes).
    Removing drv_rtc.o(i.drv_rtc_compare_pending), (14 bytes).
    Removing drv_rtc.o(i.drv_rtc_compare_set), (80 bytes).
    Removing drv_rtc.o(i.drv_rtc_init), (216 bytes).
    Removing drv_rtc.o(i.drv_rtc_overflow_disable), (16 bytes).
    Removing drv_rtc.o(i.drv_rtc_overflow_enable), (8 bytes).
    Removing drv_rtc.o(i.drv_rtc_overflow_pending), (8 bytes).
    Removing drv_rtc.o(i.drv_rtc_start), (8 bytes).
    Removing drv_rtc.o(i.drv_rtc_stop), (8 bytes).
    Removing drv_rtc.o(i.drv_rtc_tick_disable), (16 bytes).
    Removing drv_rtc.o(i.drv_rtc_tick_enable), (8 bytes).
    Removing drv_rtc.o(i.drv_rtc_tick_pending), (8 bytes).
    Removing drv_rtc.o(i.drv_rtc_uninit), (128 bytes).
    Removing drv_rtc.o(i.drv_rtc_windowed_compare_set), (222 bytes).
    Removing drv_rtc.o(i.evt_enable), (18 bytes).
    Removing drv_rtc.o(i.evt_pending), (20 bytes).
    Removing drv_rtc.o(i.nrf_rtc_event_clear), (12 bytes).
    Removing drv_rtc.o(i.nrfx_coredep_delay_us), (16 bytes).
    Removing drv_rtc.o(.constdata), (6 bytes).
    Removing nrf_assert.o(.rev16_text), (4 bytes).
    Removing nrf_assert.o(.revsh_text), (4 bytes).
    Removing nrf_assert.o(.rrx_text), (6 bytes).
    Removing nrf_assert.o(i.assert_nrf_callback), (20 bytes).
    Removing nrf_atfifo.o(.rev16_text), (4 bytes).
    Removing nrf_atfifo.o(.revsh_text), (4 bytes).
    Removing nrf_atfifo.o(.rrx_text), (6 bytes).
    Removing nrf_atfifo.o(i.nrf_atfifo_alloc_put), (46 bytes).
    Removing nrf_atfifo.o(i.nrf_atfifo_clear), (16 bytes).
    Removing nrf_atfifo.o(i.nrf_atfifo_get_free), (48 bytes).
    Removing nrf_atfifo.o(i.nrf_atfifo_init), (38 bytes).
    Removing nrf_atfifo.o(i.nrf_atfifo_item_free), (22 bytes).
    Removing nrf_atfifo.o(i.nrf_atfifo_item_get), (22 bytes).
    Removing nrf_atomic.o(.rev16_text), (4 bytes).
    Removing nrf_atomic.o(.revsh_text), (4 bytes).
    Removing nrf_atomic.o(.rrx_text), (6 bytes).
    Removing nrf_atomic.o(i.nrf_atomic_flag_clear), (6 bytes).
    Removing nrf_atomic.o(i.nrf_atomic_flag_set_fetch), (6 bytes).
    Removing nrf_atomic.o(i.nrf_atomic_u32_and), (12 bytes).
    Removing nrf_atomic.o(i.nrf_atomic_u32_cmp_exch), (4 bytes).
    Removing nrf_atomic.o(i.nrf_atomic_u32_fetch_add), (10 bytes).
    Removing nrf_atomic.o(i.nrf_atomic_u32_fetch_or), (10 bytes).
    Removing nrf_atomic.o(i.nrf_atomic_u32_fetch_sub), (10 bytes).
    Removing nrf_atomic.o(i.nrf_atomic_u32_fetch_sub_hs), (10 bytes).
    Removing nrf_atomic.o(i.nrf_atomic_u32_fetch_xor), (10 bytes).
    Removing nrf_atomic.o(i.nrf_atomic_u32_store), (12 bytes).
    Removing nrf_atomic.o(i.nrf_atomic_u32_sub_hs), (12 bytes).
    Removing nrf_atomic.o(i.nrf_atomic_u32_xor), (12 bytes).
    Removing nrf_balloc.o(.rev16_text), (4 bytes).
    Removing nrf_balloc.o(.revsh_text), (4 bytes).
    Removing nrf_balloc.o(.rrx_text), (6 bytes).
    Removing nrf_fprintf.o(.rev16_text), (4 bytes).
    Removing nrf_fprintf.o(.revsh_text), (4 bytes).
    Removing nrf_fprintf.o(.rrx_text), (6 bytes).
    Removing nrf_fprintf_format.o(.rev16_text), (4 bytes).
    Removing nrf_fprintf_format.o(.revsh_text), (4 bytes).
    Removing nrf_fprintf_format.o(.rrx_text), (6 bytes).
    Removing nrf_libuarte_async.o(.rev16_text), (4 bytes).
    Removing nrf_libuarte_async.o(.revsh_text), (4 bytes).
    Removing nrf_libuarte_async.o(.rrx_text), (6 bytes).
    Removing nrf_libuarte_async.o(i.nrf_libuarte_async_rts_clear), (6 bytes).
    Removing nrf_libuarte_async.o(i.nrf_libuarte_async_rts_set), (6 bytes).
    Removing nrf_libuarte_async.o(i.nrf_libuarte_async_uninit), (108 bytes).
    Removing nrf_libuarte_drv.o(.rev16_text), (4 bytes).
    Removing nrf_libuarte_drv.o(.revsh_text), (4 bytes).
    Removing nrf_libuarte_drv.o(.rrx_text), (6 bytes).
    Removing nrf_libuarte_drv.o(i.nrf_libuarte_drv_rts_clear), (2 bytes).
    Removing nrf_libuarte_drv.o(i.nrf_libuarte_drv_rts_set), (2 bytes).
    Removing nrf_libuarte_drv.o(i.nrf_libuarte_drv_rx_stop), (22 bytes).
    Removing nrf_libuarte_drv.o(i.nrf_libuarte_drv_uninit), (250 bytes).
    Removing nrf_libuarte_drv.o(i.rx_ppi_disable), (28 bytes).
    Removing nrf_memobj.o(.rev16_text), (4 bytes).
    Removing nrf_memobj.o(.revsh_text), (4 bytes).
    Removing nrf_memobj.o(.rrx_text), (6 bytes).
    Removing nrf_queue.o(.rev16_text), (4 bytes).
    Removing nrf_queue.o(.revsh_text), (4 bytes).
    Removing nrf_queue.o(.rrx_text), (6 bytes).
    Removing nrf_queue.o(i.continous_items_get), (38 bytes).
    Removing nrf_queue.o(i.nrf_queue_available_get), (14 bytes).
    Removing nrf_queue.o(i.nrf_queue_in), (62 bytes).
    Removing nrf_queue.o(i.nrf_queue_max_utilization_get), (6 bytes).
    Removing nrf_queue.o(i.nrf_queue_max_utilization_reset), (8 bytes).
    Removing nrf_queue.o(i.nrf_queue_out), (50 bytes).
    Removing nrf_queue.o(i.nrf_queue_read), (58 bytes).
    Removing nrf_queue.o(i.nrf_queue_utilization_get), (28 bytes).
    Removing nrf_queue.o(i.nrf_queue_write), (62 bytes).
    Removing nrf_queue.o(i.queue_read), (100 bytes).
    Removing nrf_queue.o(i.queue_write), (144 bytes).
    Removing nrf_ringbuf.o(.rev16_text), (4 bytes).
    Removing nrf_ringbuf.o(.revsh_text), (4 bytes).
    Removing nrf_ringbuf.o(.rrx_text), (6 bytes).
    Removing nrf_ringbuf.o(i.nrf_ringbuf_alloc), (112 bytes).
    Removing nrf_ringbuf.o(i.nrf_ringbuf_cpy_get), (128 bytes).
    Removing nrf_ringbuf.o(i.nrf_ringbuf_cpy_put), (118 bytes).
    Removing nrf_ringbuf.o(i.nrf_ringbuf_free), (38 bytes).
    Removing nrf_ringbuf.o(i.nrf_ringbuf_get), (112 bytes).
    Removing nrf_ringbuf.o(i.nrf_ringbuf_put), (48 bytes).
    Removing nrf_sortlist.o(.rev16_text), (4 bytes).
    Removing nrf_sortlist.o(.revsh_text), (4 bytes).
    Removing nrf_sortlist.o(.rrx_text), (6 bytes).
    Removing nrf_sortlist.o(i.nrf_sortlist_add), (34 bytes).
    Removing nrf_sortlist.o(i.nrf_sortlist_next), (4 bytes).
    Removing nrf_sortlist.o(i.nrf_sortlist_peek), (6 bytes).
    Removing nrf_sortlist.o(i.nrf_sortlist_pop), (14 bytes).
    Removing nrf_sortlist.o(i.nrf_sortlist_remove), (30 bytes).
    Removing nrf_strerror.o(.rev16_text), (4 bytes).
    Removing nrf_strerror.o(.revsh_text), (4 bytes).
    Removing nrf_strerror.o(.rrx_text), (6 bytes).
    Removing nrf_log_backend_rtt.o(.rev16_text), (4 bytes).
    Removing nrf_log_backend_rtt.o(.revsh_text), (4 bytes).
    Removing nrf_log_backend_rtt.o(.rrx_text), (6 bytes).
    Removing nrf_log_backend_serial.o(.rev16_text), (4 bytes).
    Removing nrf_log_backend_serial.o(.revsh_text), (4 bytes).
    Removing nrf_log_backend_serial.o(.rrx_text), (6 bytes).
    Removing nrf_log_default_backends.o(.rev16_text), (4 bytes).
    Removing nrf_log_default_backends.o(.revsh_text), (4 bytes).
    Removing nrf_log_default_backends.o(.rrx_text), (6 bytes).
    Removing nrf_log_frontend.o(.rev16_text), (4 bytes).
    Removing nrf_log_frontend.o(.revsh_text), (4 bytes).
    Removing nrf_log_frontend.o(.rrx_text), (6 bytes).
    Removing nrf_log_frontend.o(i.nrf_log_backend_remove), (52 bytes).
    Removing nrf_log_frontend.o(i.nrf_log_frontend_hexdump), (172 bytes).
    Removing nrf_log_frontend.o(i.nrf_log_frontend_std_4), (20 bytes).
    Removing nrf_log_frontend.o(i.nrf_log_frontend_std_5), (28 bytes).
    Removing nrf_log_frontend.o(i.nrf_log_frontend_std_6), (28 bytes).
    Removing nrf_log_frontend.o(i.nrf_log_module_filter_get), (36 bytes).
    Removing nrf_log_frontend.o(i.nrf_log_module_filter_set), (2 bytes).
    Removing nrf_log_frontend.o(i.nrf_log_push), (96 bytes).
    Removing nrf_log_str_formatter.o(.rev16_text), (4 bytes).
    Removing nrf_log_str_formatter.o(.revsh_text), (4 bytes).
    Removing nrf_log_str_formatter.o(.rrx_text), (6 bytes).
    Removing nrf_log_str_formatter.o(i.nrf_log_str_formatter_timestamp_freq_set), (32 bytes).
    Removing segger_rtt.o(.rev16_text), (4 bytes).
    Removing segger_rtt.o(.revsh_text), (4 bytes).
    Removing segger_rtt.o(.rrx_text), (6 bytes).
    Removing segger_rtt.o(i.SEGGER_RTT_AllocDownBuffer), (104 bytes).
    Removing segger_rtt.o(i.SEGGER_RTT_AllocUpBuffer), (104 bytes).
    Removing segger_rtt.o(i.SEGGER_RTT_ConfigDownBuffer), (92 bytes).
    Removing segger_rtt.o(i.SEGGER_RTT_ConfigUpBuffer), (92 bytes).
    Removing segger_rtt.o(i.SEGGER_RTT_GetKey), (28 bytes).
    Removing segger_rtt.o(i.SEGGER_RTT_HasData), (24 bytes).
    Removing segger_rtt.o(i.SEGGER_RTT_HasKey), (32 bytes).
    Removing segger_rtt.o(i.SEGGER_RTT_PutChar), (88 bytes).
    Removing segger_rtt.o(i.SEGGER_RTT_PutCharSkip), (76 bytes).
    Removing segger_rtt.o(i.SEGGER_RTT_PutCharSkipNoLock), (52 bytes).
    Removing segger_rtt.o(i.SEGGER_RTT_Read), (36 bytes).
    Removing segger_rtt.o(i.SEGGER_RTT_ReadNoLock), (120 bytes).
    Removing segger_rtt.o(i.SEGGER_RTT_SetFlagsDownBuffer), (60 bytes).
    Removing segger_rtt.o(i.SEGGER_RTT_SetFlagsUpBuffer), (60 bytes).
    Removing segger_rtt.o(i.SEGGER_RTT_SetNameDownBuffer), (60 bytes).
    Removing segger_rtt.o(i.SEGGER_RTT_SetNameUpBuffer), (60 bytes).
    Removing segger_rtt.o(i.SEGGER_RTT_SetTerminal), (128 bytes).
    Removing segger_rtt.o(i.SEGGER_RTT_TerminalOut), (168 bytes).
    Removing segger_rtt.o(i.SEGGER_RTT_WaitKey), (14 bytes).
    Removing segger_rtt.o(i.SEGGER_RTT_Write), (52 bytes).
    Removing segger_rtt.o(i.SEGGER_RTT_WriteSkipNoLock), (116 bytes).
    Removing segger_rtt.o(i.SEGGER_RTT_WriteString), (26 bytes).
    Removing segger_rtt.o(i.SEGGER_RTT_WriteWithOverwriteNoLock), (148 bytes).
    Removing segger_rtt.o(i._PostTerminalSwitch), (32 bytes).
    Removing segger_rtt.o(.data), (17 bytes).
    Removing segger_rtt_syscalls_keil.o(.rev16_text), (4 bytes).
    Removing segger_rtt_syscalls_keil.o(.revsh_text), (4 bytes).
    Removing segger_rtt_syscalls_keil.o(.rrx_text), (6 bytes).
    Removing segger_rtt_syscalls_keil.o(i._sys_close), (4 bytes).
    Removing segger_rtt_syscalls_keil.o(i._sys_command_string), (2 bytes).
    Removing segger_rtt_syscalls_keil.o(i._sys_ensure), (6 bytes).
    Removing segger_rtt_syscalls_keil.o(i._sys_exit), (2 bytes).
    Removing segger_rtt_syscalls_keil.o(i._sys_flen), (4 bytes).
    Removing segger_rtt_syscalls_keil.o(i._sys_istty), (14 bytes).
    Removing segger_rtt_syscalls_keil.o(i._sys_open), (44 bytes).
    Removing segger_rtt_syscalls_keil.o(i._sys_read), (4 bytes).
    Removing segger_rtt_syscalls_keil.o(i._sys_seek), (4 bytes).
    Removing segger_rtt_syscalls_keil.o(i._sys_tmpnam), (4 bytes).
    Removing segger_rtt_syscalls_keil.o(i._sys_write), (26 bytes).
    Removing segger_rtt_syscalls_keil.o(i._ttywrch), (24 bytes).
    Removing segger_rtt_syscalls_keil.o(.constdata), (14 bytes).
    Removing segger_rtt_printf.o(.rev16_text), (4 bytes).
    Removing segger_rtt_printf.o(.revsh_text), (4 bytes).
    Removing segger_rtt_printf.o(.rrx_text), (6 bytes).
    Removing segger_rtt_printf.o(i.SEGGER_RTT_printf), (22 bytes).
    Removing segger_rtt_printf.o(i.SEGGER_RTT_vprintf), (406 bytes).
    Removing segger_rtt_printf.o(i._PrintInt), (198 bytes).
    Removing segger_rtt_printf.o(i._PrintUnsigned), (212 bytes).
    Removing segger_rtt_printf.o(i._StoreChar), (62 bytes).
    Removing segger_rtt_printf.o(.constdata), (16 bytes).
    Removing arm_startup_nrf52840.o(HEAP), (8192 bytes).
    Removing system_nrf52.o(.rev16_text), (4 bytes).
    Removing system_nrf52.o(.revsh_text), (4 bytes).
    Removing system_nrf52.o(.rrx_text), (6 bytes).
    Removing system_nrf52.o(i.SystemCoreClockUpdate), (16 bytes).
    Removing system_nrf52.o(i.nvmc_wait), (16 bytes).

358 unused section(s) (total 19107 bytes) removed from the image.

==============================================================================

Image Symbol Table

    Local Symbols

    Symbol Name                              Value     Ov Type        Size  Object(Section)

    RESET                                    0x00000000   Section      512  arm_startup_nrf52840.o(RESET)
    ../clib/microlib/ctype/ctype.c           0x00000000   Number         0  isalnum_o.o ABSOLUTE
    ../clib/microlib/ctype/ctype.c           0x00000000   Number         0  isprint_o.o ABSOLUTE
    ../clib/microlib/ctype/ctype.c           0x00000000   Number         0  islower_o.o ABSOLUTE
    ../clib/microlib/ctype/ctype.c           0x00000000   Number         0  isgraph_o.o ABSOLUTE
    ../clib/microlib/ctype/ctype.c           0x00000000   Number         0  isdigit_o.o ABSOLUTE
    ../clib/microlib/ctype/ctype.c           0x00000000   Number         0  isupper_o.o ABSOLUTE
    ../clib/microlib/ctype/ctype.c           0x00000000   Number         0  isxdigit_o.o ABSOLUTE
    ../clib/microlib/ctype/ctype.c           0x00000000   Number         0  isalpha_o.o ABSOLUTE
    ../clib/microlib/ctype/ctype.c           0x00000000   Number         0  iscntrl_o.o ABSOLUTE
    ../clib/microlib/ctype/ctype.c           0x00000000   Number         0  ispunct_o.o ABSOLUTE
    ../clib/microlib/ctype/ctype.c           0x00000000   Number         0  isblank_o.o ABSOLUTE
    ../clib/microlib/ctype/ctype.c           0x00000000   Number         0  ctype_o.o ABSOLUTE
    ../clib/microlib/ctype/ctype.c           0x00000000   Number         0  isspace_o.o ABSOLUTE
    ../clib/microlib/division.c              0x00000000   Number         0  uldiv.o ABSOLUTE
    ../clib/microlib/init/entry.s            0x00000000   Number         0  entry11b.o ABSOLUTE
    ../clib/microlib/init/entry.s            0x00000000   Number         0  entry10b.o ABSOLUTE
    ../clib/microlib/init/entry.s            0x00000000   Number         0  entry9b.o ABSOLUTE
    ../clib/microlib/init/entry.s            0x00000000   Number         0  entry9a.o ABSOLUTE
    ../clib/microlib/init/entry.s            0x00000000   Number         0  entry8b.o ABSOLUTE
    ../clib/microlib/init/entry.s            0x00000000   Number         0  entry8a.o ABSOLUTE
    ../clib/microlib/init/entry.s            0x00000000   Number         0  entry7b.o ABSOLUTE
    ../clib/microlib/init/entry.s            0x00000000   Number         0  entry11a.o ABSOLUTE
    ../clib/microlib/init/entry.s            0x00000000   Number         0  entry.o ABSOLUTE
    ../clib/microlib/init/entry.s            0x00000000   Number         0  entry5.o ABSOLUTE
    ../clib/microlib/init/entry.s            0x00000000   Number         0  entry2.o ABSOLUTE
    ../clib/microlib/init/entry.s            0x00000000   Number         0  entry7a.o ABSOLUTE
    ../clib/microlib/init/entry.s            0x00000000   Number         0  entry10a.o ABSOLUTE
    ../clib/microlib/longlong.c              0x00000000   Number         0  llshl.o ABSOLUTE
    ../clib/microlib/longlong.c              0x00000000   Number         0  llushr.o ABSOLUTE
    ../clib/microlib/stdio/fflush.c          0x00000000   Number         0  fflush.o ABSOLUTE
    ../clib/microlib/stdio/fputc.c           0x00000000   Number         0  fputc.o ABSOLUTE
    ../clib/microlib/stdio/semi.s            0x00000000   Number         0  semi.o ABSOLUTE
    ../clib/microlib/stdio/streams.c         0x00000000   Number         0  stdout.o ABSOLUTE
    ../clib/microlib/string/memcpy.c         0x00000000   Number         0  memcpyb.o ABSOLUTE
    ../clib/microlib/string/memcpy.c         0x00000000   Number         0  memcpya.o ABSOLUTE
    ../clib/microlib/string/memset.c         0x00000000   Number         0  memseta.o ABSOLUTE
    ../clib/microlib/string/strcmp.c         0x00000000   Number         0  strcmp.o ABSOLUTE
    ../clib/microlib/string/strcpy.c         0x00000000   Number         0  strcpy.o ABSOLUTE
    ../clib/microlib/string/strlen.c         0x00000000   Number         0  strlen.o ABSOLUTE
    ../clib/microlib/stubs.s                 0x00000000   Number         0  useno.o ABSOLUTE
    ../clib/microlib/stubs.s                 0x00000000   Number         0  iusesemip.o ABSOLUTE
    ..\..\..\..\..\..\components\boards\boards.c 0x00000000   Number         0  boards.o ABSOLUTE
    ..\..\..\..\..\..\components\drivers_nrf\nrf_soc_nosd\nrf_nvic.c 0x00000000   Number         0  nrf_nvic.o ABSOLUTE
    ..\..\..\..\..\..\components\drivers_nrf\nrf_soc_nosd\nrf_soc.c 0x00000000   Number         0  nrf_soc.o ABSOLUTE
    ..\..\..\..\..\..\components\libraries\atomic\nrf_atomic.c 0x00000000   Number         0  nrf_atomic.o ABSOLUTE
    ..\..\..\..\..\..\components\libraries\atomic_fifo\nrf_atfifo.c 0x00000000   Number         0  nrf_atfifo.o ABSOLUTE
    ..\..\..\..\..\..\components\libraries\balloc\nrf_balloc.c 0x00000000   Number         0  nrf_balloc.o ABSOLUTE
    ..\..\..\..\..\..\components\libraries\libuarte\nrf_libuarte_async.c 0x00000000   Number         0  nrf_libuarte_async.o ABSOLUTE
    ..\..\..\..\..\..\components\libraries\libuarte\nrf_libuarte_drv.c 0x00000000   Number         0  nrf_libuarte_drv.o ABSOLUTE
    ..\..\..\..\..\..\components\libraries\log\src\nrf_log_backend_rtt.c 0x00000000   Number         0  nrf_log_backend_rtt.o ABSOLUTE
    ..\..\..\..\..\..\components\libraries\log\src\nrf_log_backend_serial.c 0x00000000   Number         0  nrf_log_backend_serial.o ABSOLUTE
    ..\..\..\..\..\..\components\libraries\log\src\nrf_log_default_backends.c 0x00000000   Number         0  nrf_log_default_backends.o ABSOLUTE
    ..\..\..\..\..\..\components\libraries\log\src\nrf_log_frontend.c 0x00000000   Number         0  nrf_log_frontend.o ABSOLUTE
    ..\..\..\..\..\..\components\libraries\log\src\nrf_log_str_formatter.c 0x00000000   Number         0  nrf_log_str_formatter.o ABSOLUTE
    ..\..\..\..\..\..\components\libraries\memobj\nrf_memobj.c 0x00000000   Number         0  nrf_memobj.o ABSOLUTE
    ..\..\..\..\..\..\components\libraries\queue\nrf_queue.c 0x00000000   Number         0  nrf_queue.o ABSOLUTE
    ..\..\..\..\..\..\components\libraries\ringbuf\nrf_ringbuf.c 0x00000000   Number         0  nrf_ringbuf.o ABSOLUTE
    ..\..\..\..\..\..\components\libraries\scheduler\app_scheduler.c 0x00000000   Number         0  app_scheduler.o ABSOLUTE
    ..\..\..\..\..\..\components\libraries\sortlist\nrf_sortlist.c 0x00000000   Number         0  nrf_sortlist.o ABSOLUTE
    ..\..\..\..\..\..\components\libraries\strerror\nrf_strerror.c 0x00000000   Number         0  nrf_strerror.o ABSOLUTE
    ..\..\..\..\..\..\components\libraries\timer\app_timer2.c 0x00000000   Number         0  app_timer2.o ABSOLUTE
    ..\..\..\..\..\..\components\libraries\timer\drv_rtc.c 0x00000000   Number         0  drv_rtc.o ABSOLUTE
    ..\..\..\..\..\..\components\libraries\util\app_error.c 0x00000000   Number         0  app_error.o ABSOLUTE
    ..\..\..\..\..\..\components\libraries\util\app_error_handler_keil.c 0x00000000   Number         0  app_error_handler_keil.o ABSOLUTE
    ..\..\..\..\..\..\components\libraries\util\app_error_weak.c 0x00000000   Number         0  app_error_weak.o ABSOLUTE
    ..\..\..\..\..\..\components\libraries\util\app_util_platform.c 0x00000000   Number         0  app_util_platform.o ABSOLUTE
    ..\..\..\..\..\..\components\libraries\util\nrf_assert.c 0x00000000   Number         0  nrf_assert.o ABSOLUTE
    ..\..\..\..\..\..\external\fprintf\nrf_fprintf.c 0x00000000   Number         0  nrf_fprintf.o ABSOLUTE
    ..\..\..\..\..\..\external\fprintf\nrf_fprintf_format.c 0x00000000   Number         0  nrf_fprintf_format.o ABSOLUTE
    ..\..\..\..\..\..\external\segger_rtt\SEGGER_RTT.c 0x00000000   Number         0  segger_rtt.o ABSOLUTE
    ..\..\..\..\..\..\external\segger_rtt\SEGGER_RTT_Syscalls_KEIL.c 0x00000000   Number         0  segger_rtt_syscalls_keil.o ABSOLUTE
    ..\..\..\..\..\..\external\segger_rtt\SEGGER_RTT_printf.c 0x00000000   Number         0  segger_rtt_printf.o ABSOLUTE
    ..\..\..\..\..\..\integration\nrfx\legacy\nrf_drv_clock.c 0x00000000   Number         0  nrf_drv_clock.o ABSOLUTE
    ..\..\..\..\..\..\modules\nrfx\drivers\src\nrfx_clock.c 0x00000000   Number         0  nrfx_clock.o ABSOLUTE
    ..\..\..\..\..\..\modules\nrfx\drivers\src\nrfx_ppi.c 0x00000000   Number         0  nrfx_ppi.o ABSOLUTE
    ..\..\..\..\..\..\modules\nrfx\drivers\src\nrfx_rtc.c 0x00000000   Number         0  nrfx_rtc.o ABSOLUTE
    ..\..\..\..\..\..\modules\nrfx\drivers\src\nrfx_timer.c 0x00000000   Number         0  nrfx_timer.o ABSOLUTE
    ..\..\..\..\..\..\modules\nrfx\soc\nrfx_atomic.c 0x00000000   Number         0  nrfx_atomic.o ABSOLUTE
    ..\..\..\main.c                          0x00000000   Number         0  main.o ABSOLUTE
    ..\\..\\..\\..\\..\\..\\components\\boards\\boards.c 0x00000000   Number         0  boards.o ABSOLUTE
    ..\\..\\..\\..\\..\\..\\components\\drivers_nrf\\nrf_soc_nosd\\nrf_nvic.c 0x00000000   Number         0  nrf_nvic.o ABSOLUTE
    ..\\..\\..\\..\\..\\..\\components\\drivers_nrf\\nrf_soc_nosd\\nrf_soc.c 0x00000000   Number         0  nrf_soc.o ABSOLUTE
    ..\\..\\..\\..\\..\\..\\components\\libraries\\atomic\\nrf_atomic.c 0x00000000   Number         0  nrf_atomic.o ABSOLUTE
    ..\\..\\..\\..\\..\\..\\components\\libraries\\atomic_fifo\\nrf_atfifo.c 0x00000000   Number         0  nrf_atfifo.o ABSOLUTE
    ..\\..\\..\\..\\..\\..\\components\\libraries\\balloc\\nrf_balloc.c 0x00000000   Number         0  nrf_balloc.o ABSOLUTE
    ..\\..\\..\\..\\..\\..\\components\\libraries\\libuarte\\nrf_libuarte_async.c 0x00000000   Number         0  nrf_libuarte_async.o ABSOLUTE
    ..\\..\\..\\..\\..\\..\\components\\libraries\\libuarte\\nrf_libuarte_drv.c 0x00000000   Number         0  nrf_libuarte_drv.o ABSOLUTE
    ..\\..\\..\\..\\..\\..\\components\\libraries\\log\\src\\nrf_log_backend_rtt.c 0x00000000   Number         0  nrf_log_backend_rtt.o ABSOLUTE
    ..\\..\\..\\..\\..\\..\\components\\libraries\\log\\src\\nrf_log_backend_serial.c 0x00000000   Number         0  nrf_log_backend_serial.o ABSOLUTE
    ..\\..\\..\\..\\..\\..\\components\\libraries\\log\\src\\nrf_log_default_backends.c 0x00000000   Number         0  nrf_log_default_backends.o ABSOLUTE
    ..\\..\\..\\..\\..\\..\\components\\libraries\\log\\src\\nrf_log_frontend.c 0x00000000   Number         0  nrf_log_frontend.o ABSOLUTE
    ..\\..\\..\\..\\..\\..\\components\\libraries\\log\\src\\nrf_log_str_formatter.c 0x00000000   Number         0  nrf_log_str_formatter.o ABSOLUTE
    ..\\..\\..\\..\\..\\..\\components\\libraries\\memobj\\nrf_memobj.c 0x00000000   Number         0  nrf_memobj.o ABSOLUTE
    ..\\..\\..\\..\\..\\..\\components\\libraries\\queue\\nrf_queue.c 0x00000000   Number         0  nrf_queue.o ABSOLUTE
    ..\\..\\..\\..\\..\\..\\components\\libraries\\ringbuf\\nrf_ringbuf.c 0x00000000   Number         0  nrf_ringbuf.o ABSOLUTE
    ..\\..\\..\\..\\..\\..\\components\\libraries\\scheduler\\app_scheduler.c 0x00000000   Number         0  app_scheduler.o ABSOLUTE
    ..\\..\\..\\..\\..\\..\\components\\libraries\\sortlist\\nrf_sortlist.c 0x00000000   Number         0  nrf_sortlist.o ABSOLUTE
    ..\\..\\..\\..\\..\\..\\components\\libraries\\strerror\\nrf_strerror.c 0x00000000   Number         0  nrf_strerror.o ABSOLUTE
    ..\\..\\..\\..\\..\\..\\components\\libraries\\timer\\app_timer2.c 0x00000000   Number         0  app_timer2.o ABSOLUTE
    ..\\..\\..\\..\\..\\..\\components\\libraries\\timer\\drv_rtc.c 0x00000000   Number         0  drv_rtc.o ABSOLUTE
    ..\\..\\..\\..\\..\\..\\components\\libraries\\util\\app_error.c 0x00000000   Number         0  app_error.o ABSOLUTE
    ..\\..\\..\\..\\..\\..\\components\\libraries\\util\\app_error_handler_keil.c 0x00000000   Number         0  app_error_handler_keil.o ABSOLUTE
    ..\\..\\..\\..\\..\\..\\components\\libraries\\util\\app_error_weak.c 0x00000000   Number         0  app_error_weak.o ABSOLUTE
    ..\\..\\..\\..\\..\\..\\components\\libraries\\util\\app_util_platform.c 0x00000000   Number         0  app_util_platform.o ABSOLUTE
    ..\\..\\..\\..\\..\\..\\components\\libraries\\util\\nrf_assert.c 0x00000000   Number         0  nrf_assert.o ABSOLUTE
    ..\\..\\..\\..\\..\\..\\external\\fprintf\\nrf_fprintf.c 0x00000000   Number         0  nrf_fprintf.o ABSOLUTE
    ..\\..\\..\\..\\..\\..\\external\\fprintf\\nrf_fprintf_format.c 0x00000000   Number         0  nrf_fprintf_format.o ABSOLUTE
    ..\\..\\..\\..\\..\\..\\external\\segger_rtt\\SEGGER_RTT.c 0x00000000   Number         0  segger_rtt.o ABSOLUTE
    ..\\..\\..\\..\\..\\..\\external\\segger_rtt\\SEGGER_RTT_Syscalls_KEIL.c 0x00000000   Number         0  segger_rtt_syscalls_keil.o ABSOLUTE
    ..\\..\\..\\..\\..\\..\\external\\segger_rtt\\SEGGER_RTT_printf.c 0x00000000   Number         0  segger_rtt_printf.o ABSOLUTE
    ..\\..\\..\\..\\..\\..\\integration\\nrfx\\legacy\\nrf_drv_clock.c 0x00000000   Number         0  nrf_drv_clock.o ABSOLUTE
    ..\\..\\..\\..\\..\\..\\modules\\nrfx\\drivers\\src\\nrfx_clock.c 0x00000000   Number         0  nrfx_clock.o ABSOLUTE
    ..\\..\\..\\..\\..\\..\\modules\\nrfx\\drivers\\src\\nrfx_ppi.c 0x00000000   Number         0  nrfx_ppi.o ABSOLUTE
    ..\\..\\..\\..\\..\\..\\modules\\nrfx\\drivers\\src\\nrfx_rtc.c 0x00000000   Number         0  nrfx_rtc.o ABSOLUTE
    ..\\..\\..\\..\\..\\..\\modules\\nrfx\\drivers\\src\\nrfx_timer.c 0x00000000   Number         0  nrfx_timer.o ABSOLUTE
    ..\\..\\..\\..\\..\\..\\modules\\nrfx\\soc\\nrfx_atomic.c 0x00000000   Number         0  nrfx_atomic.o ABSOLUTE
    ..\\..\\..\\main.c                       0x00000000   Number         0  main.o ABSOLUTE
    RTE\Device\nRF52840_xxAA\arm_startup_nrf52840.s 0x00000000   Number         0  arm_startup_nrf52840.o ABSOLUTE
    RTE\Device\nRF52840_xxAA\system_nrf52.c  0x00000000   Number         0  system_nrf52.o ABSOLUTE
    RTE\\Device\\nRF52840_xxAA\\system_nrf52.c 0x00000000   Number         0  system_nrf52.o ABSOLUTE
    dc.s                                     0x00000000   Number         0  dc.o ABSOLUTE
    handlers.s                               0x00000000   Number         0  handlers.o ABSOLUTE
    init.s                                   0x00000000   Number         0  init.o ABSOLUTE
    .ARM.Collect$$$$00000000                 0x00000200   Section        0  entry.o(.ARM.Collect$$$$00000000)
    .ARM.Collect$$$$00000001                 0x00000200   Section        4  entry2.o(.ARM.Collect$$$$00000001)
    .ARM.Collect$$$$00000004                 0x00000204   Section        4  entry5.o(.ARM.Collect$$$$00000004)
    .ARM.Collect$$$$00000008                 0x00000208   Section        0  entry7b.o(.ARM.Collect$$$$00000008)
    .ARM.Collect$$$$0000000A                 0x00000208   Section        0  entry8b.o(.ARM.Collect$$$$0000000A)
    .ARM.Collect$$$$0000000B                 0x00000208   Section        8  entry9a.o(.ARM.Collect$$$$0000000B)
    .ARM.Collect$$$$0000000D                 0x00000210   Section        0  entry10a.o(.ARM.Collect$$$$0000000D)
    .ARM.Collect$$$$0000000F                 0x00000210   Section        0  entry11a.o(.ARM.Collect$$$$0000000F)
    .ARM.Collect$$$$00002712                 0x00000210   Section        4  entry2.o(.ARM.Collect$$$$00002712)
    __lit__00000000                          0x00000210   Data           4  entry2.o(.ARM.Collect$$$$00002712)
    .emb_text                                0x00000214   Section      200  nrf_atfifo.o(.emb_text)
    $v0                                      0x00000214   Number         0  nrf_atfifo.o(.emb_text)
    .emb_text                                0x000002dc   Section      226  nrf_atomic.o(.emb_text)
    $v0                                      0x000002dc   Number         0  nrf_atomic.o(.emb_text)
    .text                                    0x000003c0   Section       36  arm_startup_nrf52840.o(.text)
    $v0                                      0x000003c0   Number         0  arm_startup_nrf52840.o(.text)
    .text                                    0x000003e4   Section        0  uldiv.o(.text)
    .text                                    0x00000448   Section        0  ctype_o.o(.text)
    .text                                    0x00000450   Section        0  memcpya.o(.text)
    .text                                    0x00000474   Section        0  memseta.o(.text)
    .text                                    0x00000498   Section        0  strlen.o(.text)
    .text                                    0x000004a6   Section        0  strcpy.o(.text)
    .text                                    0x000004b8   Section        0  llshl.o(.text)
    .text                                    0x000004d6   Section        0  llushr.o(.text)
    .text                                    0x000004f8   Section       36  init.o(.text)
    i.POWER_CLOCK_IRQHandler                 0x0000051c   Section        0  nrfx_clock.o(i.POWER_CLOCK_IRQHandler)
    i.RTC0_IRQHandler                        0x00000574   Section        0  nrfx_rtc.o(i.RTC0_IRQHandler)
    i.RTC1_IRQHandler                        0x00000584   Section        0  drv_rtc.o(i.RTC1_IRQHandler)
    i.RTC2_IRQHandler                        0x00000594   Section        0  nrfx_rtc.o(i.RTC2_IRQHandler)
    i.SEGGER_RTT_Init                        0x000005a4   Section        0  segger_rtt.o(i.SEGGER_RTT_Init)
    i.SEGGER_RTT_WriteNoLock                 0x000005a8   Section        0  segger_rtt.o(i.SEGGER_RTT_WriteNoLock)
    i.SystemInit                             0x00000604   Section        0  system_nrf52.o(i.SystemInit)
    i.TIMER0_IRQHandler                      0x000007e0   Section        0  nrfx_timer.o(i.TIMER0_IRQHandler)
    i.TIMER1_IRQHandler                      0x000007f4   Section        0  nrfx_timer.o(i.TIMER1_IRQHandler)
    i.UARTE0_UART0_IRQHandler                0x00000808   Section        0  nrf_libuarte_drv.o(i.UARTE0_UART0_IRQHandler)
    i.UARTE1_IRQHandler                      0x00000814   Section        0  nrf_libuarte_drv.o(i.UARTE1_IRQHandler)
    i._DoInit                                0x00000820   Section        0  segger_rtt.o(i._DoInit)
    _DoInit                                  0x00000821   Thumb Code    76  segger_rtt.o(i._DoInit)
    i._GetAvailWriteSpace                    0x00000888   Section        0  segger_rtt.o(i._GetAvailWriteSpace)
    _GetAvailWriteSpace                      0x00000889   Thumb Code    22  segger_rtt.o(i._GetAvailWriteSpace)
    i._WriteBlocking                         0x0000089e   Section        0  segger_rtt.o(i._WriteBlocking)
    _WriteBlocking                           0x0000089f   Thumb Code    90  segger_rtt.o(i._WriteBlocking)
    i._WriteNoCheck                          0x000008f8   Section        0  segger_rtt.o(i._WriteNoCheck)
    _WriteNoCheck                            0x000008f9   Thumb Code    66  segger_rtt.o(i._WriteNoCheck)
    i.__scatterload_copy                     0x0000093a   Section       14  handlers.o(i.__scatterload_copy)
    i.__scatterload_null                     0x00000948   Section        2  handlers.o(i.__scatterload_null)
    i.__scatterload_zeroinit                 0x0000094a   Section       14  handlers.o(i.__scatterload_zeroinit)
    i.app_error_fault_handler                0x00000958   Section        0  app_error_weak.o(i.app_error_fault_handler)
    i.app_error_handler_bare                 0x000009dc   Section        0  app_error.o(i.app_error_handler_bare)
    i.app_timer_cnt_diff_compute             0x000009f2   Section        0  app_timer2.o(i.app_timer_cnt_diff_compute)
    i.app_timer_cnt_get                      0x000009fc   Section        0  app_timer2.o(i.app_timer_cnt_get)
    i.app_timer_create                       0x00000a08   Section        0  app_timer2.o(i.app_timer_create)
    i.app_timer_handler                      0x00000a28   Section        0  nrf_libuarte_async.o(i.app_timer_handler)
    app_timer_handler                        0x00000a29   Thumb Code   144  nrf_libuarte_async.o(i.app_timer_handler)
    i.app_timer_start                        0x00000ac0   Section        0  app_timer2.o(i.app_timer_start)
    i.app_util_critical_region_enter         0x00000b0c   Section        0  app_util_platform.o(i.app_util_critical_region_enter)
    i.app_util_critical_region_exit          0x00000b10   Section        0  app_util_platform.o(i.app_util_critical_region_exit)
    i.app_util_disable_irq                   0x00000b14   Section        0  app_util_platform.o(i.app_util_disable_irq)
    i.app_util_enable_irq                    0x00000b24   Section        0  app_util_platform.o(i.app_util_enable_irq)
    i.bsp_board_led_invert                   0x00000b38   Section        0  boards.o(i.bsp_board_led_invert)
    i.buf_prealloc                           0x00000b64   Section        0  nrf_log_frontend.o(i.buf_prealloc)
    buf_prealloc                             0x00000b65   Thumb Code   132  nrf_log_frontend.o(i.buf_prealloc)
    i.buffer_add                             0x00000bf0   Section        0  nrf_fprintf_format.o(i.buffer_add)
    buffer_add                               0x00000bf1   Thumb Code    46  nrf_fprintf_format.o(i.buffer_add)
    i.buffer_is_empty                        0x00000c20   Section        0  nrf_log_frontend.o(i.buffer_is_empty)
    i.clock_clk_started_notify               0x00000c38   Section        0  nrf_drv_clock.o(i.clock_clk_started_notify)
    clock_clk_started_notify                 0x00000c39   Thumb Code    34  nrf_drv_clock.o(i.clock_clk_started_notify)
    i.clock_irq_handler                      0x00000c60   Section        0  nrf_drv_clock.o(i.clock_irq_handler)
    clock_irq_handler                        0x00000c61   Thumb Code    24  nrf_drv_clock.o(i.clock_irq_handler)
    i.compare_func                           0x00000c7c   Section        0  app_timer2.o(i.compare_func)
    compare_func                             0x00000c7d   Thumb Code    24  app_timer2.o(i.compare_func)
    i.dropped_sat16_get                      0x00000c94   Section        0  nrf_log_frontend.o(i.dropped_sat16_get)
    dropped_sat16_get                        0x00000c95   Thumb Code    16  nrf_log_frontend.o(i.dropped_sat16_get)
    i.drv_rtc_counter_get                    0x00000ca8   Section        0  drv_rtc.o(i.drv_rtc_counter_get)
    i.drv_rtc_irq_trigger                    0x00000cb0   Section        0  drv_rtc.o(i.drv_rtc_irq_trigger)
    i.get_now                                0x00000cd0   Section        0  app_timer2.o(i.get_now)
    get_now                                  0x00000cd1   Thumb Code    46  app_timer2.o(i.get_now)
    i.int_print                              0x00000d04   Section        0  nrf_fprintf_format.o(i.int_print)
    int_print                                0x00000d05   Thumb Code   166  nrf_fprintf_format.o(i.int_print)
    i.invalid_packets_omit                   0x00000daa   Section        0  nrf_log_frontend.o(i.invalid_packets_omit)
    invalid_packets_omit                     0x00000dab   Thumb Code    52  nrf_log_frontend.o(i.invalid_packets_omit)
    i.irq_handler                            0x00000de0   Section        0  nrfx_rtc.o(i.irq_handler)
    irq_handler                              0x00000de1   Thumb Code   154  nrfx_rtc.o(i.irq_handler)
    i.irq_handler                            0x00000e80   Section        0  nrfx_timer.o(i.irq_handler)
    irq_handler                              0x00000e81   Thumb Code    70  nrfx_timer.o(i.irq_handler)
    i.irq_handler                            0x00000ec8   Section        0  nrf_libuarte_drv.o(i.irq_handler)
    irq_handler                              0x00000ec9   Thumb Code   512  nrf_libuarte_drv.o(i.irq_handler)
    i.is_allocated_channel                   0x000010cc   Section        0  nrfx_ppi.o(i.is_allocated_channel)
    is_allocated_channel                     0x000010cd   Thumb Code    20  nrfx_ppi.o(i.is_allocated_channel)
    i.is_allocated_group                     0x000010e4   Section        0  nrfx_ppi.o(i.is_allocated_group)
    is_allocated_group                       0x000010e5   Thumb Code    20  nrfx_ppi.o(i.is_allocated_group)
    i.is_app_group                           0x000010fc   Section        0  nrfx_ppi.o(i.is_app_group)
    is_app_group                             0x000010fd   Thumb Code    12  nrfx_ppi.o(i.is_app_group)
    i.is_programmable_app_channel            0x00001108   Section        0  nrfx_ppi.o(i.is_programmable_app_channel)
    is_programmable_app_channel              0x00001109   Thumb Code    12  nrfx_ppi.o(i.is_programmable_app_channel)
    i.item_enqueue                           0x00001114   Section        0  nrf_drv_clock.o(i.item_enqueue)
    item_enqueue                             0x00001115   Thumb Code    22  nrf_drv_clock.o(i.item_enqueue)
    i.libuarte1_rtc_handler                  0x0000112c   Section        0  main.o(i.libuarte1_rtc_handler)
    libuarte1_rtc_handler                    0x0000112d   Thumb Code    30  main.o(i.libuarte1_rtc_handler)
    i.libuarte_rtc_handler                   0x00001154   Section        0  main.o(i.libuarte_rtc_handler)
    libuarte_rtc_handler                     0x00001155   Thumb Code    30  main.o(i.libuarte_rtc_handler)
    i.log_pending_hook                       0x0000117c   Section        0  nrf_log_frontend.o(i.log_pending_hook)
    i.log_skip                               0x00001180   Section        0  nrf_log_frontend.o(i.log_skip)
    log_skip                                 0x00001181   Thumb Code   150  nrf_log_frontend.o(i.log_skip)
    i.main                                   0x00001224   Section        0  main.o(i.main)
    i.memobj_op                              0x000012d0   Section        0  nrf_memobj.o(i.memobj_op)
    memobj_op                                0x000012d1   Thumb Code   126  nrf_memobj.o(i.memobj_op)
    i.module_idx_get                         0x00001350   Section        0  nrf_log_frontend.o(i.module_idx_get)
    module_idx_get                           0x00001351   Thumb Code    42  nrf_log_frontend.o(i.module_idx_get)
    i.nrf_atfifo_item_alloc                  0x00001380   Section        0  nrf_atfifo.o(i.nrf_atfifo_item_alloc)
    i.nrf_atfifo_item_put                    0x00001396   Section        0  nrf_atfifo.o(i.nrf_atfifo_item_put)
    i.nrf_atomic_flag_clear_fetch            0x000013ac   Section        0  nrf_atomic.o(i.nrf_atomic_flag_clear_fetch)
    i.nrf_atomic_flag_set                    0x000013b2   Section        0  nrf_atomic.o(i.nrf_atomic_flag_set)
    i.nrf_atomic_u32_add                     0x000013b8   Section        0  nrf_atomic.o(i.nrf_atomic_u32_add)
    i.nrf_atomic_u32_fetch_and               0x000013c4   Section        0  nrf_atomic.o(i.nrf_atomic_u32_fetch_and)
    i.nrf_atomic_u32_fetch_store             0x000013ce   Section        0  nrf_atomic.o(i.nrf_atomic_u32_fetch_store)
    i.nrf_atomic_u32_or                      0x000013d8   Section        0  nrf_atomic.o(i.nrf_atomic_u32_or)
    i.nrf_atomic_u32_sub                     0x000013e4   Section        0  nrf_atomic.o(i.nrf_atomic_u32_sub)
    i.nrf_balloc_alloc                       0x000013f0   Section        0  nrf_balloc.o(i.nrf_balloc_alloc)
    i.nrf_balloc_free                        0x0000142e   Section        0  nrf_balloc.o(i.nrf_balloc_free)
    i.nrf_balloc_init                        0x00001458   Section        0  nrf_balloc.o(i.nrf_balloc_init)
    i.nrf_clock_event_check                  0x00001488   Section        0  nrfx_clock.o(i.nrf_clock_event_check)
    nrf_clock_event_check                    0x00001489   Thumb Code    14  nrfx_clock.o(i.nrf_clock_event_check)
    i.nrf_clock_event_clear                  0x00001496   Section        0  nrfx_clock.o(i.nrf_clock_event_clear)
    nrf_clock_event_clear                    0x00001497   Thumb Code    16  nrfx_clock.o(i.nrf_clock_event_clear)
    i.nrf_drv_clock_init                     0x000014a8   Section        0  nrf_drv_clock.o(i.nrf_drv_clock_init)
    i.nrf_drv_clock_lfclk_request            0x000014e4   Section        0  nrf_drv_clock.o(i.nrf_drv_clock_lfclk_request)
    i.nrf_fprintf                            0x0000152c   Section        0  nrf_fprintf.o(i.nrf_fprintf)
    i.nrf_fprintf_buffer_flush               0x00001546   Section        0  nrf_fprintf.o(i.nrf_fprintf_buffer_flush)
    i.nrf_fprintf_fmt                        0x0000155e   Section        0  nrf_fprintf_format.o(i.nrf_fprintf_fmt)
    i.nrf_gpio_cfg                           0x00001738   Section        0  nrf_libuarte_drv.o(i.nrf_gpio_cfg)
    nrf_gpio_cfg                             0x00001739   Thumb Code    50  nrf_libuarte_drv.o(i.nrf_gpio_cfg)
    i.nrf_gpio_cfg_output                    0x0000176a   Section        0  nrf_libuarte_drv.o(i.nrf_gpio_cfg_output)
    nrf_gpio_cfg_output                      0x0000176b   Thumb Code    20  nrf_libuarte_drv.o(i.nrf_gpio_cfg_output)
    i.nrf_gpio_pin_port_decode               0x00001780   Section        0  boards.o(i.nrf_gpio_pin_port_decode)
    nrf_gpio_pin_port_decode                 0x00001781   Thumb Code    22  boards.o(i.nrf_gpio_pin_port_decode)
    i.nrf_gpio_pin_port_decode               0x0000179c   Section        0  nrf_libuarte_drv.o(i.nrf_gpio_pin_port_decode)
    nrf_gpio_pin_port_decode                 0x0000179d   Thumb Code    22  nrf_libuarte_drv.o(i.nrf_gpio_pin_port_decode)
    i.nrf_libuarte_async_enable              0x000017b8   Section        0  nrf_libuarte_async.o(i.nrf_libuarte_async_enable)
    i.nrf_libuarte_async_init                0x00001858   Section        0  nrf_libuarte_async.o(i.nrf_libuarte_async_init)
    i.nrf_libuarte_async_rx_free             0x00001a68   Section        0  nrf_libuarte_async.o(i.nrf_libuarte_async_rx_free)
    i.nrf_libuarte_async_timeout_handler     0x00001ac4   Section        0  nrf_libuarte_async.o(i.nrf_libuarte_async_timeout_handler)
    i.nrf_libuarte_async_tx                  0x00001b4e   Section        0  nrf_libuarte_async.o(i.nrf_libuarte_async_tx)
    i.nrf_libuarte_drv_init                  0x00001b54   Section        0  nrf_libuarte_drv.o(i.nrf_libuarte_drv_init)
    i.nrf_libuarte_drv_rx_buf_rsp            0x00001ce4   Section        0  nrf_libuarte_drv.o(i.nrf_libuarte_drv_rx_buf_rsp)
    i.nrf_libuarte_drv_rx_start              0x00001cfe   Section        0  nrf_libuarte_drv.o(i.nrf_libuarte_drv_rx_start)
    i.nrf_libuarte_drv_tx                    0x00001d6c   Section        0  nrf_libuarte_drv.o(i.nrf_libuarte_drv_tx)
    i.nrf_log_backend_add                    0x00001e1c   Section        0  nrf_log_frontend.o(i.nrf_log_backend_add)
    i.nrf_log_backend_rtt_flush              0x00001e78   Section        0  nrf_log_backend_rtt.o(i.nrf_log_backend_rtt_flush)
    nrf_log_backend_rtt_flush                0x00001e79   Thumb Code     2  nrf_log_backend_rtt.o(i.nrf_log_backend_rtt_flush)
    i.nrf_log_backend_rtt_init               0x00001e7a   Section        0  nrf_log_backend_rtt.o(i.nrf_log_backend_rtt_init)
    i.nrf_log_backend_rtt_panic_set          0x00001e7e   Section        0  nrf_log_backend_rtt.o(i.nrf_log_backend_rtt_panic_set)
    nrf_log_backend_rtt_panic_set            0x00001e7f   Thumb Code     2  nrf_log_backend_rtt.o(i.nrf_log_backend_rtt_panic_set)
    i.nrf_log_backend_rtt_put                0x00001e80   Section        0  nrf_log_backend_rtt.o(i.nrf_log_backend_rtt_put)
    nrf_log_backend_rtt_put                  0x00001e81   Thumb Code    16  nrf_log_backend_rtt.o(i.nrf_log_backend_rtt_put)
    i.nrf_log_backend_serial_put             0x00001e98   Section        0  nrf_log_backend_serial.o(i.nrf_log_backend_serial_put)
    i.nrf_log_color_id_get                   0x00001f60   Section        0  nrf_log_frontend.o(i.nrf_log_color_id_get)
    i.nrf_log_default_backends_init          0x00001f90   Section        0  nrf_log_default_backends.o(i.nrf_log_default_backends_init)
    i.nrf_log_frontend_dequeue               0x00001fac   Section        0  nrf_log_frontend.o(i.nrf_log_frontend_dequeue)
    i.nrf_log_frontend_std_0                 0x000021e0   Section        0  nrf_log_frontend.o(i.nrf_log_frontend_std_0)
    i.nrf_log_frontend_std_1                 0x000021e8   Section        0  nrf_log_frontend.o(i.nrf_log_frontend_std_1)
    i.nrf_log_frontend_std_2                 0x000021f6   Section        0  nrf_log_frontend.o(i.nrf_log_frontend_std_2)
    i.nrf_log_frontend_std_3                 0x00002206   Section        0  nrf_log_frontend.o(i.nrf_log_frontend_std_3)
    i.nrf_log_hexdump_entry_process          0x00002218   Section        0  nrf_log_str_formatter.o(i.nrf_log_hexdump_entry_process)
    i.nrf_log_init                           0x000022c8   Section        0  nrf_log_frontend.o(i.nrf_log_init)
    i.nrf_log_module_cnt_get                 0x000022f0   Section        0  nrf_log_frontend.o(i.nrf_log_module_cnt_get)
    i.nrf_log_module_name_get                0x00002304   Section        0  nrf_log_frontend.o(i.nrf_log_module_name_get)
    i.nrf_log_panic                          0x00002320   Section        0  nrf_log_frontend.o(i.nrf_log_panic)
    i.nrf_log_std_entry_process              0x00002348   Section        0  nrf_log_str_formatter.o(i.nrf_log_std_entry_process)
    i.nrf_memobj_alloc                       0x000023fe   Section        0  nrf_memobj.o(i.nrf_memobj_alloc)
    i.nrf_memobj_free                        0x0000245e   Section        0  nrf_memobj.o(i.nrf_memobj_free)
    i.nrf_memobj_get                         0x00002490   Section        0  nrf_memobj.o(i.nrf_memobj_get)
    i.nrf_memobj_pool_init                   0x00002498   Section        0  nrf_memobj.o(i.nrf_memobj_pool_init)
    i.nrf_memobj_put                         0x0000249c   Section        0  nrf_memobj.o(i.nrf_memobj_put)
    i.nrf_memobj_read                        0x000024ba   Section        0  nrf_memobj.o(i.nrf_memobj_read)
    i.nrf_memobj_write                       0x000024ca   Section        0  nrf_memobj.o(i.nrf_memobj_write)
    i.nrf_queue_generic_pop                  0x000024da   Section        0  nrf_queue.o(i.nrf_queue_generic_pop)
    i.nrf_queue_is_empty                     0x00002562   Section        0  nrf_queue.o(i.nrf_queue_is_empty)
    i.nrf_queue_is_full                      0x00002574   Section        0  nrf_queue.o(i.nrf_queue_is_full)
    i.nrf_queue_next_idx                     0x00002592   Section        0  nrf_queue.o(i.nrf_queue_next_idx)
    nrf_queue_next_idx                       0x00002593   Thumb Code    14  nrf_queue.o(i.nrf_queue_next_idx)
    i.nrf_queue_push                         0x000025a0   Section        0  nrf_queue.o(i.nrf_queue_push)
    i.nrf_queue_reset                        0x0000264c   Section        0  nrf_queue.o(i.nrf_queue_reset)
    i.nrf_ringbuf_init                       0x0000266a   Section        0  nrf_ringbuf.o(i.nrf_ringbuf_init)
    i.nrf_rtc_event_clear                    0x00002686   Section        0  nrfx_rtc.o(i.nrf_rtc_event_clear)
    nrf_rtc_event_clear                      0x00002687   Thumb Code    12  nrfx_rtc.o(i.nrf_rtc_event_clear)
    i.nrf_strerror_find                      0x00002694   Section        0  nrf_strerror.o(i.nrf_strerror_find)
    i.nrf_strerror_get                       0x000026cc   Section        0  nrf_strerror.o(i.nrf_strerror_get)
    i.nrf_timer_event_clear                  0x000026e0   Section        0  nrfx_timer.o(i.nrf_timer_event_clear)
    nrf_timer_event_clear                    0x000026e1   Thumb Code    12  nrfx_timer.o(i.nrf_timer_event_clear)
    i.nrf_uarte_event_check                  0x000026ec   Section        0  nrf_libuarte_drv.o(i.nrf_uarte_event_check)
    nrf_uarte_event_check                    0x000026ed   Thumb Code    10  nrf_libuarte_drv.o(i.nrf_uarte_event_check)
    i.nrf_uarte_event_clear                  0x000026f6   Section        0  nrf_libuarte_drv.o(i.nrf_uarte_event_clear)
    nrf_uarte_event_clear                    0x000026f7   Thumb Code    12  nrf_libuarte_drv.o(i.nrf_uarte_event_clear)
    i.nrf_wdt_started                        0x00002704   Section        0  nrf_drv_clock.o(i.nrf_wdt_started)
    nrf_wdt_started                          0x00002705   Thumb Code    12  nrf_drv_clock.o(i.nrf_wdt_started)
    i.nrfx_clock_enable                      0x00002714   Section        0  nrfx_clock.o(i.nrfx_clock_enable)
    i.nrfx_clock_init                        0x00002740   Section        0  nrfx_clock.o(i.nrfx_clock_init)
    i.nrfx_clock_lfclk_start                 0x00002760   Section        0  nrfx_clock.o(i.nrfx_clock_lfclk_start)
    i.nrfx_ppi_channel_alloc                 0x00002780   Section        0  nrfx_ppi.o(i.nrfx_ppi_channel_alloc)
    i.nrfx_ppi_channel_assign                0x00002854   Section        0  nrfx_ppi.o(i.nrfx_ppi_channel_assign)
    i.nrfx_ppi_channel_disable               0x0000293c   Section        0  nrfx_ppi.o(i.nrfx_ppi_channel_disable)
    i.nrfx_ppi_channel_enable                0x000029b0   Section        0  nrfx_ppi.o(i.nrfx_ppi_channel_enable)
    i.nrfx_ppi_channel_fork_assign           0x00002a24   Section        0  nrfx_ppi.o(i.nrfx_ppi_channel_fork_assign)
    i.nrfx_ppi_channel_free                  0x00002adc   Section        0  nrfx_ppi.o(i.nrfx_ppi_channel_free)
    i.nrfx_ppi_channels_include_in_group     0x00002b60   Section        0  nrfx_ppi.o(i.nrfx_ppi_channels_include_in_group)
    i.nrfx_ppi_group_alloc                   0x00002bf0   Section        0  nrfx_ppi.o(i.nrfx_ppi_group_alloc)
    i.nrfx_ppi_group_enable                  0x00002cc0   Section        0  nrfx_ppi.o(i.nrfx_ppi_group_enable)
    i.nrfx_ppi_group_free                    0x00002d38   Section        0  nrfx_ppi.o(i.nrfx_ppi_group_free)
    i.nrfx_rtc_cc_set                        0x00002dc8   Section        0  nrfx_rtc.o(i.nrfx_rtc_cc_set)
    i.nrfx_rtc_init                          0x00002e4c   Section        0  nrfx_rtc.o(i.nrfx_rtc_init)
    i.nrfx_timer_clear                       0x00002edc   Section        0  nrfx_timer.o(i.nrfx_timer_clear)
    i.nrfx_timer_compare                     0x00002ee4   Section        0  nrfx_timer.o(i.nrfx_timer_compare)
    i.nrfx_timer_enable                      0x00002f20   Section        0  nrfx_timer.o(i.nrfx_timer_enable)
    i.nrfx_timer_init                        0x00002f3c   Section        0  nrfx_timer.o(i.nrfx_timer_init)
    i.nvmc_config                            0x00002ffc   Section        0  system_nrf52.o(i.nvmc_config)
    i.postfix_process                        0x00003014   Section        0  nrf_log_str_formatter.o(i.postfix_process)
    postfix_process                          0x00003015   Thumb Code    48  nrf_log_str_formatter.o(i.postfix_process)
    i.ppi_ch_disable                         0x00003050   Section        0  nrf_libuarte_drv.o(i.ppi_ch_disable)
    ppi_ch_disable                           0x00003051   Thumb Code     6  nrf_libuarte_drv.o(i.ppi_ch_disable)
    i.ppi_ch_enable                          0x00003056   Section        0  nrf_libuarte_drv.o(i.ppi_ch_enable)
    ppi_ch_enable                            0x00003057   Thumb Code     6  nrf_libuarte_drv.o(i.ppi_ch_enable)
    i.ppi_channel_configure                  0x0000305c   Section        0  nrf_libuarte_drv.o(i.ppi_channel_configure)
    ppi_channel_configure                    0x0000305d   Thumb Code    56  nrf_libuarte_drv.o(i.ppi_channel_configure)
    i.ppi_configure                          0x00003094   Section        0  nrf_libuarte_drv.o(i.ppi_configure)
    ppi_configure                            0x00003095   Thumb Code   284  nrf_libuarte_drv.o(i.ppi_configure)
    i.ppi_free                               0x000031b0   Section        0  nrf_libuarte_drv.o(i.ppi_free)
    ppi_free                                 0x000031b1   Thumb Code    74  nrf_libuarte_drv.o(i.ppi_free)
    i.ppi_group_configure                    0x000031fc   Section        0  nrf_libuarte_drv.o(i.ppi_group_configure)
    ppi_group_configure                      0x000031fd   Thumb Code    82  nrf_libuarte_drv.o(i.ppi_group_configure)
    i.prefix_process                         0x00003254   Section        0  nrf_log_str_formatter.o(i.prefix_process)
    prefix_process                           0x00003255   Thumb Code    90  nrf_log_str_formatter.o(i.prefix_process)
    i.queue_utilization_get                  0x000032ec   Section        0  nrf_queue.o(i.queue_utilization_get)
    queue_utilization_get                    0x000032ed   Thumb Code    24  nrf_queue.o(i.queue_utilization_get)
    i.rx_buffer_schedule                     0x00003304   Section        0  nrf_libuarte_async.o(i.rx_buffer_schedule)
    rx_buffer_schedule                       0x00003305   Thumb Code    52  nrf_libuarte_async.o(i.rx_buffer_schedule)
    i.serial_tx                              0x00003338   Section        0  nrf_log_backend_rtt.o(i.serial_tx)
    serial_tx                                0x00003339   Thumb Code    70  nrf_log_backend_rtt.o(i.serial_tx)
    i.std_n                                  0x00003388   Section        0  nrf_log_frontend.o(i.std_n)
    std_n                                    0x00003389   Thumb Code   144  nrf_log_frontend.o(i.std_n)
    i.timer_req_schedule                     0x00003420   Section        0  app_timer2.o(i.timer_req_schedule)
    timer_req_schedule                       0x00003421   Thumb Code    46  app_timer2.o(i.timer_req_schedule)
    i.tmr_evt_handler                        0x00003458   Section        0  nrf_libuarte_async.o(i.tmr_evt_handler)
    tmr_evt_handler                          0x00003459   Thumb Code     6  nrf_libuarte_async.o(i.tmr_evt_handler)
    i.tmr_evt_handler                        0x0000345e   Section        0  nrf_libuarte_drv.o(i.tmr_evt_handler)
    i.tx_ppi_disable                         0x00003460   Section        0  nrf_libuarte_drv.o(i.tx_ppi_disable)
    tx_ppi_disable                           0x00003461   Thumb Code    16  nrf_libuarte_drv.o(i.tx_ppi_disable)
    i.uart_event_handler                     0x00003470   Section        0  main.o(i.uart_event_handler)
    i.uart_evt_handler                       0x000034fc   Section        0  nrf_libuarte_async.o(i.uart_evt_handler)
    uart_evt_handler                         0x000034fd   Thumb Code   202  nrf_libuarte_async.o(i.uart_evt_handler)
    i.unsigned_print                         0x000035cc   Section        0  nrf_fprintf_format.o(i.unsigned_print)
    unsigned_print                           0x000035cd   Thumb Code   176  nrf_fprintf_format.o(i.unsigned_print)
    .constdata                               0x00003680   Section       16  main.o(.constdata)
    libuarte_libuarte                        0x00003680   Data          16  main.o(.constdata)
    .constdata                               0x00003690   Section      160  main.o(.constdata)
    libuarte_rtc                             0x00003690   Data           8  main.o(.constdata)
    libuarte1_rtc                            0x00003698   Data           8  main.o(.constdata)
    libuarte                                 0x000036a0   Data          40  main.o(.constdata)
    libuarte1                                0x000036c8   Data          40  main.o(.constdata)
    .constdata                               0x00003730   Section       16  main.o(.constdata)
    libuarte1_libuarte                       0x00003730   Data          16  main.o(.constdata)
    .constdata                               0x00003740   Section        4  boards.o(.constdata)
    m_board_led_list                         0x00003740   Data           4  boards.o(.constdata)
    .constdata                               0x00003744   Section      304  nrfx_ppi.o(.constdata)
    __func__                                 0x00003744   Data          23  nrfx_ppi.o(.constdata)
    __func__                                 0x0000375b   Data          22  nrfx_ppi.o(.constdata)
    __func__                                 0x00003771   Data          24  nrfx_ppi.o(.constdata)
    __func__                                 0x00003789   Data          29  nrfx_ppi.o(.constdata)
    __func__                                 0x000037a6   Data          24  nrfx_ppi.o(.constdata)
    __func__                                 0x000037be   Data          25  nrfx_ppi.o(.constdata)
    __func__                                 0x000037d7   Data          21  nrfx_ppi.o(.constdata)
    __func__                                 0x000037ec   Data          20  nrfx_ppi.o(.constdata)
    __func__                                 0x00003800   Data          22  nrfx_ppi.o(.constdata)
    __func__                                 0x00003816   Data          23  nrfx_ppi.o(.constdata)
    __func__                                 0x0000382d   Data          36  nrfx_ppi.o(.constdata)
    __func__                                 0x00003851   Data          35  nrfx_ppi.o(.constdata)
    .constdata                               0x00003874   Section       20  app_timer2.o(.constdata)
    m_req_fifo                               0x00003874   Data           4  app_timer2.o(.constdata)
    m_app_timer_sortlist                     0x0000387c   Data          12  app_timer2.o(.constdata)
    .constdata                               0x00003888   Section       16  nrf_fprintf_format.o(.constdata)
    _aV2C                                    0x00003888   Data          16  nrf_fprintf_format.o(.constdata)
    .constdata                               0x00003898   Section       52  nrf_libuarte_async.o(.constdata)
    .constdata                               0x000038cc   Section       60  nrf_libuarte_drv.o(.constdata)
    .constdata                               0x00003908   Section      300  nrf_strerror.o(.constdata)
    m_unknown_str                            0x00003908   Data          19  nrf_strerror.o(.constdata)
    nrf_strerror_array                       0x0000391c   Data         280  nrf_strerror.o(.constdata)
    .constdata                               0x00003a34   Section       12  nrf_log_backend_rtt.o(.constdata)
    .constdata                               0x00003a40   Section        6  nrf_log_backend_rtt.o(.constdata)
    delay_machine_code                       0x00003a40   Data           6  nrf_log_backend_rtt.o(.constdata)
    .constdata                               0x00003a48   Section       12  nrf_log_frontend.o(.constdata)
    m_log_push_ringbuf                       0x00003a48   Data          12  nrf_log_frontend.o(.constdata)
    .constdata                               0x00003a54   Section      129  ctype_o.o(.constdata)
    .constdata                               0x00003ad8   Section        4  ctype_o.o(.constdata)
    table                                    0x00003ad8   Data           4  ctype_o.o(.constdata)
    .conststring                             0x00003adc   Section      959  nrf_strerror.o(.conststring)
    .conststring                             0x00003e9c   Section      102  nrf_log_str_formatter.o(.conststring)
    .conststrlit                             0x00003f04   Section        6  nrf_drv_clock.o(.conststrlit)
    .conststrlit                             0x00003f0c   Section        6  nrfx_clock.o(.conststrlit)
    .conststrlit                             0x00003f14   Section        4  nrfx_ppi.o(.conststrlit)
    .conststrlit                             0x00003f18   Section        4  nrfx_rtc.o(.conststrlit)
    .conststrlit                             0x00003f1c   Section        6  nrfx_timer.o(.conststrlit)
    .conststrlit                             0x00003f24   Section       10  app_timer2.o(.conststrlit)
    .conststrlit                             0x00003f30   Section       15  nrf_libuarte_async.o(.conststrlit)
    .conststrlit                             0x00003f40   Section        9  nrf_libuarte_drv.o(.conststrlit)
    .conststrlit                             0x00003f4c   Section        9  nrf_sortlist.o(.conststrlit)
    .conststrlit                             0x00003f58   Section       16  nrf_log_default_backends.o(.conststrlit)
    .conststrlit                             0x00003f68   Section        4  nrf_log_frontend.o(.conststrlit)
    log_backends                             0x00003f8c   Section       16  nrf_log_default_backends.o(log_backends)
    __tagsym$$used                           0x00003f8c   Number         0  nrf_log_default_backends.o(log_backends)
    rtt_log_backend                          0x00003f8c   Data          16  nrf_log_default_backends.o(log_backends)
    log_const_data                           0x00003f9c   Section        8  nrf_drv_clock.o(log_const_data)
    __tagsym$$used                           0x00003f9c   Number         0  nrf_drv_clock.o(log_const_data)
    log_const_data                           0x00003fa4   Section        8  nrfx_clock.o(log_const_data)
    __tagsym$$used                           0x00003fa4   Number         0  nrfx_clock.o(log_const_data)
    log_const_data                           0x00003fac   Section        8  nrfx_ppi.o(log_const_data)
    __tagsym$$used                           0x00003fac   Number         0  nrfx_ppi.o(log_const_data)
    log_const_data                           0x00003fb4   Section        8  nrfx_rtc.o(log_const_data)
    __tagsym$$used                           0x00003fb4   Number         0  nrfx_rtc.o(log_const_data)
    log_const_data                           0x00003fbc   Section        8  nrfx_timer.o(log_const_data)
    __tagsym$$used                           0x00003fbc   Number         0  nrfx_timer.o(log_const_data)
    log_const_data                           0x00003fc4   Section        8  app_timer2.o(log_const_data)
    __tagsym$$used                           0x00003fc4   Number         0  app_timer2.o(log_const_data)
    log_const_data                           0x00003fcc   Section        8  nrf_libuarte_async.o(log_const_data)
    __tagsym$$used                           0x00003fcc   Number         0  nrf_libuarte_async.o(log_const_data)
    log_const_data                           0x00003fd4   Section        8  nrf_libuarte_drv.o(log_const_data)
    __tagsym$$used                           0x00003fd4   Number         0  nrf_libuarte_drv.o(log_const_data)
    log_const_data                           0x00003fdc   Section        8  nrf_sortlist.o(log_const_data)
    __tagsym$$used                           0x00003fdc   Number         0  nrf_sortlist.o(log_const_data)
    log_const_data                           0x00003fe4   Section        8  nrf_log_frontend.o(log_const_data)
    __tagsym$$used                           0x00003fe4   Number         0  nrf_log_frontend.o(log_const_data)
    nrf_balloc                               0x00003fec   Section       40  main.o(nrf_balloc)
    __tagsym$$used                           0x00003fec   Number         0  main.o(nrf_balloc)
    __tagsym$$used                           0x00004000   Number         0  main.o(nrf_balloc)
    nrf_balloc                               0x00004014   Section       20  nrf_log_frontend.o(nrf_balloc)
    __tagsym$$used                           0x00004014   Number         0  nrf_log_frontend.o(nrf_balloc)
    nrf_queue                                0x00004028   Section       60  main.o(nrf_queue)
    __tagsym$$used                           0x00004028   Number         0  main.o(nrf_queue)
    __tagsym$$used                           0x0000403c   Number         0  main.o(nrf_queue)
    __tagsym$$used                           0x00004050   Number         0  main.o(nrf_queue)
    .data                                    0x20000000   Section       38  main.o(.data)
    text_size                                0x20000000   Data           1  main.o(.data)
    m_loopback_phase                         0x20000001   Data           1  main.o(.data)
    text                                     0x20000002   Data          36  main.o(.data)
    .data                                    0x20000026   Section        3  main.o(.data)
    libuarte_rx_pool_nrf_balloc_pool_stack   0x20000026   Data           3  main.o(.data)
    .data                                    0x2000002c   Section        8  main.o(.data)
    libuarte_rx_pool_nrf_balloc_cb           0x2000002c   Data           8  main.o(.data)
    .data                                    0x20000034   Section        3  main.o(.data)
    libuarte1_rx_pool_nrf_balloc_pool_stack  0x20000034   Data           3  main.o(.data)
    .data                                    0x20000038   Section        8  main.o(.data)
    libuarte1_rx_pool_nrf_balloc_cb          0x20000038   Data           8  main.o(.data)
    .data                                    0x20000040   Section        8  nrfx_clock.o(.data)
    m_clock_cb                               0x20000040   Data           8  nrfx_clock.o(.data)
    .data                                    0x20000048   Section        8  nrfx_ppi.o(.data)
    m_groups_allocated                       0x20000048   Data           1  nrfx_ppi.o(.data)
    m_channels_allocated                     0x2000004c   Data           4  nrfx_ppi.o(.data)
    .data                                    0x20000050   Section       16  nrfx_rtc.o(.data)
    m_cb                                     0x20000050   Data           6  nrfx_rtc.o(.data)
    m_handlers                               0x20000058   Data           8  nrfx_rtc.o(.data)
    .data                                    0x20000060   Section       32  app_timer2.o(.data)
    m_global_active                          0x20000060   Data           1  app_timer2.o(.data)
    mp_active_timer                          0x20000064   Data           4  app_timer2.o(.data)
    m_rtc_inst                               0x20000068   Data           8  app_timer2.o(.data)
    m_base_counter                           0x20000070   Data           8  app_timer2.o(.data)
    m_stamp64                                0x20000078   Data           8  app_timer2.o(.data)
    .data                                    0x20000080   Section        4  app_timer2.o(.data)
    m_app_timer_sortlist_sortlist_cb         0x20000080   Data           4  app_timer2.o(.data)
    .data                                    0x20000084   Section        4  app_util_platform.o(.data)
    m_in_critical_region                     0x20000084   Data           4  app_util_platform.o(.data)
    .data                                    0x20000088   Section       12  drv_rtc.o(.data)
    m_handlers                               0x20000088   Data           4  drv_rtc.o(.data)
    m_cb                                     0x2000008c   Data           8  drv_rtc.o(.data)
    .data                                    0x20000094   Section        8  nrf_libuarte_drv.o(.data)
    m_libuarte_instance                      0x20000094   Data           8  nrf_libuarte_drv.o(.data)
    .data                                    0x2000009c   Section        1  nrf_log_backend_rtt.o(.data)
    m_host_present                           0x2000009c   Data           1  nrf_log_backend_rtt.o(.data)
    .data                                    0x200000a0   Section        8  nrf_log_default_backends.o(.data)
    log_backend_cb_rtt_log_backend           0x200000a0   Data           8  nrf_log_default_backends.o(.data)
    .data                                    0x200000a8   Section        4  nrf_log_frontend.o(.data)
    m_buffer_mask                            0x200000a8   Data           4  nrf_log_frontend.o(.data)
    .data                                    0x200000ac   Section        8  nrf_log_frontend.o(.data)
    log_mempool_nrf_balloc_pool_stack        0x200000ac   Data           8  nrf_log_frontend.o(.data)
    .data                                    0x200000b4   Section        8  nrf_log_frontend.o(.data)
    log_mempool_nrf_balloc_cb                0x200000b4   Data           8  nrf_log_frontend.o(.data)
    .data                                    0x200000bc   Section       64  nrf_log_str_formatter.o(.data)
    m_freq                                   0x200000bc   Data           4  nrf_log_str_formatter.o(.data)
    m_timestamp_div                          0x200000c0   Data           4  nrf_log_str_formatter.o(.data)
    severity_names                           0x200000c4   Data          20  nrf_log_str_formatter.o(.data)
    m_colors                                 0x200000d8   Data          36  nrf_log_str_formatter.o(.data)
    .data                                    0x200000fc   Section        4  system_nrf52.o(.data)
    __tagsym$$used                           0x200000fc   Number         0  system_nrf52.o(.data)
    .bss                                     0x20000100   Section       64  main.o(.bss)
    libuarte_libuartectrl_blk                0x20000100   Data          64  main.o(.bss)
    .bss                                     0x20000140   Section       16  main.o(.bss)
    libuarte_rxdata_queue_nrf_queue_buffer   0x20000140   Data          16  main.o(.bss)
    .bss                                     0x20000150   Section       12  main.o(.bss)
    libuarte_rxdata_queue_nrf_queue_cb       0x20000150   Data          12  main.o(.bss)
    .bss                                     0x2000015c   Section      768  main.o(.bss)
    libuarte_rx_pool_nrf_balloc_pool_mem     0x2000015c   Data         768  main.o(.bss)
    .bss                                     0x2000045c   Section       80  main.o(.bss)
    libuartectrl_blk                         0x2000045c   Data          40  main.o(.bss)
    libuarte1ctrl_blk                        0x20000484   Data          40  main.o(.bss)
    .bss                                     0x200004ac   Section       64  main.o(.bss)
    libuarte1_libuartectrl_blk               0x200004ac   Data          64  main.o(.bss)
    .bss                                     0x200004ec   Section       16  main.o(.bss)
    libuarte1_rxdata_queue_nrf_queue_buffer  0x200004ec   Data          16  main.o(.bss)
    .bss                                     0x200004fc   Section       12  main.o(.bss)
    libuarte1_rxdata_queue_nrf_queue_cb      0x200004fc   Data          12  main.o(.bss)
    .bss                                     0x20000508   Section      768  main.o(.bss)
    libuarte1_rx_pool_nrf_balloc_pool_mem    0x20000508   Data         768  main.o(.bss)
    .bss                                     0x20000808   Section       88  main.o(.bss)
    m_buf_queue_nrf_queue_buffer             0x20000808   Data          88  main.o(.bss)
    .bss                                     0x20000860   Section       12  main.o(.bss)
    m_buf_queue_nrf_queue_cb                 0x20000860   Data          12  main.o(.bss)
    .bss                                     0x2000086c   Section       20  nrf_drv_clock.o(.bss)
    m_clock_cb                               0x2000086c   Data          20  nrf_drv_clock.o(.bss)
    .bss                                     0x20000880   Section       24  nrfx_timer.o(.bss)
    m_cb                                     0x20000880   Data          24  nrfx_timer.o(.bss)
    .bss                                     0x20000898   Section       16  app_timer2.o(.bss)
    m_req_fifo_inst                          0x20000898   Data          16  app_timer2.o(.bss)
    .bss                                     0x200008a8   Section       64  nrf_log_backend_rtt.o(.bss)
    m_string_buff                            0x200008a8   Data          64  nrf_log_backend_rtt.o(.bss)
    .bss                                     0x200008e8   Section      192  nrf_log_frontend.o(.bss)
    log_mempool_nrf_balloc_pool_mem          0x200008e8   Data         192  nrf_log_frontend.o(.bss)
    .bss                                     0x200009a8   Section      128  nrf_log_frontend.o(.bss)
    m_log_push_ringbuf_buf                   0x200009a8   Data         128  nrf_log_frontend.o(.bss)
    .bss                                     0x20000a28   Section       24  nrf_log_frontend.o(.bss)
    m_log_push_ringbuf_cb                    0x20000a28   Data          24  nrf_log_frontend.o(.bss)
    .bss                                     0x20000a40   Section     1056  nrf_log_frontend.o(.bss)
    m_log_data                               0x20000a40   Data        1056  nrf_log_frontend.o(.bss)
    .bss                                     0x20000e60   Section      648  segger_rtt.o(.bss)
    _acUpBuffer                              0x20000ed8   Data         512  segger_rtt.o(.bss)
    _acDownBuffer                            0x200010d8   Data          16  segger_rtt.o(.bss)
    STACK                                    0x200010e8   Section     8192  arm_startup_nrf52840.o(STACK)

    Global Symbols

    Symbol Name                              Value     Ov Type        Size  Object(Section)

    BuildAttributes$$THM_ISAv4$E$P$D$K$B$S$7EM$VFPi3$EXTD16$VFPS$VFMA$PE$A:L22UL41UL21$X:L11$S22US41US21$IEEE1$IW$USESV6$~STKCKD$USESV7$~SHL$OSPACE$EBA8$MICROLIB$REQ8$EABIv2 0x00000000   Number         0  anon$$obj.o ABSOLUTE
    __ARM_use_no_argv                        0x00000000   Number         0  main.o ABSOLUTE
    __Vectors                                0x00000000   Data           4  arm_startup_nrf52840.o(RESET)
    __use_no_errno                           0x00000000   Number         0  useno.o ABSOLUTE
    __use_no_exception_handling              0x00000000   Number         0  useno.o ABSOLUTE
    __use_no_fp                              0x00000000   Number         0  useno.o ABSOLUTE
    __use_no_heap                            0x00000000   Number         0  useno.o ABSOLUTE
    __use_no_heap_region                     0x00000000   Number         0  useno.o ABSOLUTE
    __use_no_semihosting                     0x00000000   Number         0  useno.o ABSOLUTE
    __use_no_semihosting_swi                 0x00000000   Number         0  useno.o ABSOLUTE
    __use_no_signal_handling                 0x00000000   Number         0  useno.o ABSOLUTE
    __cpp_initialize__aeabi_                  - Undefined Weak Reference
    __cxa_finalize                            - Undefined Weak Reference
    __decompress                              - Undefined Weak Reference
    _clock_init                               - Undefined Weak Reference
    _microlib_exit                            - Undefined Weak Reference
    log_dynamic_data$$Base                    - Undefined Reference
    __Vectors_End                            0x00000200   Data           0  arm_startup_nrf52840.o(RESET)
    __Vectors_Size                           0x00000200   Number         0  arm_startup_nrf52840.o ABSOLUTE
    __main                                   0x00000201   Thumb Code     0  entry.o(.ARM.Collect$$$$00000000)
    _main_stk                                0x00000201   Thumb Code     0  entry2.o(.ARM.Collect$$$$00000001)
    _main_scatterload                        0x00000205   Thumb Code     0  entry5.o(.ARM.Collect$$$$00000004)
    __main_after_scatterload                 0x00000209   Thumb Code     0  entry5.o(.ARM.Collect$$$$00000004)
    _main_clock                              0x00000209   Thumb Code     0  entry7b.o(.ARM.Collect$$$$00000008)
    _main_cpp_init                           0x00000209   Thumb Code     0  entry8b.o(.ARM.Collect$$$$0000000A)
    _main_init                               0x00000209   Thumb Code     0  entry9a.o(.ARM.Collect$$$$0000000B)
    __rt_final_cpp                           0x00000211   Thumb Code     0  entry10a.o(.ARM.Collect$$$$0000000D)
    __rt_final_exit                          0x00000211   Thumb Code     0  entry11a.o(.ARM.Collect$$$$0000000F)
    __asm___12_nrf_atfifo_c_51f461e1__nrf_atfifo_wspace_req 0x00000215   Thumb Code    56  nrf_atfifo.o(.emb_text)
    __asm___12_nrf_atfifo_c_51f461e1__nrf_atfifo_wspace_close 0x0000024d   Thumb Code    18  nrf_atfifo.o(.emb_text)
    __asm___12_nrf_atfifo_c_51f461e1__nrf_atfifo_rspace_req 0x0000025f   Thumb Code    58  nrf_atfifo.o(.emb_text)
    __asm___12_nrf_atfifo_c_51f461e1__nrf_atfifo_rspace_close 0x00000299   Thumb Code    18  nrf_atfifo.o(.emb_text)
    __asm___12_nrf_atfifo_c_51f461e1__nrf_atfifo_space_clear 0x000002ab   Thumb Code    50  nrf_atfifo.o(.emb_text)
    __asm___12_nrf_atomic_c_85ca2469__nrf_atomic_internal_mov 0x000002dd   Thumb Code    24  nrf_atomic.o(.emb_text)
    __asm___12_nrf_atomic_c_85ca2469__nrf_atomic_internal_orr 0x000002f5   Thumb Code    26  nrf_atomic.o(.emb_text)
    __asm___12_nrf_atomic_c_85ca2469__nrf_atomic_internal_and 0x0000030f   Thumb Code    26  nrf_atomic.o(.emb_text)
    __asm___12_nrf_atomic_c_85ca2469__nrf_atomic_internal_eor 0x00000329   Thumb Code    26  nrf_atomic.o(.emb_text)
    __asm___12_nrf_atomic_c_85ca2469__nrf_atomic_internal_add 0x00000343   Thumb Code    26  nrf_atomic.o(.emb_text)
    __asm___12_nrf_atomic_c_85ca2469__nrf_atomic_internal_sub 0x0000035d   Thumb Code    26  nrf_atomic.o(.emb_text)
    __asm___12_nrf_atomic_c_85ca2469__nrf_atomic_internal_cmp_exch 0x00000377   Thumb Code    42  nrf_atomic.o(.emb_text)
    __asm___12_nrf_atomic_c_85ca2469__nrf_atomic_internal_sub_hs 0x000003a1   Thumb Code    30  nrf_atomic.o(.emb_text)
    Reset_Handler                            0x000003c1   Thumb Code     8  arm_startup_nrf52840.o(.text)
    NMI_Handler                              0x000003c9   Thumb Code     2  arm_startup_nrf52840.o(.text)
    HardFault_Handler                        0x000003cb   Thumb Code     2  arm_startup_nrf52840.o(.text)
    MemoryManagement_Handler                 0x000003cd   Thumb Code     2  arm_startup_nrf52840.o(.text)
    BusFault_Handler                         0x000003cf   Thumb Code     2  arm_startup_nrf52840.o(.text)
    UsageFault_Handler                       0x000003d1   Thumb Code     2  arm_startup_nrf52840.o(.text)
    SVC_Handler                              0x000003d3   Thumb Code     2  arm_startup_nrf52840.o(.text)
    DebugMon_Handler                         0x000003d5   Thumb Code     2  arm_startup_nrf52840.o(.text)
    PendSV_Handler                           0x000003d7   Thumb Code     2  arm_startup_nrf52840.o(.text)
    SysTick_Handler                          0x000003d9   Thumb Code     2  arm_startup_nrf52840.o(.text)
    CCM_AAR_IRQHandler                       0x000003db   Thumb Code     0  arm_startup_nrf52840.o(.text)
    COMP_LPCOMP_IRQHandler                   0x000003db   Thumb Code     0  arm_startup_nrf52840.o(.text)
    CRYPTOCELL_IRQHandler                    0x000003db   Thumb Code     0  arm_startup_nrf52840.o(.text)
    ECB_IRQHandler                           0x000003db   Thumb Code     0  arm_startup_nrf52840.o(.text)
    FPU_IRQHandler                           0x000003db   Thumb Code     0  arm_startup_nrf52840.o(.text)
    GPIOTE_IRQHandler                        0x000003db   Thumb Code     0  arm_startup_nrf52840.o(.text)
    I2S_IRQHandler                           0x000003db   Thumb Code     0  arm_startup_nrf52840.o(.text)
    MWU_IRQHandler                           0x000003db   Thumb Code     0  arm_startup_nrf52840.o(.text)
    NFCT_IRQHandler                          0x000003db   Thumb Code     0  arm_startup_nrf52840.o(.text)
    PDM_IRQHandler                           0x000003db   Thumb Code     0  arm_startup_nrf52840.o(.text)
    PWM0_IRQHandler                          0x000003db   Thumb Code     0  arm_startup_nrf52840.o(.text)
    PWM1_IRQHandler                          0x000003db   Thumb Code     0  arm_startup_nrf52840.o(.text)
    PWM2_IRQHandler                          0x000003db   Thumb Code     0  arm_startup_nrf52840.o(.text)
    PWM3_IRQHandler                          0x000003db   Thumb Code     0  arm_startup_nrf52840.o(.text)
    QDEC_IRQHandler                          0x000003db   Thumb Code     0  arm_startup_nrf52840.o(.text)
    QSPI_IRQHandler                          0x000003db   Thumb Code     0  arm_startup_nrf52840.o(.text)
    RADIO_IRQHandler                         0x000003db   Thumb Code     0  arm_startup_nrf52840.o(.text)
    RNG_IRQHandler                           0x000003db   Thumb Code     0  arm_startup_nrf52840.o(.text)
    SAADC_IRQHandler                         0x000003db   Thumb Code     0  arm_startup_nrf52840.o(.text)
    SPIM0_SPIS0_TWIM0_TWIS0_SPI0_TWI0_IRQHandler 0x000003db   Thumb Code     0  arm_startup_nrf52840.o(.text)
    SPIM1_SPIS1_TWIM1_TWIS1_SPI1_TWI1_IRQHandler 0x000003db   Thumb Code     0  arm_startup_nrf52840.o(.text)
    SPIM2_SPIS2_SPI2_IRQHandler              0x000003db   Thumb Code     0  arm_startup_nrf52840.o(.text)
    SPIM3_IRQHandler                         0x000003db   Thumb Code     0  arm_startup_nrf52840.o(.text)
    SWI0_EGU0_IRQHandler                     0x000003db   Thumb Code     0  arm_startup_nrf52840.o(.text)
    SWI1_EGU1_IRQHandler                     0x000003db   Thumb Code     0  arm_startup_nrf52840.o(.text)
    SWI2_EGU2_IRQHandler                     0x000003db   Thumb Code     0  arm_startup_nrf52840.o(.text)
    SWI3_EGU3_IRQHandler                     0x000003db   Thumb Code     0  arm_startup_nrf52840.o(.text)
    SWI4_EGU4_IRQHandler                     0x000003db   Thumb Code     0  arm_startup_nrf52840.o(.text)
    SWI5_EGU5_IRQHandler                     0x000003db   Thumb Code     0  arm_startup_nrf52840.o(.text)
    TEMP_IRQHandler                          0x000003db   Thumb Code     0  arm_startup_nrf52840.o(.text)
    TIMER2_IRQHandler                        0x000003db   Thumb Code     0  arm_startup_nrf52840.o(.text)
    TIMER3_IRQHandler                        0x000003db   Thumb Code     0  arm_startup_nrf52840.o(.text)
    TIMER4_IRQHandler                        0x000003db   Thumb Code     0  arm_startup_nrf52840.o(.text)
    USBD_IRQHandler                          0x000003db   Thumb Code     0  arm_startup_nrf52840.o(.text)
    WDT_IRQHandler                           0x000003db   Thumb Code     0  arm_startup_nrf52840.o(.text)
    __aeabi_uldivmod                         0x000003e5   Thumb Code    98  uldiv.o(.text)
    __rt_ctype_table                         0x00000449   Thumb Code     4  ctype_o.o(.text)
    __aeabi_memcpy                           0x00000451   Thumb Code    36  memcpya.o(.text)
    __aeabi_memcpy4                          0x00000451   Thumb Code     0  memcpya.o(.text)
    __aeabi_memcpy8                          0x00000451   Thumb Code     0  memcpya.o(.text)
    __aeabi_memset                           0x00000475   Thumb Code    14  memseta.o(.text)
    __aeabi_memset4                          0x00000475   Thumb Code     0  memseta.o(.text)
    __aeabi_memset8                          0x00000475   Thumb Code     0  memseta.o(.text)
    __aeabi_memclr                           0x00000483   Thumb Code     4  memseta.o(.text)
    __aeabi_memclr4                          0x00000483   Thumb Code     0  memseta.o(.text)
    __aeabi_memclr8                          0x00000483   Thumb Code     0  memseta.o(.text)
    _memset$wrapper                          0x00000487   Thumb Code    18  memseta.o(.text)
    strlen                                   0x00000499   Thumb Code    14  strlen.o(.text)
    strcpy                                   0x000004a7   Thumb Code    18  strcpy.o(.text)
    __aeabi_llsl                             0x000004b9   Thumb Code    30  llshl.o(.text)
    _ll_shift_l                              0x000004b9   Thumb Code     0  llshl.o(.text)
    __aeabi_llsr                             0x000004d7   Thumb Code    32  llushr.o(.text)
    _ll_ushift_r                             0x000004d7   Thumb Code     0  llushr.o(.text)
    __scatterload                            0x000004f9   Thumb Code    28  init.o(.text)
    __scatterload_rt2                        0x000004f9   Thumb Code     0  init.o(.text)
    POWER_CLOCK_IRQHandler                   0x0000051d   Thumb Code    82  nrfx_clock.o(i.POWER_CLOCK_IRQHandler)
    RTC0_IRQHandler                          0x00000575   Thumb Code    10  nrfx_rtc.o(i.RTC0_IRQHandler)
    RTC1_IRQHandler                          0x00000585   Thumb Code    12  drv_rtc.o(i.RTC1_IRQHandler)
    RTC2_IRQHandler                          0x00000595   Thumb Code    10  nrfx_rtc.o(i.RTC2_IRQHandler)
    SEGGER_RTT_Init                          0x000005a5   Thumb Code     4  segger_rtt.o(i.SEGGER_RTT_Init)
    SEGGER_RTT_WriteNoLock                   0x000005a9   Thumb Code    86  segger_rtt.o(i.SEGGER_RTT_WriteNoLock)
    SystemInit                               0x00000605   Thumb Code   420  system_nrf52.o(i.SystemInit)
    TIMER0_IRQHandler                        0x000007e1   Thumb Code    10  nrfx_timer.o(i.TIMER0_IRQHandler)
    TIMER1_IRQHandler                        0x000007f5   Thumb Code    10  nrfx_timer.o(i.TIMER1_IRQHandler)
    UARTE0_UART0_IRQHandler                  0x00000809   Thumb Code     8  nrf_libuarte_drv.o(i.UARTE0_UART0_IRQHandler)
    UARTE1_IRQHandler                        0x00000815   Thumb Code     8  nrf_libuarte_drv.o(i.UARTE1_IRQHandler)
    __scatterload_copy                       0x0000093b   Thumb Code    14  handlers.o(i.__scatterload_copy)
    __scatterload_null                       0x00000949   Thumb Code     2  handlers.o(i.__scatterload_null)
    __scatterload_zeroinit                   0x0000094b   Thumb Code    14  handlers.o(i.__scatterload_zeroinit)
    app_error_fault_handler                  0x00000959   Thumb Code    86  app_error_weak.o(i.app_error_fault_handler)
    app_error_handler_bare                   0x000009dd   Thumb Code    22  app_error.o(i.app_error_handler_bare)
    app_timer_cnt_diff_compute               0x000009f3   Thumb Code     8  app_timer2.o(i.app_timer_cnt_diff_compute)
    app_timer_cnt_get                        0x000009fd   Thumb Code     6  app_timer2.o(i.app_timer_cnt_get)
    app_timer_create                         0x00000a09   Thumb Code    32  app_timer2.o(i.app_timer_create)
    app_timer_start                          0x00000ac1   Thumb Code    76  app_timer2.o(i.app_timer_start)
    app_util_critical_region_enter           0x00000b0d   Thumb Code     4  app_util_platform.o(i.app_util_critical_region_enter)
    app_util_critical_region_exit            0x00000b11   Thumb Code     4  app_util_platform.o(i.app_util_critical_region_exit)
    app_util_disable_irq                     0x00000b15   Thumb Code    12  app_util_platform.o(i.app_util_disable_irq)
    app_util_enable_irq                      0x00000b25   Thumb Code    14  app_util_platform.o(i.app_util_enable_irq)
    bsp_board_led_invert                     0x00000b39   Thumb Code    40  boards.o(i.bsp_board_led_invert)
    buffer_is_empty                          0x00000c21   Thumb Code    18  nrf_log_frontend.o(i.buffer_is_empty)
    drv_rtc_counter_get                      0x00000ca9   Thumb Code     8  drv_rtc.o(i.drv_rtc_counter_get)
    drv_rtc_irq_trigger                      0x00000cb1   Thumb Code    30  drv_rtc.o(i.drv_rtc_irq_trigger)
    log_pending_hook                         0x0000117d   Thumb Code     2  nrf_log_frontend.o(i.log_pending_hook)
    main                                     0x00001225   Thumb Code   154  main.o(i.main)
    nrf_atfifo_item_alloc                    0x00001381   Thumb Code    22  nrf_atfifo.o(i.nrf_atfifo_item_alloc)
    nrf_atfifo_item_put                      0x00001397   Thumb Code    22  nrf_atfifo.o(i.nrf_atfifo_item_put)
    nrf_atomic_flag_clear_fetch              0x000013ad   Thumb Code     6  nrf_atomic.o(i.nrf_atomic_flag_clear_fetch)
    nrf_atomic_flag_set                      0x000013b3   Thumb Code     6  nrf_atomic.o(i.nrf_atomic_flag_set)
    nrf_atomic_u32_add                       0x000013b9   Thumb Code    12  nrf_atomic.o(i.nrf_atomic_u32_add)
    nrf_atomic_u32_fetch_and                 0x000013c5   Thumb Code    10  nrf_atomic.o(i.nrf_atomic_u32_fetch_and)
    nrf_atomic_u32_fetch_store               0x000013cf   Thumb Code    10  nrf_atomic.o(i.nrf_atomic_u32_fetch_store)
    nrf_atomic_u32_or                        0x000013d9   Thumb Code    12  nrf_atomic.o(i.nrf_atomic_u32_or)
    nrf_atomic_u32_sub                       0x000013e5   Thumb Code    12  nrf_atomic.o(i.nrf_atomic_u32_sub)
    nrf_balloc_alloc                         0x000013f1   Thumb Code    62  nrf_balloc.o(i.nrf_balloc_alloc)
    nrf_balloc_free                          0x0000142f   Thumb Code    42  nrf_balloc.o(i.nrf_balloc_free)
    nrf_balloc_init                          0x00001459   Thumb Code    48  nrf_balloc.o(i.nrf_balloc_init)
    nrf_drv_clock_init                       0x000014a9   Thumb Code    50  nrf_drv_clock.o(i.nrf_drv_clock_init)
    nrf_drv_clock_lfclk_request              0x000014e5   Thumb Code    68  nrf_drv_clock.o(i.nrf_drv_clock_lfclk_request)
    nrf_fprintf                              0x0000152d   Thumb Code    26  nrf_fprintf.o(i.nrf_fprintf)
    nrf_fprintf_buffer_flush                 0x00001547   Thumb Code    24  nrf_fprintf.o(i.nrf_fprintf_buffer_flush)
    nrf_fprintf_fmt                          0x0000155f   Thumb Code   474  nrf_fprintf_format.o(i.nrf_fprintf_fmt)
    nrf_libuarte_async_enable                0x000017b9   Thumb Code   154  nrf_libuarte_async.o(i.nrf_libuarte_async_enable)
    nrf_libuarte_async_init                  0x00001859   Thumb Code   510  nrf_libuarte_async.o(i.nrf_libuarte_async_init)
    nrf_libuarte_async_rx_free               0x00001a69   Thumb Code    92  nrf_libuarte_async.o(i.nrf_libuarte_async_rx_free)
    nrf_libuarte_async_timeout_handler       0x00001ac5   Thumb Code   138  nrf_libuarte_async.o(i.nrf_libuarte_async_timeout_handler)
    nrf_libuarte_async_tx                    0x00001b4f   Thumb Code     6  nrf_libuarte_async.o(i.nrf_libuarte_async_tx)
    nrf_libuarte_drv_init                    0x00001b55   Thumb Code   380  nrf_libuarte_drv.o(i.nrf_libuarte_drv_init)
    nrf_libuarte_drv_rx_buf_rsp              0x00001ce5   Thumb Code    26  nrf_libuarte_drv.o(i.nrf_libuarte_drv_rx_buf_rsp)
    nrf_libuarte_drv_rx_start                0x00001cff   Thumb Code   110  nrf_libuarte_drv.o(i.nrf_libuarte_drv_rx_start)
    nrf_libuarte_drv_tx                      0x00001d6d   Thumb Code   174  nrf_libuarte_drv.o(i.nrf_libuarte_drv_tx)
    nrf_log_backend_add                      0x00001e1d   Thumb Code    86  nrf_log_frontend.o(i.nrf_log_backend_add)
    nrf_log_backend_rtt_init                 0x00001e7b   Thumb Code     4  nrf_log_backend_rtt.o(i.nrf_log_backend_rtt_init)
    nrf_log_backend_serial_put               0x00001e99   Thumb Code   200  nrf_log_backend_serial.o(i.nrf_log_backend_serial_put)
    nrf_log_color_id_get                     0x00001f61   Thumb Code    42  nrf_log_frontend.o(i.nrf_log_color_id_get)
    nrf_log_default_backends_init            0x00001f91   Thumb Code    24  nrf_log_default_backends.o(i.nrf_log_default_backends_init)
    nrf_log_frontend_dequeue                 0x00001fad   Thumb Code   522  nrf_log_frontend.o(i.nrf_log_frontend_dequeue)
    nrf_log_frontend_std_0                   0x000021e1   Thumb Code     8  nrf_log_frontend.o(i.nrf_log_frontend_std_0)
    nrf_log_frontend_std_1                   0x000021e9   Thumb Code    14  nrf_log_frontend.o(i.nrf_log_frontend_std_1)
    nrf_log_frontend_std_2                   0x000021f7   Thumb Code    16  nrf_log_frontend.o(i.nrf_log_frontend_std_2)
    nrf_log_frontend_std_3                   0x00002207   Thumb Code    18  nrf_log_frontend.o(i.nrf_log_frontend_std_3)
    nrf_log_hexdump_entry_process            0x00002219   Thumb Code   150  nrf_log_str_formatter.o(i.nrf_log_hexdump_entry_process)
    nrf_log_init                             0x000022c9   Thumb Code    28  nrf_log_frontend.o(i.nrf_log_init)
    nrf_log_module_cnt_get                   0x000022f1   Thumb Code    10  nrf_log_frontend.o(i.nrf_log_module_cnt_get)
    nrf_log_module_name_get                  0x00002305   Thumb Code    24  nrf_log_frontend.o(i.nrf_log_module_name_get)
    nrf_log_panic                            0x00002321   Thumb Code    36  nrf_log_frontend.o(i.nrf_log_panic)
    nrf_log_std_entry_process                0x00002349   Thumb Code   182  nrf_log_str_formatter.o(i.nrf_log_std_entry_process)
    nrf_memobj_alloc                         0x000023ff   Thumb Code    96  nrf_memobj.o(i.nrf_memobj_alloc)
    nrf_memobj_free                          0x0000245f   Thumb Code    50  nrf_memobj.o(i.nrf_memobj_free)
    nrf_memobj_get                           0x00002491   Thumb Code     8  nrf_memobj.o(i.nrf_memobj_get)
    nrf_memobj_pool_init                     0x00002499   Thumb Code     4  nrf_memobj.o(i.nrf_memobj_pool_init)
    nrf_memobj_put                           0x0000249d   Thumb Code    30  nrf_memobj.o(i.nrf_memobj_put)
    nrf_memobj_read                          0x000024bb   Thumb Code    16  nrf_memobj.o(i.nrf_memobj_read)
    nrf_memobj_write                         0x000024cb   Thumb Code    16  nrf_memobj.o(i.nrf_memobj_write)
    nrf_queue_generic_pop                    0x000024db   Thumb Code   136  nrf_queue.o(i.nrf_queue_generic_pop)
    nrf_queue_is_empty                       0x00002563   Thumb Code    18  nrf_queue.o(i.nrf_queue_is_empty)
    nrf_queue_is_full                        0x00002575   Thumb Code    30  nrf_queue.o(i.nrf_queue_is_full)
    nrf_queue_push                           0x000025a1   Thumb Code   172  nrf_queue.o(i.nrf_queue_push)
    nrf_queue_reset                          0x0000264d   Thumb Code    30  nrf_queue.o(i.nrf_queue_reset)
    nrf_ringbuf_init                         0x0000266b   Thumb Code    28  nrf_ringbuf.o(i.nrf_ringbuf_init)
    nrf_strerror_find                        0x00002695   Thumb Code    52  nrf_strerror.o(i.nrf_strerror_find)
    nrf_strerror_get                         0x000026cd   Thumb Code    14  nrf_strerror.o(i.nrf_strerror_get)
    nrfx_clock_enable                        0x00002715   Thumb Code    34  nrfx_clock.o(i.nrfx_clock_enable)
    nrfx_clock_init                          0x00002741   Thumb Code    26  nrfx_clock.o(i.nrfx_clock_init)
    nrfx_clock_lfclk_start                   0x00002761   Thumb Code    26  nrfx_clock.o(i.nrfx_clock_lfclk_start)
    nrfx_ppi_channel_alloc                   0x00002781   Thumb Code   134  nrfx_ppi.o(i.nrfx_ppi_channel_alloc)
    nrfx_ppi_channel_assign                  0x00002855   Thumb Code   120  nrfx_ppi.o(i.nrfx_ppi_channel_assign)
    nrfx_ppi_channel_disable                 0x0000293d   Thumb Code    66  nrfx_ppi.o(i.nrfx_ppi_channel_disable)
    nrfx_ppi_channel_enable                  0x000029b1   Thumb Code    66  nrfx_ppi.o(i.nrfx_ppi_channel_enable)
    nrfx_ppi_channel_fork_assign             0x00002a25   Thumb Code    88  nrfx_ppi.o(i.nrfx_ppi_channel_fork_assign)
    nrfx_ppi_channel_free                    0x00002add   Thumb Code    78  nrfx_ppi.o(i.nrfx_ppi_channel_free)
    nrfx_ppi_channels_include_in_group       0x00002b61   Thumb Code    94  nrfx_ppi.o(i.nrfx_ppi_channels_include_in_group)
    nrfx_ppi_group_alloc                     0x00002bf1   Thumb Code   134  nrfx_ppi.o(i.nrfx_ppi_group_alloc)
    nrfx_ppi_group_enable                    0x00002cc1   Thumb Code    70  nrfx_ppi.o(i.nrfx_ppi_group_enable)
    nrfx_ppi_group_free                      0x00002d39   Thumb Code    92  nrfx_ppi.o(i.nrfx_ppi_group_free)
    nrfx_rtc_cc_set                          0x00002dc9   Thumb Code   128  nrfx_rtc.o(i.nrfx_rtc_cc_set)
    nrfx_rtc_init                            0x00002e4d   Thumb Code   138  nrfx_rtc.o(i.nrfx_rtc_init)
    nrfx_timer_clear                         0x00002edd   Thumb Code     8  nrfx_timer.o(i.nrfx_timer_clear)
    nrfx_timer_compare                       0x00002ee5   Thumb Code    58  nrfx_timer.o(i.nrfx_timer_compare)
    nrfx_timer_enable                        0x00002f21   Thumb Code    24  nrfx_timer.o(i.nrfx_timer_enable)
    nrfx_timer_init                          0x00002f3d   Thumb Code   188  nrfx_timer.o(i.nrfx_timer_init)
    nvmc_config                              0x00002ffd   Thumb Code    14  system_nrf52.o(i.nvmc_config)
    tmr_evt_handler                          0x0000345f   Thumb Code     2  nrf_libuarte_drv.o(i.tmr_evt_handler)
    uart_event_handler                       0x00003471   Thumb Code   130  main.o(i.uart_event_handler)
    nrf_log_backend_rtt_api                  0x00003a34   Data          12  nrf_log_backend_rtt.o(.constdata)
    __ctype_table                            0x00003a54   Data         129  ctype_o.o(.constdata)
    Region$$Table$$Base                      0x00003f6c   Number         0  anon$$obj.o(Region$$Table)
    Region$$Table$$Limit                     0x00003f8c   Number         0  anon$$obj.o(Region$$Table)
    log_const_data$$Base                     0x00003f9c   Number         0  nrf_drv_clock.o(log_const_data)
    m_nrf_log_clock_logs_data_const          0x00003f9c   Data           8  nrf_drv_clock.o(log_const_data)
    m_nrf_log_CLOCK_logs_data_const          0x00003fa4   Data           8  nrfx_clock.o(log_const_data)
    m_nrf_log_PPI_logs_data_const            0x00003fac   Data           8  nrfx_ppi.o(log_const_data)
    m_nrf_log_RTC_logs_data_const            0x00003fb4   Data           8  nrfx_rtc.o(log_const_data)
    m_nrf_log_TIMER_logs_data_const          0x00003fbc   Data           8  nrfx_timer.o(log_const_data)
    m_nrf_log_app_timer_logs_data_const      0x00003fc4   Data           8  app_timer2.o(log_const_data)
    m_nrf_log_libUARTE_async_logs_data_const 0x00003fcc   Data           8  nrf_libuarte_async.o(log_const_data)
    m_nrf_log_libUARTE_logs_data_const       0x00003fd4   Data           8  nrf_libuarte_drv.o(log_const_data)
    m_nrf_log_sortlist_logs_data_const       0x00003fdc   Data           8  nrf_sortlist.o(log_const_data)
    m_nrf_log_app_logs_data_const            0x00003fe4   Data           8  nrf_log_frontend.o(log_const_data)
    libuarte_rx_pool                         0x00003fec   Data          20  main.o(nrf_balloc)
    log_const_data$$Limit                    0x00003fec   Number         0  nrf_log_frontend.o(log_const_data)
    libuarte1_rx_pool                        0x00004000   Data          20  main.o(nrf_balloc)
    log_mempool                              0x00004014   Data          20  nrf_log_frontend.o(nrf_balloc)
    libuarte_rxdata_queue                    0x00004028   Data          20  main.o(nrf_queue)
    libuarte1_rxdata_queue                   0x0000403c   Data          20  main.o(nrf_queue)
    m_buf_queue                              0x00004050   Data          20  main.o(nrf_queue)
    SystemCoreClock                          0x200000fc   Data           4  system_nrf52.o(.data)
    _SEGGER_RTT                              0x20000e60   Data         120  segger_rtt.o(.bss)
    __initial_sp                             0x200030e8   Data           0  arm_startup_nrf52840.o(STACK)



==============================================================================

Memory Map of the image

  Image Entry point : 0x00000201

  Load Region LR_IROM1 (Base: 0x00000000, Size: 0x00004164, Max: 0x00100000, ABSOLUTE)

    Execution Region ER_IROM1 (Exec base: 0x00000000, Load base: 0x00000000, Size: 0x00004064, Max: 0x00100000, ABSOLUTE)

    Exec Addr    Load Addr    Size         Type   Attr      Idx    E Section Name        Object

    0x00000000   0x00000000   0x00000200   Data   RO         3623    RESET               arm_startup_nrf52840.o
    0x00000200   0x00000200   0x00000000   Code   RO         3695  * .ARM.Collect$$$$00000000  mc_w.l(entry.o)
    0x00000200   0x00000200   0x00000004   Code   RO         3745    .ARM.Collect$$$$00000001  mc_w.l(entry2.o)
    0x00000204   0x00000204   0x00000004   Code   RO         3748    .ARM.Collect$$$$00000004  mc_w.l(entry5.o)
    0x00000208   0x00000208   0x00000000   Code   RO         3750    .ARM.Collect$$$$00000008  mc_w.l(entry7b.o)
    0x00000208   0x00000208   0x00000000   Code   RO         3752    .ARM.Collect$$$$0000000A  mc_w.l(entry8b.o)
    0x00000208   0x00000208   0x00000008   Code   RO         3753    .ARM.Collect$$$$0000000B  mc_w.l(entry9a.o)
    0x00000210   0x00000210   0x00000000   Code   RO         3755    .ARM.Collect$$$$0000000D  mc_w.l(entry10a.o)
    0x00000210   0x00000210   0x00000000   Code   RO         3757    .ARM.Collect$$$$0000000F  mc_w.l(entry11a.o)
    0x00000210   0x00000210   0x00000004   Code   RO         3746    .ARM.Collect$$$$00002712  mc_w.l(entry2.o)
    0x00000214   0x00000214   0x000000c8   Code   RO         1887    .emb_text           nrf_atfifo.o
    0x000002dc   0x000002dc   0x000000e2   Code   RO         1957    .emb_text           nrf_atomic.o
    0x000003be   0x000003be   0x00000002   PAD
    0x000003c0   0x000003c0   0x00000024   Code   RO         3624    .text               arm_startup_nrf52840.o
    0x000003e4   0x000003e4   0x00000062   Code   RO         3703    .text               mc_w.l(uldiv.o)
    0x00000446   0x00000446   0x00000002   PAD
    0x00000448   0x00000448   0x00000008   Code   RO         3705    .text               mc_w.l(ctype_o.o)
    0x00000450   0x00000450   0x00000024   Code   RO         3733    .text               mc_w.l(memcpya.o)
    0x00000474   0x00000474   0x00000024   Code   RO         3735    .text               mc_w.l(memseta.o)
    0x00000498   0x00000498   0x0000000e   Code   RO         3737    .text               mc_w.l(strlen.o)
    0x000004a6   0x000004a6   0x00000012   Code   RO         3741    .text               mc_w.l(strcpy.o)
    0x000004b8   0x000004b8   0x0000001e   Code   RO         3760    .text               mc_w.l(llshl.o)
    0x000004d6   0x000004d6   0x00000020   Code   RO         3762    .text               mc_w.l(llushr.o)
    0x000004f6   0x000004f6   0x00000002   PAD
    0x000004f8   0x000004f8   0x00000024   Code   RO         3765    .text               mc_w.l(init.o)
    0x0000051c   0x0000051c   0x00000058   Code   RO          794    i.POWER_CLOCK_IRQHandler  nrfx_clock.o
    0x00000574   0x00000574   0x00000010   Code   RO         1068    i.RTC0_IRQHandler   nrfx_rtc.o
    0x00000584   0x00000584   0x00000010   Code   RO         1691    i.RTC1_IRQHandler   drv_rtc.o
    0x00000594   0x00000594   0x00000010   Code   RO         1069    i.RTC2_IRQHandler   nrfx_rtc.o
    0x000005a4   0x000005a4   0x00000004   Code   RO         3277    i.SEGGER_RTT_Init   segger_rtt.o
    0x000005a8   0x000005a8   0x0000005c   Code   RO         3291    i.SEGGER_RTT_WriteNoLock  segger_rtt.o
    0x00000604   0x00000604   0x000001dc   Code   RO         3632    i.SystemInit        system_nrf52.o
    0x000007e0   0x000007e0   0x00000014   Code   RO         1195    i.TIMER0_IRQHandler  nrfx_timer.o
    0x000007f4   0x000007f4   0x00000014   Code   RO         1196    i.TIMER1_IRQHandler  nrfx_timer.o
    0x00000808   0x00000808   0x0000000c   Code   RO         2342    i.UARTE0_UART0_IRQHandler  nrf_libuarte_drv.o
    0x00000814   0x00000814   0x0000000c   Code   RO         2343    i.UARTE1_IRQHandler  nrf_libuarte_drv.o
    0x00000820   0x00000820   0x00000068   Code   RO         3295    i._DoInit           segger_rtt.o
    0x00000888   0x00000888   0x00000016   Code   RO         3296    i._GetAvailWriteSpace  segger_rtt.o
    0x0000089e   0x0000089e   0x0000005a   Code   RO         3298    i._WriteBlocking    segger_rtt.o
    0x000008f8   0x000008f8   0x00000042   Code   RO         3299    i._WriteNoCheck     segger_rtt.o
    0x0000093a   0x0000093a   0x0000000e   Code   RO         3769    i.__scatterload_copy  mc_w.l(handlers.o)
    0x00000948   0x00000948   0x00000002   Code   RO         3770    i.__scatterload_null  mc_w.l(handlers.o)
    0x0000094a   0x0000094a   0x0000000e   Code   RO         3771    i.__scatterload_zeroinit  mc_w.l(handlers.o)
    0x00000958   0x00000958   0x00000084   Code   RO         1401    i.app_error_fault_handler  app_error_weak.o
    0x000009dc   0x000009dc   0x00000016   Code   RO         1335    i.app_error_handler_bare  app_error.o
    0x000009f2   0x000009f2   0x00000008   Code   RO         1490    i.app_timer_cnt_diff_compute  app_timer2.o
    0x000009fa   0x000009fa   0x00000002   PAD
    0x000009fc   0x000009fc   0x0000000c   Code   RO         1491    i.app_timer_cnt_get  app_timer2.o
    0x00000a08   0x00000a08   0x00000020   Code   RO         1492    i.app_timer_create  app_timer2.o
    0x00000a28   0x00000a28   0x00000098   Code   RO         2212    i.app_timer_handler  nrf_libuarte_async.o
    0x00000ac0   0x00000ac0   0x0000004c   Code   RO         1496    i.app_timer_start   app_timer2.o
    0x00000b0c   0x00000b0c   0x00000004   Code   RO         1629    i.app_util_critical_region_enter  app_util_platform.o
    0x00000b10   0x00000b10   0x00000004   Code   RO         1630    i.app_util_critical_region_exit  app_util_platform.o
    0x00000b14   0x00000b14   0x00000010   Code   RO         1631    i.app_util_disable_irq  app_util_platform.o
    0x00000b24   0x00000b24   0x00000014   Code   RO         1632    i.app_util_enable_irq  app_util_platform.o
    0x00000b38   0x00000b38   0x0000002c   Code   RO          301    i.bsp_board_led_invert  boards.o
    0x00000b64   0x00000b64   0x0000008c   Code   RO         3025    i.buf_prealloc      nrf_log_frontend.o
    0x00000bf0   0x00000bf0   0x0000002e   Code   RO         2172    i.buffer_add        nrf_fprintf_format.o
    0x00000c1e   0x00000c1e   0x00000002   PAD
    0x00000c20   0x00000c20   0x00000018   Code   RO         3026    i.buffer_is_empty   nrf_log_frontend.o
    0x00000c38   0x00000c38   0x00000028   Code   RO          397    i.clock_clk_started_notify  nrf_drv_clock.o
    0x00000c60   0x00000c60   0x0000001c   Code   RO          398    i.clock_irq_handler  nrf_drv_clock.o
    0x00000c7c   0x00000c7c   0x00000018   Code   RO         1499    i.compare_func      app_timer2.o
    0x00000c94   0x00000c94   0x00000014   Code   RO         3027    i.dropped_sat16_get  nrf_log_frontend.o
    0x00000ca8   0x00000ca8   0x00000008   Code   RO         1697    i.drv_rtc_counter_get  drv_rtc.o
    0x00000cb0   0x00000cb0   0x0000001e   Code   RO         1699    i.drv_rtc_irq_trigger  drv_rtc.o
    0x00000cce   0x00000cce   0x00000002   PAD
    0x00000cd0   0x00000cd0   0x00000034   Code   RO         1500    i.get_now           app_timer2.o
    0x00000d04   0x00000d04   0x000000a6   Code   RO         2173    i.int_print         nrf_fprintf_format.o
    0x00000daa   0x00000daa   0x00000034   Code   RO         3028    i.invalid_packets_omit  nrf_log_frontend.o
    0x00000dde   0x00000dde   0x00000002   PAD
    0x00000de0   0x00000de0   0x000000a0   Code   RO         1070    i.irq_handler       nrfx_rtc.o
    0x00000e80   0x00000e80   0x00000046   Code   RO         1197    i.irq_handler       nrfx_timer.o
    0x00000ec6   0x00000ec6   0x00000002   PAD
    0x00000ec8   0x00000ec8   0x00000204   Code   RO         2344    i.irq_handler       nrf_libuarte_drv.o
    0x000010cc   0x000010cc   0x00000018   Code   RO          933    i.is_allocated_channel  nrfx_ppi.o
    0x000010e4   0x000010e4   0x00000018   Code   RO          934    i.is_allocated_group  nrfx_ppi.o
    0x000010fc   0x000010fc   0x0000000c   Code   RO          935    i.is_app_group      nrfx_ppi.o
    0x00001108   0x00001108   0x0000000c   Code   RO          936    i.is_programmable_app_channel  nrfx_ppi.o
    0x00001114   0x00001114   0x00000016   Code   RO          399    i.item_enqueue      nrf_drv_clock.o
    0x0000112a   0x0000112a   0x00000002   PAD
    0x0000112c   0x0000112c   0x00000028   Code   RO            4    i.libuarte1_rtc_handler  main.o
    0x00001154   0x00001154   0x00000028   Code   RO            5    i.libuarte_rtc_handler  main.o
    0x0000117c   0x0000117c   0x00000002   Code   RO         3029    i.log_pending_hook  nrf_log_frontend.o
    0x0000117e   0x0000117e   0x00000002   PAD
    0x00001180   0x00001180   0x000000a4   Code   RO         3030    i.log_skip          nrf_log_frontend.o
    0x00001224   0x00001224   0x000000ac   Code   RO            6    i.main              main.o
    0x000012d0   0x000012d0   0x0000007e   Code   RO         2538    i.memobj_op         nrf_memobj.o
    0x0000134e   0x0000134e   0x00000002   PAD
    0x00001350   0x00001350   0x00000030   Code   RO         3031    i.module_idx_get    nrf_log_frontend.o
    0x00001380   0x00001380   0x00000016   Code   RO         1892    i.nrf_atfifo_item_alloc  nrf_atfifo.o
    0x00001396   0x00001396   0x00000016   Code   RO         1895    i.nrf_atfifo_item_put  nrf_atfifo.o
    0x000013ac   0x000013ac   0x00000006   Code   RO         1959    i.nrf_atomic_flag_clear_fetch  nrf_atomic.o
    0x000013b2   0x000013b2   0x00000006   Code   RO         1960    i.nrf_atomic_flag_set  nrf_atomic.o
    0x000013b8   0x000013b8   0x0000000c   Code   RO         1962    i.nrf_atomic_u32_add  nrf_atomic.o
    0x000013c4   0x000013c4   0x0000000a   Code   RO         1966    i.nrf_atomic_u32_fetch_and  nrf_atomic.o
    0x000013ce   0x000013ce   0x0000000a   Code   RO         1968    i.nrf_atomic_u32_fetch_store  nrf_atomic.o
    0x000013d8   0x000013d8   0x0000000c   Code   RO         1972    i.nrf_atomic_u32_or  nrf_atomic.o
    0x000013e4   0x000013e4   0x0000000c   Code   RO         1974    i.nrf_atomic_u32_sub  nrf_atomic.o
    0x000013f0   0x000013f0   0x0000003e   Code   RO         2096    i.nrf_balloc_alloc  nrf_balloc.o
    0x0000142e   0x0000142e   0x0000002a   Code   RO         2097    i.nrf_balloc_free   nrf_balloc.o
    0x00001458   0x00001458   0x00000030   Code   RO         2098    i.nrf_balloc_init   nrf_balloc.o
    0x00001488   0x00001488   0x0000000e   Code   RO          795    i.nrf_clock_event_check  nrfx_clock.o
    0x00001496   0x00001496   0x00000010   Code   RO          796    i.nrf_clock_event_clear  nrfx_clock.o
    0x000014a6   0x000014a6   0x00000002   PAD
    0x000014a8   0x000014a8   0x0000003c   Code   RO          405    i.nrf_drv_clock_init  nrf_drv_clock.o
    0x000014e4   0x000014e4   0x00000048   Code   RO          410    i.nrf_drv_clock_lfclk_request  nrf_drv_clock.o
    0x0000152c   0x0000152c   0x0000001a   Code   RO         2133    i.nrf_fprintf       nrf_fprintf.o
    0x00001546   0x00001546   0x00000018   Code   RO         2134    i.nrf_fprintf_buffer_flush  nrf_fprintf.o
    0x0000155e   0x0000155e   0x000001da   Code   RO         2174    i.nrf_fprintf_fmt   nrf_fprintf_format.o
    0x00001738   0x00001738   0x00000032   Code   RO         2345    i.nrf_gpio_cfg      nrf_libuarte_drv.o
    0x0000176a   0x0000176a   0x00000014   Code   RO         2346    i.nrf_gpio_cfg_output  nrf_libuarte_drv.o
    0x0000177e   0x0000177e   0x00000002   PAD
    0x00001780   0x00001780   0x0000001c   Code   RO          308    i.nrf_gpio_pin_port_decode  boards.o
    0x0000179c   0x0000179c   0x0000001c   Code   RO         2347    i.nrf_gpio_pin_port_decode  nrf_libuarte_drv.o
    0x000017b8   0x000017b8   0x000000a0   Code   RO         2213    i.nrf_libuarte_async_enable  nrf_libuarte_async.o
    0x00001858   0x00001858   0x00000210   Code   RO         2214    i.nrf_libuarte_async_init  nrf_libuarte_async.o
    0x00001a68   0x00001a68   0x0000005c   Code   RO         2217    i.nrf_libuarte_async_rx_free  nrf_libuarte_async.o
    0x00001ac4   0x00001ac4   0x0000008a   Code   RO         2218    i.nrf_libuarte_async_timeout_handler  nrf_libuarte_async.o
    0x00001b4e   0x00001b4e   0x00000006   Code   RO         2219    i.nrf_libuarte_async_tx  nrf_libuarte_async.o
    0x00001b54   0x00001b54   0x00000190   Code   RO         2348    i.nrf_libuarte_drv_init  nrf_libuarte_drv.o
    0x00001ce4   0x00001ce4   0x0000001a   Code   RO         2351    i.nrf_libuarte_drv_rx_buf_rsp  nrf_libuarte_drv.o
    0x00001cfe   0x00001cfe   0x0000006e   Code   RO         2352    i.nrf_libuarte_drv_rx_start  nrf_libuarte_drv.o
    0x00001d6c   0x00001d6c   0x000000ae   Code   RO         2354    i.nrf_libuarte_drv_tx  nrf_libuarte_drv.o
    0x00001e1a   0x00001e1a   0x00000002   PAD
    0x00001e1c   0x00001e1c   0x0000005c   Code   RO         3032    i.nrf_log_backend_add  nrf_log_frontend.o
    0x00001e78   0x00001e78   0x00000002   Code   RO         2886    i.nrf_log_backend_rtt_flush  nrf_log_backend_rtt.o
    0x00001e7a   0x00001e7a   0x00000004   Code   RO         2887    i.nrf_log_backend_rtt_init  nrf_log_backend_rtt.o
    0x00001e7e   0x00001e7e   0x00000002   Code   RO         2888    i.nrf_log_backend_rtt_panic_set  nrf_log_backend_rtt.o
    0x00001e80   0x00001e80   0x00000018   Code   RO         2889    i.nrf_log_backend_rtt_put  nrf_log_backend_rtt.o
    0x00001e98   0x00001e98   0x000000c8   Code   RO         2955    i.nrf_log_backend_serial_put  nrf_log_backend_serial.o
    0x00001f60   0x00001f60   0x00000030   Code   RO         3034    i.nrf_log_color_id_get  nrf_log_frontend.o
    0x00001f90   0x00001f90   0x0000001c   Code   RO         2989    i.nrf_log_default_backends_init  nrf_log_default_backends.o
    0x00001fac   0x00001fac   0x00000234   Code   RO         3035    i.nrf_log_frontend_dequeue  nrf_log_frontend.o
    0x000021e0   0x000021e0   0x00000008   Code   RO         3037    i.nrf_log_frontend_std_0  nrf_log_frontend.o
    0x000021e8   0x000021e8   0x0000000e   Code   RO         3038    i.nrf_log_frontend_std_1  nrf_log_frontend.o
    0x000021f6   0x000021f6   0x00000010   Code   RO         3039    i.nrf_log_frontend_std_2  nrf_log_frontend.o
    0x00002206   0x00002206   0x00000012   Code   RO         3040    i.nrf_log_frontend_std_3  nrf_log_frontend.o
    0x00002218   0x00002218   0x000000b0   Code   RO         3218    i.nrf_log_hexdump_entry_process  nrf_log_str_formatter.o
    0x000022c8   0x000022c8   0x00000028   Code   RO         3044    i.nrf_log_init      nrf_log_frontend.o
    0x000022f0   0x000022f0   0x00000014   Code   RO         3045    i.nrf_log_module_cnt_get  nrf_log_frontend.o
    0x00002304   0x00002304   0x0000001c   Code   RO         3048    i.nrf_log_module_name_get  nrf_log_frontend.o
    0x00002320   0x00002320   0x00000028   Code   RO         3049    i.nrf_log_panic     nrf_log_frontend.o
    0x00002348   0x00002348   0x000000b6   Code   RO         3219    i.nrf_log_std_entry_process  nrf_log_str_formatter.o
    0x000023fe   0x000023fe   0x00000060   Code   RO         2539    i.nrf_memobj_alloc  nrf_memobj.o
    0x0000245e   0x0000245e   0x00000032   Code   RO         2540    i.nrf_memobj_free   nrf_memobj.o
    0x00002490   0x00002490   0x00000008   Code   RO         2541    i.nrf_memobj_get    nrf_memobj.o
    0x00002498   0x00002498   0x00000004   Code   RO         2542    i.nrf_memobj_pool_init  nrf_memobj.o
    0x0000249c   0x0000249c   0x0000001e   Code   RO         2543    i.nrf_memobj_put    nrf_memobj.o
    0x000024ba   0x000024ba   0x00000010   Code   RO         2544    i.nrf_memobj_read   nrf_memobj.o
    0x000024ca   0x000024ca   0x00000010   Code   RO         2545    i.nrf_memobj_write  nrf_memobj.o
    0x000024da   0x000024da   0x00000088   Code   RO         2615    i.nrf_queue_generic_pop  nrf_queue.o
    0x00002562   0x00002562   0x00000012   Code   RO         2617    i.nrf_queue_is_empty  nrf_queue.o
    0x00002574   0x00002574   0x0000001e   Code   RO         2618    i.nrf_queue_is_full  nrf_queue.o
    0x00002592   0x00002592   0x0000000e   Code   RO         2621    i.nrf_queue_next_idx  nrf_queue.o
    0x000025a0   0x000025a0   0x000000ac   Code   RO         2623    i.nrf_queue_push    nrf_queue.o
    0x0000264c   0x0000264c   0x0000001e   Code   RO         2625    i.nrf_queue_reset   nrf_queue.o
    0x0000266a   0x0000266a   0x0000001c   Code   RO         2739    i.nrf_ringbuf_init  nrf_ringbuf.o
    0x00002686   0x00002686   0x0000000c   Code   RO         1071    i.nrf_rtc_event_clear  nrfx_rtc.o
    0x00002692   0x00002692   0x00000002   PAD
    0x00002694   0x00002694   0x00000038   Code   RO         2853    i.nrf_strerror_find  nrf_strerror.o
    0x000026cc   0x000026cc   0x00000014   Code   RO         2854    i.nrf_strerror_get  nrf_strerror.o
    0x000026e0   0x000026e0   0x0000000c   Code   RO         1198    i.nrf_timer_event_clear  nrfx_timer.o
    0x000026ec   0x000026ec   0x0000000a   Code   RO         2356    i.nrf_uarte_event_check  nrf_libuarte_drv.o
    0x000026f6   0x000026f6   0x0000000c   Code   RO         2357    i.nrf_uarte_event_clear  nrf_libuarte_drv.o
    0x00002702   0x00002702   0x00000002   PAD
    0x00002704   0x00002704   0x00000010   Code   RO          412    i.nrf_wdt_started   nrf_drv_clock.o
    0x00002714   0x00002714   0x0000002c   Code   RO          801    i.nrfx_clock_enable  nrfx_clock.o
    0x00002740   0x00002740   0x00000020   Code   RO          804    i.nrfx_clock_init   nrfx_clock.o
    0x00002760   0x00002760   0x00000020   Code   RO          806    i.nrfx_clock_lfclk_start  nrfx_clock.o
    0x00002780   0x00002780   0x000000d4   Code   RO          937    i.nrfx_ppi_channel_alloc  nrfx_ppi.o
    0x00002854   0x00002854   0x000000e8   Code   RO          938    i.nrfx_ppi_channel_assign  nrfx_ppi.o
    0x0000293c   0x0000293c   0x00000074   Code   RO          939    i.nrfx_ppi_channel_disable  nrfx_ppi.o
    0x000029b0   0x000029b0   0x00000074   Code   RO          940    i.nrfx_ppi_channel_enable  nrfx_ppi.o
    0x00002a24   0x00002a24   0x000000b8   Code   RO          941    i.nrfx_ppi_channel_fork_assign  nrfx_ppi.o
    0x00002adc   0x00002adc   0x00000084   Code   RO          942    i.nrfx_ppi_channel_free  nrfx_ppi.o
    0x00002b60   0x00002b60   0x00000090   Code   RO          943    i.nrfx_ppi_channels_include_in_group  nrfx_ppi.o
    0x00002bf0   0x00002bf0   0x000000d0   Code   RO          946    i.nrfx_ppi_group_alloc  nrfx_ppi.o
    0x00002cc0   0x00002cc0   0x00000078   Code   RO          948    i.nrfx_ppi_group_enable  nrfx_ppi.o
    0x00002d38   0x00002d38   0x00000090   Code   RO          949    i.nrfx_ppi_group_free  nrfx_ppi.o
    0x00002dc8   0x00002dc8   0x00000084   Code   RO         1073    i.nrfx_rtc_cc_set   nrfx_rtc.o
    0x00002e4c   0x00002e4c   0x00000090   Code   RO         1076    i.nrfx_rtc_init     nrfx_rtc.o
    0x00002edc   0x00002edc   0x00000008   Code   RO         1200    i.nrfx_timer_clear  nrfx_timer.o
    0x00002ee4   0x00002ee4   0x0000003a   Code   RO         1201    i.nrfx_timer_compare  nrfx_timer.o
    0x00002f1e   0x00002f1e   0x00000002   PAD
    0x00002f20   0x00002f20   0x0000001c   Code   RO         1205    i.nrfx_timer_enable  nrfx_timer.o
    0x00002f3c   0x00002f3c   0x000000c0   Code   RO         1208    i.nrfx_timer_init   nrfx_timer.o
    0x00002ffc   0x00002ffc   0x00000018   Code   RO         3633    i.nvmc_config       system_nrf52.o
    0x00003014   0x00003014   0x0000003c   Code   RO         3221    i.postfix_process   nrf_log_str_formatter.o
    0x00003050   0x00003050   0x00000006   Code   RO         2358    i.ppi_ch_disable    nrf_libuarte_drv.o
    0x00003056   0x00003056   0x00000006   Code   RO         2359    i.ppi_ch_enable     nrf_libuarte_drv.o
    0x0000305c   0x0000305c   0x00000038   Code   RO         2360    i.ppi_channel_configure  nrf_libuarte_drv.o
    0x00003094   0x00003094   0x0000011c   Code   RO         2361    i.ppi_configure     nrf_libuarte_drv.o
    0x000031b0   0x000031b0   0x0000004a   Code   RO         2362    i.ppi_free          nrf_libuarte_drv.o
    0x000031fa   0x000031fa   0x00000002   PAD
    0x000031fc   0x000031fc   0x00000058   Code   RO         2363    i.ppi_group_configure  nrf_libuarte_drv.o
    0x00003254   0x00003254   0x00000098   Code   RO         3222    i.prefix_process    nrf_log_str_formatter.o
    0x000032ec   0x000032ec   0x00000018   Code   RO         2629    i.queue_utilization_get  nrf_queue.o
    0x00003304   0x00003304   0x00000034   Code   RO         2221    i.rx_buffer_schedule  nrf_libuarte_async.o
    0x00003338   0x00003338   0x00000050   Code   RO         2890    i.serial_tx         nrf_log_backend_rtt.o
    0x00003388   0x00003388   0x00000098   Code   RO         3051    i.std_n             nrf_log_frontend.o
    0x00003420   0x00003420   0x00000038   Code   RO         1507    i.timer_req_schedule  app_timer2.o
    0x00003458   0x00003458   0x00000006   Code   RO         2222    i.tmr_evt_handler   nrf_libuarte_async.o
    0x0000345e   0x0000345e   0x00000002   Code   RO         2365    i.tmr_evt_handler   nrf_libuarte_drv.o
    0x00003460   0x00003460   0x00000010   Code   RO         2366    i.tx_ppi_disable    nrf_libuarte_drv.o
    0x00003470   0x00003470   0x0000008c   Code   RO            7    i.uart_event_handler  main.o
    0x000034fc   0x000034fc   0x000000d0   Code   RO         2223    i.uart_evt_handler  nrf_libuarte_async.o
    0x000035cc   0x000035cc   0x000000b4   Code   RO         2175    i.unsigned_print    nrf_fprintf_format.o
    0x00003680   0x00003680   0x00000010   Data   RO           20    .constdata          main.o
    0x00003690   0x00003690   0x000000a0   Data   RO           21    .constdata          main.o
    0x00003730   0x00003730   0x00000010   Data   RO           22    .constdata          main.o
    0x00003740   0x00003740   0x00000004   Data   RO          310    .constdata          boards.o
    0x00003744   0x00003744   0x00000130   Data   RO          950    .constdata          nrfx_ppi.o
    0x00003874   0x00003874   0x00000014   Data   RO         1510    .constdata          app_timer2.o
    0x00003888   0x00003888   0x00000010   Data   RO         2176    .constdata          nrf_fprintf_format.o
    0x00003898   0x00003898   0x00000034   Data   RO         2224    .constdata          nrf_libuarte_async.o
    0x000038cc   0x000038cc   0x0000003c   Data   RO         2367    .constdata          nrf_libuarte_drv.o
    0x00003908   0x00003908   0x0000012c   Data   RO         2855    .constdata          nrf_strerror.o
    0x00003a34   0x00003a34   0x0000000c   Data   RO         2892    .constdata          nrf_log_backend_rtt.o
    0x00003a40   0x00003a40   0x00000006   Data   RO         2893    .constdata          nrf_log_backend_rtt.o
    0x00003a46   0x00003a46   0x00000002   PAD
    0x00003a48   0x00003a48   0x0000000c   Data   RO         3056    .constdata          nrf_log_frontend.o
    0x00003a54   0x00003a54   0x00000081   Data   RO         3706    .constdata          mc_w.l(ctype_o.o)
    0x00003ad5   0x00003ad5   0x00000003   PAD
    0x00003ad8   0x00003ad8   0x00000004   Data   RO         3707    .constdata          mc_w.l(ctype_o.o)
    0x00003adc   0x00003adc   0x000003bf   Data   RO         2856    .conststring        nrf_strerror.o
    0x00003e9b   0x00003e9b   0x00000001   PAD
    0x00003e9c   0x00003e9c   0x00000066   Data   RO         3223    .conststring        nrf_log_str_formatter.o
    0x00003f02   0x00003f02   0x00000002   PAD
    0x00003f04   0x00003f04   0x00000006   Data   RO          418    .conststrlit        nrf_drv_clock.o
    0x00003f0a   0x00003f0a   0x00000002   PAD
    0x00003f0c   0x00003f0c   0x00000006   Data   RO          811    .conststrlit        nrfx_clock.o
    0x00003f12   0x00003f12   0x00000002   PAD
    0x00003f14   0x00003f14   0x00000004   Data   RO          951    .conststrlit        nrfx_ppi.o
    0x00003f18   0x00003f18   0x00000004   Data   RO         1086    .conststrlit        nrfx_rtc.o
    0x00003f1c   0x00003f1c   0x00000006   Data   RO         1215    .conststrlit        nrfx_timer.o
    0x00003f22   0x00003f22   0x00000002   PAD
    0x00003f24   0x00003f24   0x0000000a   Data   RO         1511    .conststrlit        app_timer2.o
    0x00003f2e   0x00003f2e   0x00000002   PAD
    0x00003f30   0x00003f30   0x0000000f   Data   RO         2225    .conststrlit        nrf_libuarte_async.o
    0x00003f3f   0x00003f3f   0x00000001   PAD
    0x00003f40   0x00003f40   0x00000009   Data   RO         2368    .conststrlit        nrf_libuarte_drv.o
    0x00003f49   0x00003f49   0x00000003   PAD
    0x00003f4c   0x00003f4c   0x00000009   Data   RO         2802    .conststrlit        nrf_sortlist.o
    0x00003f55   0x00003f55   0x00000003   PAD
    0x00003f58   0x00003f58   0x00000010   Data   RO         2990    .conststrlit        nrf_log_default_backends.o
    0x00003f68   0x00003f68   0x00000004   Data   RO         3057    .conststrlit        nrf_log_frontend.o
    0x00003f6c   0x00003f6c   0x00000020   Data   RO         3767    Region$$Table       anon$$obj.o
    0x00003f8c   0x00003f8c   0x00000010   Data   RO         2992    log_backends        nrf_log_default_backends.o
    0x00003f9c   0x00003f9c   0x00000008   Data   RO          419    log_const_data      nrf_drv_clock.o
    0x00003fa4   0x00003fa4   0x00000008   Data   RO          813    log_const_data      nrfx_clock.o
    0x00003fac   0x00003fac   0x00000008   Data   RO          953    log_const_data      nrfx_ppi.o
    0x00003fb4   0x00003fb4   0x00000008   Data   RO         1088    log_const_data      nrfx_rtc.o
    0x00003fbc   0x00003fbc   0x00000008   Data   RO         1216    log_const_data      nrfx_timer.o
    0x00003fc4   0x00003fc4   0x00000008   Data   RO         1514    log_const_data      app_timer2.o
    0x00003fcc   0x00003fcc   0x00000008   Data   RO         2226    log_const_data      nrf_libuarte_async.o
    0x00003fd4   0x00003fd4   0x00000008   Data   RO         2370    log_const_data      nrf_libuarte_drv.o
    0x00003fdc   0x00003fdc   0x00000008   Data   RO         2803    log_const_data      nrf_sortlist.o
    0x00003fe4   0x00003fe4   0x00000008   Data   RO         3061    log_const_data      nrf_log_frontend.o
    0x00003fec   0x00003fec   0x00000028   Data   RO           28    nrf_balloc          main.o
    0x00004014   0x00004014   0x00000014   Data   RO         3062    nrf_balloc          nrf_log_frontend.o
    0x00004028   0x00004028   0x0000003c   Data   RO           29    nrf_queue           main.o


    Execution Region RW_IRAM1 (Exec base: 0x20000000, Load base: 0x00004064, Size: 0x000030e8, Max: 0x00040000, ABSOLUTE)

    Exec Addr    Load Addr    Size         Type   Attr      Idx    E Section Name        Object

    0x20000000   0x00004064   0x00000026   Data   RW           23    .data               main.o
    0x20000026   0x0000408a   0x00000003   Data   RW           24    .data               main.o
    0x20000029   0x0000408d   0x00000003   PAD
    0x2000002c   0x00004090   0x00000008   Data   RW           25    .data               main.o
    0x20000034   0x00004098   0x00000003   Data   RW           26    .data               main.o
    0x20000037   0x0000409b   0x00000001   PAD
    0x20000038   0x0000409c   0x00000008   Data   RW           27    .data               main.o
    0x20000040   0x000040a4   0x00000008   Data   RW          812    .data               nrfx_clock.o
    0x20000048   0x000040ac   0x00000008   Data   RW          952    .data               nrfx_ppi.o
    0x20000050   0x000040b4   0x00000010   Data   RW         1087    .data               nrfx_rtc.o
    0x20000060   0x000040c4   0x00000020   Data   RW         1512    .data               app_timer2.o
    0x20000080   0x000040e4   0x00000004   Data   RW         1513    .data               app_timer2.o
    0x20000084   0x000040e8   0x00000004   Data   RW         1635    .data               app_util_platform.o
    0x20000088   0x000040ec   0x0000000c   Data   RW         1715    .data               drv_rtc.o
    0x20000094   0x000040f8   0x00000008   Data   RW         2369    .data               nrf_libuarte_drv.o
    0x2000009c   0x00004100   0x00000001   Data   RW         2894    .data               nrf_log_backend_rtt.o
    0x2000009d   0x00004101   0x00000003   PAD
    0x200000a0   0x00004104   0x00000008   Data   RW         2991    .data               nrf_log_default_backends.o
    0x200000a8   0x0000410c   0x00000004   Data   RW         3058    .data               nrf_log_frontend.o
    0x200000ac   0x00004110   0x00000008   Data   RW         3059    .data               nrf_log_frontend.o
    0x200000b4   0x00004118   0x00000008   Data   RW         3060    .data               nrf_log_frontend.o
    0x200000bc   0x00004120   0x00000040   Data   RW         3224    .data               nrf_log_str_formatter.o
    0x200000fc   0x00004160   0x00000004   Data   RW         3635    .data               system_nrf52.o
    0x20000100        -       0x00000040   Zero   RW            9    .bss                main.o
    0x20000140        -       0x00000010   Zero   RW           10    .bss                main.o
    0x20000150        -       0x0000000c   Zero   RW           11    .bss                main.o
    0x2000015c        -       0x00000300   Zero   RW           12    .bss                main.o
    0x2000045c        -       0x00000050   Zero   RW           13    .bss                main.o
    0x200004ac        -       0x00000040   Zero   RW           14    .bss                main.o
    0x200004ec        -       0x00000010   Zero   RW           15    .bss                main.o
    0x200004fc        -       0x0000000c   Zero   RW           16    .bss                main.o
    0x20000508        -       0x00000300   Zero   RW           17    .bss                main.o
    0x20000808        -       0x00000058   Zero   RW           18    .bss                main.o
    0x20000860        -       0x0000000c   Zero   RW           19    .bss                main.o
    0x2000086c        -       0x00000014   Zero   RW          413    .bss                nrf_drv_clock.o
    0x20000880        -       0x00000018   Zero   RW         1213    .bss                nrfx_timer.o
    0x20000898        -       0x00000010   Zero   RW         1508    .bss                app_timer2.o
    0x200008a8        -       0x00000040   Zero   RW         2891    .bss                nrf_log_backend_rtt.o
    0x200008e8        -       0x000000c0   Zero   RW         3052    .bss                nrf_log_frontend.o
    0x200009a8        -       0x00000080   Zero   RW         3053    .bss                nrf_log_frontend.o
    0x20000a28        -       0x00000018   Zero   RW         3054    .bss                nrf_log_frontend.o
    0x20000a40        -       0x00000420   Zero   RW         3055    .bss                nrf_log_frontend.o
    0x20000e60        -       0x00000288   Zero   RW         3300    .bss                segger_rtt.o
    0x200010e8        -       0x00002000   Zero   RW         3621    STACK               arm_startup_nrf52840.o


==============================================================================

Image component sizes


      Code (inc. data)   RO Data    RW Data    ZI Data      Debug   Object Name

        22          0          0          0          0       2545   app_error.o
         0          0          0          0          0        392   app_error_handler_keil.o
       132         46          0          0          0      30889   app_error_weak.o
       260         22         38         36         16      11552   app_timer2.o
        44         10          0          4          0       3420   app_util_platform.o
        36          8        512          0       8192        948   arm_startup_nrf52840.o
        72         10          4          0          0       6823   boards.o
        54          4          0         12          0      37216   drv_rtc.o
       392         48        292         60       1900     101931   main.o
       244          0          0          0          0       3693   nrf_atfifo.o
       294          0          0          0          0       8007   nrf_atomic.o
       152          0          0          0          0       3628   nrf_balloc.o
       238         28         14          0         20      12897   nrf_drv_clock.o
        50          0          0          0          0       3585   nrf_fprintf.o
       866          4         16          0          0       6618   nrf_fprintf_format.o
      1342         44         75          0          0      71166   nrf_libuarte_async.o
      1902         44         77          8          0      77644   nrf_libuarte_drv.o
       112         18         18          1         64       6249   nrf_log_backend_rtt.o
       200          0          0          0          0      10981   nrf_log_backend_serial.o
        28          4         32          8          0       3373   nrf_log_default_backends.o
      1490        130         44         20       1400      31542   nrf_log_frontend.o
       570        108        102         64          0       5736   nrf_log_str_formatter.o
       346          0          0          0          0       8219   nrf_memobj.o
         0          0          0          0          0       1472   nrf_nvic.o
       424          0          0          0          0      14053   nrf_queue.o
        28          0          0          0          0       2411   nrf_ringbuf.o
         0          0         17          0          0       1085   nrf_sortlist.o
        76         10       1259          0          0       2795   nrf_strerror.o
       226         28         14          8          0      47241   nrfx_clock.o
      1680        674        316          8          0      22308   nrfx_ppi.o
       480         28         12         16          0      15306   nrfx_rtc.o
       408         28         14          0         24      15501   nrfx_timer.o
       378         34          0          0        648       9198   segger_rtt.o
       500         66          0          4          0      31617   system_nrf52.o

    ----------------------------------------------------------------------
     13078       1396       2908        256      12264     612041   Object Totals
         0          0         32          0          0          0   (incl. Generated)
        32          0         20          7          0          0   (incl. Padding)

    ----------------------------------------------------------------------

      Code (inc. data)   RO Data    RW Data    ZI Data      Debug   Library Member Name

         8          4        133          0          0         68   ctype_o.o
         0          0          0          0          0          0   entry.o
         0          0          0          0          0          0   entry10a.o
         0          0          0          0          0          0   entry11a.o
         8          4          0          0          0          0   entry2.o
         4          0          0          0          0          0   entry5.o
         0          0          0          0          0          0   entry7b.o
         0          0          0          0          0          0   entry8b.o
         8          4          0          0          0          0   entry9a.o
        30          0          0          0          0          0   handlers.o
        36          8          0          0          0         68   init.o
        30          0          0          0          0         68   llshl.o
        32          0          0          0          0         68   llushr.o
        36          0          0          0          0         68   memcpya.o
        36          0          0          0          0        108   memseta.o
        18          0          0          0          0         68   strcpy.o
        14          0          0          0          0         68   strlen.o
        98          0          0          0          0         92   uldiv.o

    ----------------------------------------------------------------------
       362         20        136          0          0        676   Library Totals
         4          0          3          0          0          0   (incl. Padding)

    ----------------------------------------------------------------------

      Code (inc. data)   RO Data    RW Data    ZI Data      Debug   Library Name

       358         20        133          0          0        676   mc_w.l

    ----------------------------------------------------------------------
       362         20        136          0          0        676   Library Totals

    ----------------------------------------------------------------------

==============================================================================


      Code (inc. data)   RO Data    RW Data    ZI Data      Debug   

     13440       1416       3044        256      12264     596713   Grand Totals
     13440       1416       3044        256      12264     596713   ELF Image Totals
     13440       1416       3044        256          0          0   ROM Totals

==============================================================================

    Total RO  Size (Code + RO Data)                16484 (  16.10kB)
    Total RW  Size (RW Data + ZI Data)             12520 (  12.23kB)
    Total ROM Size (Code + RO Data + RW Data)      16740 (  16.35kB)

==============================================================================

